:020000040800F2
:10400000005000206DDD0008EDB20008EFB200089E
:10401000F1B20008F3B20008F5B200080000000099
:10402000000000000000000000000000F9B20008DD
:10403000F7B2000800000000FBB20008B1960008CB
:10404000FDB20008FFB2000801B3000803B3000886
:1040500005B3000807B3000809B300080BB3000854
:104060000DB300080FB3000811B3000800000000F2
:104070000000000000000000000000000000000040
:10408000000000000000000021B3000823B3000876
:104090002DB3000839B3000845B3000851B3000838
:1040A00053B3000855B3000857B3000859B30008CC
:1040B0005BB300085DB300085FB3000861B300089C
:1040C00063B3000865B3000867B3000869B300086C
:1040D0006BB30008258F00086FB3000871B30008A8
:1040E00073B3000875B3000877B300080000000040
:1040F00000000000000000000000000000000000C0
:0C41000000000000000000005FF800005C
:1041100030BF704720BF704740BF7047BFF36F8FFD
:104120007047BFF34F8F7047BFF35F8F704701DF5A
:104130007047EFF31480704780F31488BFF36F8FDC
:104140007047EFF30980704780F309887047EFF3F9
:104150000880704780F30888704772B6704762B66F
:10416000704771B6704761B6704780F31188704729
:10417000EFF31280704740BA704700BA70470000F2
:104180000C4B10B59B680C4C13F480530B480C4936
:104190000C4A07D0012323700B4B03600B480860C7
:1041A000136010BD23700A4B03600A4B0B600A4B6F
:1041B000F6E700BF000C0140A80E0020B40E00205E
:1041C000080F0020BC0E00209D960008379C0008B8
:1041D000F9910008A19000084D910008000000002E
:1041E0002DE9F3410121484808F0D2F901210420CA
:1041F00008F0B6FC032510264AF21003434C01A92F
:104200002046ADF804308DF807608DF8065008F0B0
:104210002CF94FF420434FF0040826616361062314
:104220000DEB08012046ADF804308DF807808DF8BD
:10423000065008F01AF90121082008F091FC40F618
:10424000FC43334F0DEB08013846ADF804308DF8D0
:1042500007608DF8065008F008F940F618433B61F6
:10426000E4237B614FF480530DEB08018DF8078048
:104270004FF440483846ADF8043007F580678DF8B4
:10428000065008F0F2F83046012108F069FC01A957
:1042900038468DF80760ADF804808DF806504FF46D
:1042A000005608F0E2F84823C7F8148001A9384600
:1042B0008DF80730ADF804608DF8065008F0D5F899
:1042C0000121144808F064F900230A211A466661A6
:1042D000A06826614504A06858BF0132400448BF69
:1042E00001330139F3D10A2A0B4A0AD10A2B08D12A
:1042F000012301210448137008F04AF902B0BDE817
:10430000F0810023F5E700BF000230000008014003
:10431000000C014000043000B90E0020F7B5114B2D
:104320001B78E3B14FF400610F4B0F464FF48060F0
:1043300000241E460D4D5F6118610194019AAA4246
:1043400009D9316170610194019AAA42F3D8019AA6
:1043500001320192F8E7019A01320192EEE703B0CF
:10436000F0BD00BFB90E0020000C01403F0D03005E
:1043700010B90422014B5A61704700BF000C014084
:1043800010B90422014B1A61704700BF000C0140B4
:1043900010B50021044644FA01F3DB07C8B205D585
:1043A000FFF7EEFF01310829F5D110BDFFF7E0FF5F
:1043B000F8E7012808B50ED003D3022810D000205A
:1043C00008BD002005F068FA40F24C43984294BFC3
:1043D0000020012008BD054B9868C0F3800008BD8F
:1043E000024B9868C0F3400008BD00BF00080140C0
:1043F00020B9034BD868C0F3800070470020704795
:10440000000C014070B5002401262546E0B2FFF7FC
:10441000D0FF18B106FA04F31D43EDB20134082CA5
:10442000F4D1284670BD08B108F0D6B908F0DCB95F
:1044300062B6704772B6704708B9014B1870704782
:104440006805002050B9064B5A6842F040525A6045
:104450004FF400425A610122024B1A70704700BFAC
:1044600000100140680500204022064B10F0010FAB
:1044700014BF5A611A61802210F0020F14BF5A61F2
:104480001A617047000C0140074B9A88C2F307225B
:10449000042A06D19A88D2B2D82A02D1188980B2C9
:1044A00070470020704700BF006C004038B5254BB6
:1044B000254C9D6815F4005501D0606838BD05F0A5
:1044C00043F9217B2A46A06000290CBFFF2100216F
:1044D000022000F0BFFB217B0546012200290CBF12
:1044E000FF210021022000F0B5FB237B40EA0520DC
:1044F000A3B110F4804318BF012301046FEA000048
:10450000637348BF637BC0F3090044BF43F00203F9
:104510006373236923EA0000606038BD10F0020372
:1045200018BF012380086373C20442BF637B43F05A
:1045300002036373830442BF637B43F0040363732A
:10454000E7E700BF001001406805002038B54C4B7C
:104550009B689B0451D4FFF7A9FF4A4B5A699042CC
:104560005CDD9969821A8A42474C0BDA2168D3E9EB
:1045700008455143641845EBE175996AC3E908455C
:104580000A4449E093F82C104D0737D51A6924687E
:10459000821A5443E517C3E908459A6200240025AE
:1045A000C3E90C4521F0040183F82C109A6B9D6A35
:1045B000AC1A84EAE471DA6BA1EBE471914253D94D
:1045C0009A68196C511A64294ED91A6442F2107211
:1045D000624392FBF1F13C224A4319699D63013128
:1045E00092FBF1F240F6B831002A5A64B8BF524249
:1045F0008A4228DDC822DA63586138BD1969013161
:104600008A1A2168D3E908455143641A65EBE175BC
:10461000C3E90845996A8A1A9A62C7E7C6DA9969AE
:10462000121A8A42184CECDB93F82C104D0706D571
:10463000246898624443E517C3E90845AEE7196961
:1046400001318A1A92E7B2F57A7F01DD6422D2E75E
:10465000322A01DD0A22CEE70A2A01DD0522CAE755
:10466000012AC9DD0122C6E79A68196C521AB2F50F
:10467000FA6F81BF0122DA6300225A64BCE700BFEF
:1046800000100140680500200400002008B568B94A
:10469000FFF75CFF0649D1E90823D1E90C01121AA2
:1046A00063EB0103100A40EA036008BD002008BD67
:1046B0006805002038B50D46E0B9114CFFF746FFFC
:1046C000D4E908012269002871F100034FEA0222AF
:1046D0004FEAE2730FDB0BF047FBC4E90C23E91749
:1046E0000B022A02D4E90C0143EA156312184B416C
:1046F000C4E9082338BD404261EB4101EBE700BF4C
:104700006805002010B9024B09011960704700BF0D
:104710000400002010B9024B83F82C10704700BF32
:1047200068050020014B586C704700BF68050020E9
:1047300010B9024B587B7047002070476805002075
:1047400070B5012000F0FAFA00220220114600F0B4
:1047500081FA01220021022000F07CFA642400BFCB
:10476000013CFCD122462146022000F073FA21468A
:104770000122022000F06EFA642400BF013CFCD14B
:104780002246A021022000F065FA214601220220E3
:1047900000F060FA2246A021022000F05BFA2146D8
:1047A0000122022000F056FA00F00F000B2808BF8B
:1047B00001232D4C08BF2373257B002D4DD12846A6
:1047C00000F0BCFA2A46FE21022000F043FA012242
:1047D0004021022000F03EFA2A462946022000F03D
:1047E00039FA01222946022000F034FA2A46FE2135
:1047F000022000F02FFA01224021022000F02AFAC4
:104800002A462946022000F025FA064601222946BA
:10481000022000F01FFA082E0BBF40F6FF7340F293
:10482000FF33236123610CBF4FF400634FF4007327
:104830000022E7210220A36100F00CFA01220021EE
:10484000022000F007FAFFF731FE60610002C11795
:10485000C4E90C01C4E9080170BD40F2FF332361D3
:104860004FF40073A361EEE76805002008B5082047
:1048700005F012F859281BD9184B93F8482012B9A3
:10488000012283F84820082005F006F8592817D996
:10489000124B1B78A3B903F1804303F588335A68A0
:1048A00022F030425A605A6842F080425A6008BD95
:1048B000082004F0F1FF4F28E5D80022074BE0E77D
:1048C000082004F0E9FF4F2807D8054B5A6842F04A
:1048D00040525A604FF400425A6108BD68050020FA
:1048E00000100140044B93F84800013801288CBFA8
:1048F00000200120704700BF68050020044B93F89A
:10490000480001280ABF0222002083F8482070478F
:104910006805002008B5FFF7C9FD052808D9FFF78D
:10492000C5FD40F2F933984294BF0020012008BD34
:10493000012008BD37B5144B4FF4804298B95A6135
:104940000623ADF8043003238DF80630042300F16C
:1049500080400DEB030100F584308DF8073007F03F
:1049600084FD03B030BD1A61032302258DF80630A3
:104970001023064C01A92046ADF804508DF80730ED
:1049800007F073FD6561ECE700100140000801408D
:1049900008B540B904F080FF40F24C43984294BF00
:1049A0000020012008BD002008BD18B9024B93F873
:1049B0002C00704700207047680500204FF48032BB
:1049C0003A21002005F0C8BF2DE9F743484D0446C1
:1049D00005EB4015AB680BB16E8B96B938212046BC
:1049E00005F0E4FF382120F48062204605F0B4FF92
:1049F0004FF480323A21204603B0BDE8F04305F081
:104A0000ABBF06F06CF9C0F1080006FA00F00AF03E
:104A10009FFBAD68064685EAE570A0EBE5700F46A2
:104A20000AF096FB02460B46304639460AF020FD56
:104A3000304B002206460F460AF0F0FB6A468046DD
:104A400089460BF035FC002200230AF04FFEA0B18E
:104A5000494640460AF092FE002D06464FF03801C6
:104A6000B8BF4642204605F0A1FF382120F48062FD
:104A7000204605F071FF3246BCE7304639466A46AB
:104A80000BF016FC002D06460F46DDE9000118DD8F
:104A90000AF074FE14A3D3E9002305043946304616
:104AA0000AF0BCFB0AF06AFE05433821204605F0F7
:104AB0007DFF382140F48062204605F04DFF2A46F4
:104AC00098E70AF05BFE08A3D3E90023C543394603
:104AD00030460AF0A3FB0AF051FEC0F51C502D042D
:104AE0001030E1E7AFF30080000000000088C34011
:104AF000000A00200000F04010B5044606F0EFF870
:104B0000054BC0F1080053F820102046BDE81040C6
:104B10004909FFF7F7BD00BFA40A01082DE9F04FCE
:104B20000024474B89B001214FF480401C7008F0ED
:104B300023F80121084608F013F803264FF4204318
:104B40004FF0180A3F4D02A92846ADF808308DF8FD
:104B50000BA04FF0040B8DF80A6007F086FC4FF4B1
:104B6000804302A92846ADF808308DF80A608DF818
:104B70000BB007F07AFC102301254FF482794FF037
:104B800002084FF40077ADF818302F4B03A91846F0
:104B9000ADF80C40ADF81040ADF81A40ADF81C402F
:104BA0000193ADF80E90ADF81280ADF81450ADF849
:104BB000167008F08DF8019B2946184608F00CF98C
:104BC00029464FF4805007F0CBFF2146284607F0D6
:104BD000DFFCA0238DF80BA0DFF874A002A95046DB
:104BE000ADF808308DF80A6007F03FFC402302A9B9
:104BF0005046ADF808308DF80A608DF80BB007F01C
:104C000034FC0823ADF80C40ADF81040ADF81A4064
:104C1000ADF81C400D4C03A92046ADF81830ADF896
:104C20000E90ADF81280ADF81450ADF8167008F083
:104C30004FF82946204608F0CFF809B0BDE8F08FBC
:104C4000B1050020000C0140003800400030014058
:104C5000000801400128F8B505460E4614462ED03E
:104C600003D302282DD000245BE010222E4B2F4FBF
:104C70005A610221384608F031F90028F9D031464E
:104C80002A4808F0D7F8294E0121304608F026F9C5
:104C90000028F9D0002C40D0012D3CD033D3022D78
:104CA000E1D11022224B1A61224B1B782BB9224AE8
:104CB00013889BB243F0020313801F4827E00822A9
:104CC000D4E71C4B1B7833B91B4A138823F002032B
:104CD0001B041B0C13801022154B174D5A61022127
:104CE000284608F0FBF80028F9D03146124808F0B1
:104CF000A1F8114D0121284608F0F0F80028F9D05C
:104D0000002CDAD0CDE71022074B1A61074808F0D3
:104D100093F8C4B205E00822F6E7012DF6D9022D7A
:104D2000CBD02046F8BD00BF000C01400038004049
:104D300000080140B105002000300140084A09493F
:104D4000138838B123F003031B041B0C13800123C9
:104D50000B7070479BB243F00303138008707047D9
:104D600000300140B1050020044B9A78044B12B189
:104D700004221A7070470322FBE700BF280A0020B4
:104D80009C0A0020002330B519464FF0FF350D4A2C
:104D90000D4813705370141D44F82350C15401334F
:104DA0002F2BF9D1094B82F8C0101960084B82F8FB
:104DB000CC101960074BC2F8C410C2F8C8101960B3
:104DC00030BD00BFB40500200C0F0020880A002071
:104DD000A40A0020300A0020F7B56B4CA57815B165
:104DE0006378022B6AD10026684B5E55684B5E558E
:104DF0006378012B2CD003D3022B6DD00322BFE0AC
:104E0000644F7B5D53B1644B272103EB8503D3F8DB
:104E1000D020284605F0A0FDA378FE54A0785F4D71
:104E20002B5C43B15E4B262153F8202005F094FD06
:104E30000022A378EA542D21D4F80320A07805F0AD
:104E40008BFD0023A078019300931A46202170E087
:104E5000514F7A1992F8D420012A37D030D3022A40
:104E600036D0A0784B4D2B5C4BB107EB8003D3F8C9
:104E7000D020272105F070FD0022A378EA54A07805
:104E8000464D2B5C43B1464B262153F8202005F0BC
:104E900063FD0022A378EA54D4F803302D211E4488
:104EA0003246A07805F058FD0023A07801930093C6
:104EB0001A46202105F01CFD3A4B5E6003B0F0BDA0
:104EC0002D21284605F072FD0646CAE72121F8E7A4
:104ED0002846FFF7DBFBF7E7D4F80330142B4EDC52
:104EE0002A0629D5EB07E9D52A4D2B783BB12A4B69
:104EF0002721D3F8D020304605F02EFD2E70274D07
:104F00002B783BB1264B26211A68002005F024FDA2
:104F100000232B70244BD4F803202D2153F822209A
:104F2000002005F019FD002320211A4618460193A0
:104F3000009305F0DDFCC1E70DBB164E337843B19D
:104F4000154B2721D3F8D020284605F005FDA3787E
:104F5000F554A078114D2B5C43B1114B262153F829
:104F6000202005F0F9FC0022A378EA54A078D4F8B8
:104F700003300D4A034452F823202D215FE7042219
:104F8000084B1A709AE700BF280A0020B20E0020D2
:104F9000FC090020F5090020B4050020240A0020A7
:104FA000200A00209C0A0020340A002073B5CE4D50
:104FB000AE786A782C461EB10422CC4B1A7009E2F6
:104FC000A52A00F06F8300F2C480152A00F05682F3
:104FD00057D80C2A00F000822ED8042A00F0BD8198
:104FE0000AD8012A00F09981002A00F08D81022A56
:104FF00000F097810322E0E7062A00F0D481C0F098
:10500000C381072AF6D11021002005F0CFFC03460A
:10501000EA78A878D2080192C3F307220092C3F37A
:1050200007430022102105F063FCAA78B04B03EB84
:105030004213EA785A77CDE1102A00F0FB810DD8AF
:105040000E2A00F0E88140F2D781AA4BD5F8030080
:10505000D3F8DC3098472421024658E1122A00F0A8
:10506000FB81C0F0F081132A00F0FF81142AC1D126
:10507000A04BD5F80300D3F8D83098472B2102462F
:1050800045E1202A00F04D8233D8192A00F0198218
:1050900012D8172A00F0098240F2F481342100204E
:1050A00005F084FCD5F803300246A878002B00F008
:1050B000058242F008029AE11B2A00F02082C0F02B
:1050C0000F821C2A00F024821F2A93D11021002075
:1050D00005F06CFC0246D1B2C2F30722EB78A87847
:1050E000019100921021002203F00F0305F000FC53
:1050F00070E1A02A00F0B68217D87F2A00F0228241
:105100008C2A00F02982212A7FF474AF6E210020BE
:1051100005F04CFC0246D1B2C2F30722EB78A87826
:10512000019100926E210022E0E7A22A00F0A882FD
:10513000C0F09F82A32A00F0AC82A42A7FF45AAF69
:105140000020D5F80310C9B202B0BDE8704005F0E8
:105150003BBDBF2A00F05C8353D8AE2A00F0F68234
:1051600025D8A92A00F0CE820DD8A72A00F0C18246
:1051700040F2AC820020D5F80310C9B202B0BDE8FD
:10518000704005F057BEAB2A00F0CE82C0F0C3825B
:10519000AC2A00F0D282AD2A7FF42CAF0020D5F8E3
:1051A0000310C9B202B0BDE8704005F055BEB82A80
:1051B00000F0F48211D8B52A00F0D182B62A00F0AE
:1051C000DA82B12A7FF416AF0020D5F80310C9B2F5
:1051D00002B0BDE8704005F09DBCBA2A00F0F08234
:1051E000C0F0E582BB2A00F0FE82BC2A7FF402AF49
:1051F0000020D5F80310C9B202B0BDE8704005F038
:10520000CABED22A00F0CD8133D8C32A00F0BA81B9
:105210000DD8C12A00F0B18140F20383354BD5F897
:105220000300D3F8D8309847314B1860D2E0CA2A2F
:1052300000F0B1810FD8C92A7FF4DCAE38210020FC
:1052400005F0B4FBD5F8033000F4806223F48063EA
:105250001A433821A5E0CC2A00F0EC82D12A7FF451
:10526000C9AE0020D5F8031002B0BDE87040FFF7CA
:1052700021BAD92A00F0B0810DD8D62A00F0988141
:10528000D82A00F0A581D42A7FF4B4AED5F8032043
:10529000174BDA609EE0FB2A00F0A88107D8DA2AD3
:1052A0007FF4A8AED5F80320114B1A6192E0FE2AD4
:1052B00000F0C081FF2A7FF49DAED5F80330002BAB
:1052C00000F0C381012B7FF477AE094A5376094B76
:1052D000094AC3F8D820094AC3F8E020084AC3F8AD
:1052E000DC20084ABBE100BF280A00209C0A0020FD
:1052F000000A0020B40500201DB2000881B2000899
:1053000059B20008C1B200082D21D5F803200020B1
:1053100002B0BDE8704005F01FBBD5F80320212185
:10532000F5E7D5F803302021002BC8BF012200206B
:1053300005F012FB0122AD78B74BD4F803005A55A3
:10534000B64B002803EB8503D3F8D830B8BF4042F2
:105350009847272102462846DAE7D5F80300AF4CE4
:105360000028B8BF4042D4F8D83098472021C4F86C
:10537000D000A87805F01AFB60BBA878272104EBC1
:105380008004D4F8D020C3E70022A54BD5F8030051
:105390001A70A24BD3F8DC30984726210246A14B65
:1053A0001860A078B4E71021002005F0FFFA03464A
:1053B000DAB2A8780192EA78C3F30743D2080092E0
:1053C0001021002205F094FAAA78974B03EB4213C0
:1053D000EA781A7702B070BD3421304605F0E6FA5B
:1053E000D5F803300246A8781BB942F002023421F6
:1053F0008EE722F00202FAE73421002005F0D6FA07
:10540000D5F803300246A87813B942F00102EEE75E
:1054100022F00102EBE73421002005F0C7FAD5F8AD
:1054200003300246A87813B142F01002DFE722F001
:105430001002DCE7794BD5F80300D3F8D830984751
:105440002521024663E7754BD5F80300D3F8DC301D
:105450009847282102465AE7704BD5F80300D3F845
:10546000DC3098472A21024651E76C4BD5F80300FF
:10547000D3F8D83098472321024648E7D5F80320CF
:105480002C2144E7D5F803000028FFF695AD664BC4
:105490005B7E012B01D005F0F3FE20B1634AB2FB25
:1054A000F0F215217DE7624AFBE75C4BD5F803007B
:1054B000D3F8D83098473321024628E722F0080273
:1054C00095E73421304605F071FAD5F803300246ED
:1054D000A87813B142F0040289E722F0040286E7BB
:1054E0003421002005F062FAD5F803300246A8788E
:1054F00013B142F400627AE722F4006277E70020F9
:10550000D5F80310C9B202B0BDE8704005F014BB75
:105510000020D5F80310C9B202B0BDE8704005F014
:105520001DBB6E21304605F041FAEB78AC78019353
:105530002B79324603F0030300936E21C0F3074337
:105540002046D3E5D5F80330022B3FF635ADEA7897
:10555000324B83F8D4203DE7D5F803100020C1F189
:105560000801C9B205F0C4FAA878FFF72DFAA078AF
:1055700002B0BDE87040FFF7BFBAD5F803202A4B50
:105580001A7627E7254BD5F80300D3F8D83098478B
:10559000254B58601EE7D5F80320234B00205A8383
:1055A000E3E73046E97802B0BDE87040FFF7B2B8F3
:1055B000D5F8030009F0CCFD15A3D3E9002309F0C9
:1055C00057FF0AF061FF0AF0D9F8112102469EE662
:1055D000D5F8032039219AE63046D5F80320124B3E
:1055E0009A6002B0BDE87040FFF7EEB900210846AE
:1055F00005F0DCF9D5F803100246A87819B122F0BD
:105600001002002184E642F0100281E6AFF3008030
:105610002D431CEBE236FA3FF5090020B4050020CB
:10562000240A0020200A0020000A00200024F400A0
:10563000B5001000D5F80330012B3FF6BDACE8787B
:1056400002B0BDE87040FFF775B97F4A53767F4BD3
:105650007F4AC3F8D820C3F8E020C3F8DC20C3F8A1
:10566000E420B7E63046E97802B0BDE8704005F0C6
:10567000FDBA0020E97802B0BDE8704005F0E4BA58
:105680000020D5F80310C9B202B0BDE8704005F0A3
:105690000BBA0020D5F80310C9B202B0BDE87040C3
:1056A00005F06EBA304605F036FBD5F80310AB783E
:1056B000C9B228B9184602B0BDE8704005F0C2BAB8
:1056C000184602B0BDE8704005F090BA002005F021
:1056D00022FBD5F80310C9B228B9A87802B0BDE8FA
:1056E000704005F0CFB9A87802B0BDE8704005F071
:1056F00097BA0020D5F80310C9B202B0BDE87040D7
:1057000005F0A6B93046D5F80310C9B202B0BDE81D
:10571000704005F04ABB0020D5F80310C9B202B0B2
:10572000BDE8704005F053BB0020D5F80310C9B2A6
:1057300002B0BDE8704005F026BB0020D5F803108C
:10574000C9B202B0BDE8704005F053BB3046D5F891
:105750000310C9B202B0BDE8704005F05BBBD5F8DC
:1057600003000028FFF628AC384BD3F8D830984710
:10577000354B58612EE6D5F803000028FFF61CAC27
:10578000314B5B7E012B01D005F07AFD20B1314A0F
:10579000B2FBF0F2142104E62F4AFBE73046D5F8BD
:1057A0000310C9B202B0BDE8704005F0FBB900209B
:1057B000D5F80310C9B202B0BDE8704005F086B953
:1057C000D5F803000028FFF6F7AB1F4B5B7E012BDB
:1057D00001D005F055FD20B11E4AB2FBF0F21321B5
:1057E000DFE51D4AFBE7D5F803100020C9B205F03C
:1057F000C2FB0021A87805F0D9F8D5F803100246BD
:10580000A87811B142F00402FBE622F004027FE521
:105810003046D5F80310C9B202B0BDE8704005F0BB
:1058200098BB0020D5F80310C9B202B0BDE87040A3
:1058300005F07DBB0020D5F80310C9B202B0BDE869
:10584000704005F050BB00BF000A0020B4050020E6
:10585000E9B200080024F400B500100038B5044D8A
:10586000044CAA786B783AB10423237038BD00BF8A
:10587000280A00209C0A0020FF2B00F2FB82DFE8B0
:1058800013F00001140116011F0124012B01320144
:1058900036013901400144014B0152015C016201B2
:1058A00069016E01730178017D018201870189011F
:1058B000A001A501AC01B301BA01BE01C201C90139
:1058C000C901D001D701F902F902F902F902F9027E
:1058D000F902F902F902F902F902F902F902F902F0
:1058E000F902F902F902F902F902F902F902F902E0
:1058F000F902F902F902F902F902F902F902F902D0
:10590000F902F902F902F902F902F902F902F902BF
:10591000F902F902F902F902F902F902F902F902AF
:10592000F902F902F902F902F902F902F902F9029F
:10593000F902F902F902F902F902F902F902F9028F
:10594000F902F902F902F902F902F902F902F9027F
:10595000F902F902F902F902F902F902F902F9026F
:10596000F902F902F902F902F902F902F902F9025F
:10597000F902F902F902F902F902F902F902F9024F
:10598000DD01F902F902F902F902F902F902F9025C
:10599000F902F902F902F902F902E101F902F90248
:1059A000F902F902F902F902F902F902F902F9021F
:1059B000F902F902F902F902F902F902F902F9020F
:1059C000F902460246024A024E02520256027D0285
:1059D00089028D029102950299029D02A102A502FF
:1059E000F902F902A902AD02F902AF02B602BC0245
:1059F000F902BE02C202C602CC02D002D402D60212
:105A0000E602EA02E701EA01EF01F501F801F90215
:105A1000F902F902FA01FC01F902EE02F902FF01B2
:105A20000102130219021D02F9022102F9022402E5
:105A3000F202340236023902F502F902F902F902E1
:105A4000F902F902F902F902F902F902F902F9027E
:105A5000F902F902F902F902F902F902F902F9026E
:105A6000F902F902F902F902F902F902F902F9025E
:105A7000F902F902F902F9023C02F902F902F9020B
:105A800043022D21002004F091FF6060B04B1B7891
:105A900053B1B04B62681A60AF4B002A40F0ED8101
:105AA0001A6842F008021A6038BD2121EAE727216E
:105AB000AA4BD3F8E050002004F078FFA847E4E7B1
:105AC000A64B2221D3F8E050F5E7A44BD3F8E02011
:105AD000D3F8D0009047D8E7A04BA14AD3F8E430E0
:105AE00010689847D1E79F4B1B7F6360CEE79D4BC3
:105AF0005B7FFAE73521002004F058FFC0F3402017
:105B0000C3E70020FEF744FFBFE73521002004F083
:105B10004DFFC0F34000B8E73521002004F046FFF8
:105B200000F00100B1E73421002004F03FFF10F045
:105B3000020F0CBF01230023D7E73421002004F01B
:105B400035FFC043ECE73421002004F02FFFC0F301
:105B500000109AE7814B2421D3F8E450ABE77F4B48
:105B60002521D3F8E050A6E77C4B2821D3F8E45058
:105B7000A1E77A4B2A21D3F8E4509CE7774B232105
:105B8000D3F8E05097E7754B2B21D3F8E05092E71C
:105B90002C2177E71521002004F008FF002800F0F1
:105BA0003881714BB3FBF0F06060AA786D4B03EB6A
:105BB00042135B7E002B7FF469AF606805F02EFB1B
:105BC00063E7664B3321D3F8E05074E734210020BB
:105BD00004F0ECFEC0F3C00057E73421002004F0CD
:105BE000E5FEC0F3800050E73421002004F0DEFE23
:105BF000C0F3C02049E7002005F07FF845E700200A
:105C000005F082F841E7554B0020D3F8E05004F04E
:105C1000CDF953E71021002004F0C8FEC0F3034083
:105C200033E76E21002004F0C1FEC0F309002CE729
:105C30006E21002004F0BAFE000C26E7474B93F8D3
:105C4000D43052E7002005F04AF8C0F108001CE704
:105C5000444B1B7E49E7414B424AD3F8E0303FE7D3
:105C60003E4B404AD3F8E03050683AE73F4B1B6860
:105C70003BE73F4BFBE7382104E73A4B5B8B34E7CC
:105C80006F21CFE700223B4B6260197809B10121F7
:105C900061601A70384B1A781AB1626842F00202D9
:105CA000626000221A70F1E66F21002004F07EFE8F
:105CB000000EEAE60020FEF7E9FCE6E60020FEF72B
:105CC00074FEE2E6274BDB680FE71121002004F0A9
:105CD0006DFE09F03DFA1CA3D3E9002309F09EFAFA
:105CE0000AF042FB09F04AFDCFE63921CAE61D4B16
:105CF0009B68FAE61B4B1B69F7E60021084604F097
:105D000055FE10F0100F14E7164B5B7EEDE60020F9
:105D100005F032F8B9E6002004F0D3FFB5E6002024
:105D200004F0F9FFB1E6002005F003F8ADE600202D
:105D300004F0F1FF18B9A87805F015F8A5E6A878E1
:105D400004F0FEFFA1E600BF2D431CEBE236FA3F54
:105D5000970A0020880A0020300A0020B40500209D
:105D6000200A0020000A00200024F400AC0E0020CD
:105D7000C40E0020FC090020B20E0020002004F018
:105D8000CAFF18B9A87804F095FF7EE6A87804F059
:105D9000E3FF7AE6002004F07BFF76E6002005F0C2
:105DA00094F872E6002005F070F86EE6002005F029
:105DB00073F86AE6002005F061F866E6002005F059
:105DC00072F862E6002005F087F85EE6002005F034
:105DD00071F85AE6002004F089FF56E60B2151E6DF
:105DE0006F21002004F0E2FDC0F304404DE6254B96
:105DF000254AD3F8E030506973E61421CBE6002041
:105E000004F090FF41E6002004F062FF3DE613211C
:105E1000C1E66FF07F436360C7E6002005F0E7F856
:105E200033E6002005F0EAF82FE671212AE600218A
:105E3000084604F0BBFD420707D56F21A87804F09F
:105E4000B5FD430401D501234FE600234DE60020B4
:105E500005F0C6F819E6002005F0BBF815E60020AD
:105E600005F0A9F811E6FEF721FB0EE60020FEF78B
:105E70005FFC0AE60323237008E61A6822F0080292
:105E800011E600BFB4050020000A002038B5B64B6B
:105E90009A781C46022A00F01181032A00F015812D
:105EA000002A40F097815A784D2A00F0C8802FD8F8
:105EB000462A00F0908012D8422A7CD006D8402A88
:105EC0006DD0412A72D00322A84B66E0442A77D0D5
:105ED000452AF8D1D978A64B0520597162E0492AA4
:105EE00000F096800AD8472A7DD0482AEBD1DB788B
:105EF0009F49012201F8263F262068E04B2A00F046
:105F000093804C2ADFD1D978994B0220997049E0CF
:105F1000552A00F0AF8026D8522A00F09A8011D876
:105F2000502A00F09180512ACDD1914D2A7DD2077F
:105F300004D5DB78DB0701D402F021FDE1781420E1
:105F400029752FE0532A00F08C80542ABBD1D3F856
:105F50000330012B00F23E81E3788549012201F8EC
:105F60001A3F1A2033E0832A00F097800CD8572A72
:105F700000F08C80592AA6D1D3F803307C49022244
:105F800021F8243F242022E0852A00F09180C0F0EF
:105F90008A80FF2A97D1DA78764B1A7038BD40F2A2
:105FA000FF70D978BDE8384002F082BDD978704BD7
:105FB00000201970F6E7D9786D4B01205970F1E790
:105FC00004221C20D3F80330694941F81C3FBDE886
:105FD000384002F0CCBDD3F803306549042241F8C3
:105FE0000C3F0C20F3E7624D042229460820D3F829
:105FF000033041F8083F02F0BAFD5F4B1B78002BDD
:10600000CCD12A69A9686879BDE8384003F056B94F
:10601000DA78574B1AB9DA75D97D1720C2E7012211
:106020005249DA754A60F7E7D978514C0320E1709C
:1060300002F03EFDE078BDE8384003F007B8D978BB
:106040004B4B15205975ADE7D978494B16209975FA
:10605000A8E7D3F803304649042241F8203F202026
:10606000B5E7434DD3F803302946042241F8103FE9
:106070001020C0E7D3F80320012A00F2AB80DB78C0
:106080003B49012201F81B3F1B20A0E7DB78384980
:10609000012201F8273F272099E7D3F80320374B47
:1060A000C3F8E82038BDD3F80320354B1A6038BD5B
:1060B000D3F80320314BC3F8EC2038BD5A78D3F81D
:1060C0000310304B43F8221038BD5A78282A68D084
:1060D0001DD8022A3DD00DD88AB3012A7FF4F3AE31
:1060E000D3F80320284B5A6003F02EFB234BC3F850
:1060F000F40038BD1C2A49D0272A4DD01B2A7FF432
:10610000E2AED3F80330204ADBB2137338BD2B2A3A
:1061100051D009D8292A49D02A2A7FF4D4AED3F8FD
:106120000320194BDA6138BD2D2A4ED048D32E2AD0
:106130007FF4C9AED3F80320134BDA6238BDD3F82D
:106140000320114B1A6003F0FFFA0C4BC3F8F00068
:1061500038BDD3F803200C4B9A6003F0F5FA074BD7
:10616000C3F8F80038BD00BF280A00209C0A0020B0
:1061700008000020960A0020A80E0020B405002088
:10618000980A0020A80A0020C80E0020D3F8033087
:10619000114ADBB2537338BDD3F803200E4B1A619A
:1061A00038BDD3F803200C4B5A6138BDD3F8032017
:1061B000094B9A6138BDD3F80320074B1A6238BDEA
:1061C000D3F80320044B5A6238BDD3F80320024BA6
:1061D0009A6238BD042277E6C80E002073B51E4CC3
:1061E000A578002D34D11D4B1D4E1D701D4B1D700B
:1061F00033783BB11C4B26211A68284604F0ACFBCF
:10620000A378F5540126A578184BD4F803005E5501
:10621000174B002803EB8503D3F8D830B8BF4042B2
:10622000984727210246284604F096FBD4F803300D
:10623000A078002BD8BF02224FF00003D4BF0192F8
:10624000019600931A46202104F052FB02B070BD63
:106250000422084B1A70F9E7280A0020B20E002029
:10626000240A0020FC090020200A0020F509002053
:10627000B40500209C0A002073B51E4CA578002DA3
:1062800034D11D4B1D4E1D701D4B1D7033783BB11D
:106290001C4B26211A68284604F05EFBA378F554AF
:1062A0000126A578184BD4F803005E55174B00283B
:1062B00003EB8503D3F8D830B8BF40429847272175
:1062C0000246284604F048FBD4F80330A078002B9F
:1062D000C8BF02224FF00003CCBF01920196009389
:1062E0001A46202104F004FB02B070BD0422084BC2
:1062F0001A70F9E7280A0020B20E0020240A0020B4
:10630000FC090020200A0020F5090020B405002027
:106310009C0A00207FB56421B84EB94A3378D6F87C
:106320000300292B5370117050603446154600F05D
:10633000D98700F2D680152B00F02D8457D8092B71
:1063400000F0FD811BD8042B00F0ED810AD8022B50
:1063500000F0C78100F2C881012B00F0BE8102234A
:106360002B70BCE1062B00F0E481C0F0DF81072B2D
:1063700000F0E281082BF2D1FEF7F6FCAFE10D2B25
:1063800000F0268315D80B2B00F00A8340F2DA8147
:10639000B378022B40F019837078372800F20F830E
:1063A00000F5A770974980000422014402F072FCB6
:1063B00095E10F2B00F05C83C0F03A83132B00F0C3
:1063C0009683142BCBD1904B904A1968136888425E
:1063D00080F2D38323F0030343F0040313601368B4
:1063E000002940F0D48343F00803136077E11F2BAA
:1063F00000F09B853FD8192B00F0648414D8172B2C
:10640000834B00F04E8440F24984D3F8C820002A20
:1064100000F06581013AC3F8C82003EB8202D2F88C
:10642000FC20C3F8C4205AE11B2B00F06784C0F0A5
:1064300057841C2B00F054851E2B90D17378142B9D
:1064400000F2BD82B278002A40F05085714A72494C
:10645000927E41F82300002A00F04181002B00F0D9
:106460003E8103F285108000A0F2146304221944D7
:1064700002F07DFB33E1242B00F0208611D8212B84
:1064800000F0BE85C0F08E85222B00F00F86232BF6
:106490007FF465AF5C4B1B68C6F80330FFF7F6FC72
:1064A0001DE1262B00F05886C0F03B86272B00F01C
:1064B0007B86282B7FF453AFFF2800F3108173787D
:1064C0000B2B00F20B87DFE813F07E06890694069B
:1064D0009F06AB06B906C406CF06DA06E306EB064E
:1064E000F706452B01F0FE825FD8332B01F0C881FF
:1064F00035D82D2B01F0398116D82B2B01F01880BF
:1065000040F27F8773780B2B01F22B81DFE813F0C9
:106510009E08A808B208BC08C708D408DE08EC0822
:10652000F608FF0807091209302B01F08E8109D8FF
:106530002E2B7FF414AF344B1B68C6F80330FEF7E4
:106540004BFCCCE0312B01F08C81322B7FF407AF78
:106550002D4B1B68C6F80330FFF78EFEBFE0402BC3
:1065600001F0B08213D8382B01F09281392B01F061
:10657000A881372B7FF4F3AE284B1B68FF2B00F26A
:10658000AE80D4F80310264A42F82310A7E0422B2D
:1065900001F0A082C1F09A82432B01F09F82442B2C
:1065A0007FF4DDAE03F0CEFC99E0852B01F0D382C1
:1065B00052D8802B01F0A28234D8472B01F09A8266
:1065C000C1F09482502B7FF4CAAE114BD3F8C8208F
:1065D000072A00F2848071780C2900F28080DFE8BD
:1065E00011F07C098E09A009B209C409D609E9098C
:1065F000050A170A290A3B0A4D0A5F0A280A0020E1
:106600009C0A002070050020880A0020300A002023
:10661000B405002008000020340A0020A40A00204D
:10662000A80A0020822B01F08882C1F06D82832BA2
:1066300001F08982842B7FF492AEA54B1B7D9B07D2
:1066400001F18582B0F5006F6AD20422A14B83F874
:10665000C020C3F8440142E08A2B01F023831CD8F8
:10666000872B01F0F182C1F07C82882B01F0B4828B
:10667000892B7FF474AE73788BBBB17879BB40F211
:10668000D24398422BD140F2FF7002F011FA02F08F
:1066900076F90120FDF7C7FE21E08D2B01F05A832A
:1066A0000CD88C2B7FF45BAE7678002E01F0138330
:1066B000012E01F020830323137010E0F22B01F070
:1066C0009883FF2B7FF44BAE40F2D243984206D121
:1066D0000122804B83F8782101E0FFF77FFD04B0B1
:1066E00070BDFFF7C9FDFAE7B678CEB9304604F0C1
:1066F000EFF80122A078784B27211A54324604F093
:106700002BF90223A07832460193009633462021CC
:1067100004F0EEF8A378714AD654714AD654DEE7F5
:1067200004232B70DBE7FEF757FBD8E7FEF73EFCB0
:10673000D5E7FFF793F8D2E7FEF716FBCFE7FFF7B1
:10674000A5FBCCE7B378022B00F0DA80032B00F036
:10675000DC80002B40F01D817378512B00F0888085
:1067600027D8472B6ED011D8422B61D006D8402BAA
:1067700045D0412B59D003232B7045E0452B5BD0EE
:106780005DD8442BF7D1524BDB6953E04C2B66D0DC
:1067900007D8492B5DD058D34B2BECD14C4BDB7831
:1067A00048E04F2B5ED060D84D2BE4D1484B5B7D49
:1067B00040E0812B6DD012D8552B60D005D8532BDB
:1067C000434A5AD057D9937E34E0592B5AD0802B64
:1067D0005BD0572BCFD13E4B93F827302AE0852B47
:1067E00066D005D8832B5FD05AD93E4B1B6821E079
:1067F000FE2B02D069D8F02BBDD13B4B16E040F206
:10680000FF7002F02EFA6860384B1B78002B3FF4C3
:1068100066AF374B6A681A60364B002A40F0BB807F
:106820001A6842F008021A6059E7294B1B7801E008
:10683000274B5B786B60E7E7254B5B79FAE7244BE6
:10684000DB68F7E7224B9B68F4E7214B93F826308F
:10685000F0E71F4BDB7D003318BF0123EAE71C4B39
:106860009B78E7E71A4B5B7EE4E7194B9B7DE1E7FA
:10687000174B1B7DDEE7136ADCE71369DAE7144B7D
:10688000DB7ED7E7124B9B8CD4E7124B93F8C030DA
:10689000D0E7104B93F8C0301E1F73427341C9E715
:1068A0000C4BD3F8C430C5E70A4BD3F8E830C1E746
:1068B00043F23901074A1048D2F8EC3000FB0313C9
:1068C000C2F8EC3023F00043B4E70C4B1B78C2E76E
:1068D00008000020B4050020F5090020B20E0020B9
:1068E000FC090020980A0020FC0E0020970A0020D6
:1068F000880A0020300A00206D4EC641960A00200A
:106900007278944B53F8223094E77378282B31D067
:1069100013D8022B26D006D813B3012B7FF42BAF4C
:106920008D4B5B6886E71C2B1ED0272B1FD01B2BA3
:106930007FF421AF884B1B7B7CE72B2B20D006D824
:10694000292B1AD02A2B7FF416AF834B1CE72D2B53
:106950001CD018D32E2B7FF40EAF7F4BDB6A69E778
:106960007D4B43E77C4B6EE77B4B5B7B62E77A4B6F
:106970001B695FE7784B5B695CE7774B9B6959E77D
:10698000754B1B6A56E7744B5B6A53E7724B9B6A05
:1069900050E70423F0E61A6822F008021A609EE627
:1069A000B378022B0ED17078372808D800F5A7707D
:1069B0006A4980000422014402F0D9F88FE60323DB
:1069C0002B708CE60423137089E60423137086E68B
:1069D000B07800287FF4A4AE7378012B0FD004D3D5
:1069E000022B0FD00323137079E603F0D9FA18B9FC
:1069F000B07803F065FF72E606232B706FE603F0B4
:106A000067FF6CE6002003F06BFF554B68601B7856
:106A1000002B3FF464AE534B1860534B1A6818B9FF
:106A200042F008021A605AE622F008021A6056E69E
:106A3000B37823B1022B05D0042313704FE6FDF782
:106A400013FD4CE67378072B08D818B91846FDF7E4
:106A50008FFC44E61846FDF793FC40E6FF2BAED1D1
:106A6000441C0ABF3F4BC0B21878FDF791FC36E6D4
:106A7000B378012B2ED023B1022B2FD00423137017
:106A80000FE07078082803D8FDF793FC686008E0F1
:106A90000A2815D1354B9B6883F40043C3F3C033F8
:106AA00053602F4B1B78002B3FF419AE2D4B6A68B7
:106AB0001A602D4BB2B91A6842F008021A600EE64D
:106AC0000B2802D1FDF726FFE0E7FF28E9D1FDF70B
:106AD00099FCDBE7707802F0DFFED7E77078FDF70E
:106AE00087FCD3E71A6822F008021A60F7E572788B
:106AF0001C4B092A26D8DFE802F005090C0F1319F0
:106B00001C1F22071A68104418601BE01A68101A2C
:106B1000FAE71A685043F7E71A6892FBF0F0F3E7D8
:106B2000196891FBF0F200FB1210EDE71A681040B3
:106B3000EAE71A681043E7E71A685040E4E71A6882
:106B4000D2431A601A68084B92B91A6842F00802D8
:106B50001A60C4E5A80A0020C80E002070050020B5
:106B6000970A0020880A0020300A00200010014007
:106B70001A6822F008021A60B1E50BBF23F0060381
:106B800023F0050343F0010343F0020326E423F05E
:106B900008031360A3E573780C2B3FF6A0ADDFE884
:106BA00003F0071019222B343E475059626B7400D2
:106BB000AD4B1B6819077FF592ADAC4BC3F8C40011
:106BC0008DE5A94B1B681A073FF589ADA74BC3F8A4
:106BD000C40084E5A44B1B68DB077FF580ADA34BA5
:106BE000C3F8C4007BE5A04B1B68DE073FF577AD1B
:106BF0009E4BC3F8C40072E59B4B1B685D077FF595
:106C00006EAD9A4BC3F8C40069E5974B1B6813F04F
:106C1000050F3FF464AD954BC3F8C4005FE5924B9C
:106C20001B689C077FF55BAD904BC3F8C40056E52D
:106C30008D4B1B6899073FF452AD8C4BC3F8C400D1
:106C40004DE5894B1B68DA067FF549AD874BC3F8E4
:106C5000C40044E5844B1B689B067FF540AD834B25
:106C6000C3F8C4003BE5804B1B685E067FF537AD7B
:106C70007E4BC3F8C40032E57B4B1B681D067FF5D5
:106C80002EAD7A4BC3F8C40029E5774B1B68DC05B1
:106C90007FF525AD754BC3F8C40020E5C3F8C400EB
:106CA0001DE5D3F8C820072A3FF619AD511CC3F8DB
:106CB000C810D3F8C41003EB8202C2F8FC10C3F86A
:106CC000C4000CE573782E2B03D80121684AD154F7
:106CD00005E5FF2B7FF473AE0122644B1A70FEE4CE
:106CE00073782E2B03D80021614AD154F7E4FF2B8F
:106CF0007FF465AE00225D4B1A70F0E45B4D95F8B1
:106D0000CC3093B90A23411C0BBF5A4A5843106830
:106D1000C5F81C0104BF4343C5F81C3102F014FD43
:106D20000123C5F8200185F8CC306378042B3FF6A9
:106D3000D6ACDFE803F0034471A71A0002F004FDAB
:106D4000D5F82031C01A0028D5F81C31B8BF404210
:106D500098428BBF0023D5F8C43085F8CC3003F1BE
:106D6000FF3398BFC5F8C430B9E4A07803F0B8FD8C
:106D700038B93D4A85F8CC00136823F0100313603E
:106D8000ADE4D5F81C31A3B102F0DEFCD5F820311A
:106D9000C01A0028D5F81C31B8BF4042984208D923
:106DA0000023314A85F8CC30136843F01003136098
:106DB00095E4D5F8C430013BC5F8C4308FE4A07821
:106DC000352103F0F3FD10F4007408D00023264AA7
:106DD00085F8CC30136823F0100313607FE4D5F8F6
:106DE0001C319BB102F0B0FCD5F82031C01A00284C
:106DF000D5F81C31B8BF4042984207D91A4A85F8E5
:106E0000CC40136843F01003136068E4D5F8C43035
:106E1000013BC5F8C43062E4A078352103F0C6FD1B
:106E200010F0010408D000230F4A85F8CC30136815
:106E300023F01003136052E4D5F81C31E3B102F0E3
:106E400083FCD5F82031C01A0028D5F81C31B8BF12
:106E50004042984210D9044A85F8CC40136843F068
:106E6000100313603BE400BF300A0020B40500208B
:106E70000C0F0020880A0020D5F8C430013BC5F86B
:106E8000C4302CE4A078352103F090FD10F002040A
:106E900008D00023A84A85F8CC30136823F01003EB
:106EA00013601CE4D5F81C319BB102F04DFCD5F801
:106EB0002031C01A0028D5F81C31B8BF4042984292
:106EC00007D99D4A85F8CC40136843F0100313603E
:106ED00005E4D5F8C430013BC5F8C430FFF7FFBB6B
:106EE0000022964B83F8C020FFF7F9BBFF2A7FF4FE
:106EF00017AC934D73B94FF4C364A4F214612046E8
:106F000004222944043401F032FEB4F5CD6FF4D1EB
:106F1000FFF7E5BB03F285108000A0F214610422A4
:106F2000294401F024FEFFF7DABB707814283FF6FD
:106F300046ADB378BBB9824B53F82010814B5160FA
:106F40001B78002B3FF4CBAB7F4B19607A4B1A6850
:106F500021B942F008021A60FFF7C1BB22F0080213
:106F60001A60FFF7BCBBFF2B7FF4DAAB744D70B92E
:106F70004FF4C364A4F2146120460422294404346B
:106F800001F088FEB4F5CD6FF4D1FFF7A8BB00F295
:106F900085108000A0F214610422294401F07AFED9
:106FA000FFF79DBB707814283FF609ADB3781A0639
:106FB00011D5664B9B7E002B3FF491AB00283FF42C
:106FC0008EAB00F28510624980000422014401F07A
:106FD000CEFDFFF784BB002B7FF4A2AB5B4B9B7E07
:106FE000002B3FF47CAB00283FF479AB00F2851016
:106FF000574980000422014401F0B9FDFFF76FBB3F
:107000007278514B0A2A0CD8DFE802F006151A1FD5
:10701000252D32373C4145004E491A6809680A441B
:107020001A601A68444B002A3AD11A6842F00802E2
:107030001A60FFF754BB47491A680968521AEFE70C
:10704000444A196812684A43EAE742491A680968DB
:1070500092FBF1F2E4E73F4A1868116890FBF1F205
:1070600001FB1202DCE73B491A6809680A40D7E7CE
:1070700038491A6809680A43D2E736491A68096824
:107080004A40CDE733490A68D2430A60C9E7196824
:10709000304A1160C5E72F4A196810681860F8E790
:1070A0001A6822F008021A60FFF719BB264B1B680A
:1070B000C6F80330FDF77AFFFFF711BB7378052B95
:1070C0003FF60DABDFE803F0030A11181F261A4A3A
:1070D000136803F00F031360FFF701BB164A136830
:1070E00023F010031360FFF7FABA134A136823F072
:1070F00020031360FFF7F3BA0F4A136823F040032D
:107100001360FFF7ECBA0C4A136823F08003136096
:10711000FFF7E5BA084A136823F480731360FFF79A
:10712000DEBA72782E2A3FF64AAC044B03EB820398
:107130005860FFF7D4BA00BF300A0020B405002021
:10714000340A0020970A0020880A00200800002046
:1071500020040020A40A0020B14BB24AD3F8241125
:107160001160D3F82811B04A1160D3F82C21D3F85C
:107170003011C3F8C420AD4A1160D3F8342193F81C
:10718000401183F8CC20D3F83821C3F82021D3F85C
:107190003C21C3F81C21A64A505C08B10120505480
:1071A00000225A70FFF79BBAB378002B7FF4B8AA7D
:1071B0007378142B3FF603AC9A4A11689D4A42F843
:1071C0002310FFF78CBA9C4BB17853F8200053F88A
:1071D0002120024443F82120FFF781BA964BB17871
:1071E00053F8200053F82120121A43F82120FFF70A
:1071F00076BA914BB17853F8202053F8214062437E
:1072000043F82120FFF76BBA8B4BB17853F820007D
:1072100053F8212092FBF0F243F82120FFF75FBAE8
:10722000854BB17853F8200053F8214094FBF0F2DD
:1072300000FB124243F82120FFF751BA7E4BB17890
:1072400053F8200053F82120024043F82120FFF793
:1072500046BA794BB17853F8200053F82120024305
:1072600043F82120FFF73BBA734BB17853F8200065
:1072700053F82120424043F82120FFF730BA6E4AEC
:10728000B17852F82030DB4342F82130FFF727BABB
:10729000694BB27853F8201043F82210FFF71FBA59
:1072A000654BB27853F8204053F8221043F822403F
:1072B00043F82010FFF713BA5F4BB27853F822203F
:1072C00053F820309A4240F33E82584A136823F024
:1072D000030343F004031360FFF701BA03232B7089
:1072E000FFF7FDB973780B2B00F28780DFE803F01E
:1072F00006111C2733414C57626B737EB1784E4A9E
:10730000484852F821300068034442F82130FFF722
:10731000E6B9B178484A434852F8213000681B1A50
:1073200042F82130FFF7DBB9B178434A3D4B52F8C0
:1073300021001B68434342F82130FFF7D0B9B178F0
:107340003D4A384852F82130006893FBF0F342F888
:107350002130FFF7C4B9B178374A324B52F8214097
:10736000186894FBF0F300FB134342F82130FFF759
:10737000B6B9B178304A2B4852F821300068034042
:1073800042F82130FFF7ABB9B1782B4A254852F8C3
:1073900021300068034342F82130FFF7A0B9B178EB
:1073A000254A204852F821300068434042F82130F5
:1073B000FFF795B91B4BB1781B681F4ADB4342F8B6
:1073C0002130FFF78CB9174BB27819681A4B43F884
:1073D0002210FFF784B9B178174A124B52F82100F6
:1073E0001C68186042F82140FFF779B9124BB27857
:1073F00053F822200B4B1B6864E703232B70FFF725
:107400006EB97278074B09490B2A00F28880DFE8D1
:1074100002F015252C333B454C535A60656E00BF76
:10742000B4050020880A0020A40A0020300A0020A9
:107430000C0F0020340A0020A80A0020B078A84AC7
:1074400052F82020186802441A601B68002B69D18A
:107450000B6843F008030B60FFF741B9B478A0480C
:107460001A6850F82400121AEEE79D4AB07852F8D4
:1074700020001A684243E7E7B47899481A6850F840
:10748000240092FBF0F2DFE7954AB0781C6852F8CE
:10749000200094FBF0F200FB1242D5E7B078904A4E
:1074A00052F8202018680240CEE7B0788C4A52F893
:1074B000202018680243C7E7B078894A52F8202094
:1074C00018684240C0E7B078854A52F82020D2437D
:1074D000BAE7B078824A52F82020B5E7B078804AFF
:1074E0001D6852F8204042F820501C60ADE77C4AED
:1074F000B07852F820001A6890420A6805DA22F043
:10750000030242F004020A609FE70BBF22F006026A
:1075100022F0050242F0010242F00202F3E70322E8
:107520002A7092E70B6823F008030B60FFF7D7B8C7
:1075300073780B2B00F28680DFE803F006111C271E
:1075400033414C57626B737EB178654A654852F897
:1075500021300068034442F82130FFF7C0B8B17809
:107560005F4A604852F8213000681B1A42F8213007
:10757000FFF7B5B8B1785A4A5A4B52F821001B6848
:10758000434342F82130FFF7AAB8B178544A55482E
:1075900052F82130006893FBF0F342F82130FFF7F6
:1075A0009EB8B1784E4A4F4B52F82140186894FB70
:1075B000F0F300FB134342F82130FFF790B8B178A5
:1075C000474A484852F821300068034042F82130C9
:1075D000FFF785B8B178424A424852F82130006836
:1075E000034342F82130FFF77AB8B1783C4A3D486E
:1075F00052F821300068434042F82130FFF76FB85D
:10760000384BB1781B68364ADB4342F82130FFF72C
:1076100066B8344BB2781968314B43F82210FFF743
:107620005EB8B1782E4A2F4B52F821001C681860C2
:1076300042F82140FFF753B8294BB27853F8222083
:10764000284BD8E603232B70FFF749B8254AB178B9
:10765000234B53F8213011680B441360FFF73FB8F8
:10766000204AB0781E49136851F820105B1A136045
:10767000FFF735B81B4A1A4BB17853F8211013683D
:107680004B431360FFF72BB8164AB07814491368C0
:1076900051F8201093FBF1F31360FFF720B8114A63
:1076A0000F4BB178106853F8211090FBF1F301FBF8
:1076B00013031360FFF713B80A4AB178084B53F865
:1076C000213011680B401360FFF709B8054AB17803
:1076D000034B53F8213011680B431360FEF7FFBFD3
:1076E000A80A0020A40A0020BB4AB178BB4B53F87B
:1076F000213011684B401360FEF7F1BFB278B74BF1
:1077000053F82230B44ADB431360FEF7E8BFB34BB3
:10771000B27853F82220B04B1A60FEF7E0BFB17880
:10772000AE4AAD4B52F821001C68186042F8214067
:10773000FEF7D5BFA94BB27853F82220A64B1B68A1
:107740009A42FFF6C2ADA64A13680BBF23F00603A8
:1077500023F0050343F0010343F002031360FEF737
:10776000BEBF03232B70FEF7BABF73780B2B68D80C
:10777000DFE803F0060F18212B374049525B6761A1
:10778000B178964A52F82130184442F82100FEF7A9
:10779000A6BFB178914A52F82130181A42F8210058
:1077A000FEF79DBFB1788D4A52F82130584342F818
:1077B0002100FEF794BFB178884A52F8213093FB3C
:1077C000F0F042F82100FEF78ABFB178834A52F800
:1077D000214094FBF0F300FB134042F82100FEF738
:1077E0007EBFB1787D4A52F82130184042F821001E
:1077F000FEF775BFB178794A52F82130184342F844
:107800002100FEF76CBFB178744A52F8213058401D
:1078100042F82100FEF763BFB178704A52F8213078
:10782000DB4342F82130FEF75ABFB2786B4B43F886
:107830002200FEF754BFB278684B53F822309842CA
:107840007FE703232B70FEF74ABFFDF79BFA012267
:10785000644B83F8C020D6F80320C3F8C420FEF799
:107860003EBF71785D4A52F82130013B002B42F84F
:1078700021307EF734AF5B4BC3F8C400FEF72FBF57
:10788000594B1B68C6F80330FEF7A8FCFEF774BE20
:10789000514B1B68FF2B3EF622AF504A52F8232073
:1078A000514B6A601A604E4B2AB91A6842F00802BE
:1078B0001A60FEF714BF1A6822F008021A60FEF779
:1078C0000EBF454B1B68FF2B3EF609AF464A1168B9
:1078D000424A42F82310FEF702BF414909680E07E9
:1078E0007EF5FDAE511CC3F8C810D3F8C41003EBED
:1078F0008202C2F8FC10C3F8C400FEF7F0BE38499B
:1079000009680D073EF5EBAE511CC3F8C810D3F85B
:10791000C41003EB8202C2F8FC10C3F8C400FEF7E7
:10792000DEBE2F490968CC077EF5D9AE511CC3F8DD
:10793000C810D3F8C41003EB8202C2F8FC10C3F8DD
:10794000C400FEF7CCBE26490968C9073EF5C7AE9C
:10795000511CC3F8C810D3F8C41003EB8202C2F85C
:10796000FC10C3F8C400FEF7BABE1D4909684E07F3
:107970007EF5B5AE511CC3F8C810D3F8C41003EBA4
:107980008202C2F8FC10C3F8C400FEF7A8BE144976
:10799000096811F0050F3EF4A2AE511CC3F8C810DF
:1079A000D3F8C41003EB8202C2F8FC10C3F8C40081
:1079B000FEF795BE0A4909688D077EF590AE511C09
:1079C000C3F8C810D3F8C41003EB8202C2F8FC104D
:1079D000C3F8C400FEF783BEA40A0020A80A002052
:1079E000300A0020B4050020880A0020C94909682F
:1079F0008C073EF474AE511CC3F8C810D3F8C41001
:107A000003EB8202C2F8FC10C3F8C400FEF767BEA5
:107A1000C0490968C9067EF562AE511CC3F8C8109A
:107A2000D3F8C41003EB8202C2F8FC10C3F8C40000
:107A3000FEF755BEB74909688E067EF550AE511C5B
:107A4000C3F8C810D3F8C41003EB8202C2F8FC10CC
:107A5000C3F8C400FEF743BEAE4909684D067EF583
:107A60003EAE511CC3F8C810D3F8C41003EB820219
:107A7000C2F8FC10C3F8C400FEF731BEA54909687E
:107A80000C067EF52CAE511CC3F8C810D3F8C410F8
:107A900003EB8202C2F8FC10C3F8C400FEF71FBE5D
:107AA0009C490968C9057EF51AAE511CC3F8C81077
:107AB000D3F8C41003EB8202C2F8FC10C3F8C40070
:107AC000FEF70DBE02F029FAFEF709BE02F026FA13
:107AD000FEF705BE02F023FAFEF701BE02F020FA1F
:107AE000FEF7FDBD02F02FFAFEF7F9BD02F02CFA09
:107AF000FEF7F5BD02F029FAFEF7F1BD0022864B34
:107B000083F8C020FEF7EBBD73782BB1012B09D0B1
:107B100003231370FEF7E3BD01227F4B83F8C020DF
:107B2000FEF7DDBDB0F5006FBEF4FAAD7A4A82F81B
:107B3000C030C2F8C400FEF7D2BD0222764B83F8F3
:107B4000C020FEF7CCBDFDF71DF9FEF7C8BD082328
:107B50001370FEF7C4BD00226F4B83F8C020FEF700
:107B6000BEBD01256D4B6E4A1D706E4C9378B0F50D
:107B7000006F237026D2127D12EA050622D102A9D7
:107B800000F0BCFE9DF80830267263709DF8093045
:107B9000A3709DF80A30E3709DF80E3023719DF8B4
:107BA0000D3063719DF80C30A3719DF80B30E371BB
:107BB0002B46E15C227A01330A44082B2272F8D169
:107BC000FEF78DBD2B460022E2540133082BFBD17A
:107BD00023782372FEF783BD7378012B19D005D368
:107BE000022B1FD003231370FEF779BD01224B4BEC
:107BF0001A704B4B4B4A9B7813704B4B1968002300
:107C00000139013311F8010F082BD054F9D1FEF7D7
:107C100066BD04226B71EA712D23D8222B71AA71E3
:107C2000FEF75DBD01223D4B40481A703C4B3D4A7A
:107C30009B78137000230133191811F8091C082BC5
:107C4000D154F8D1FEF74BBD7378032B3EF647AD08
:107C5000DFE803F002101E232F4B93F8C020EA71D7
:107C600093F8CC20D3F84431AA711A0A6A712B71A7
:107C7000FEF735BD284B93F8C020EA7193F8CC206D
:107C8000D3F8C430AA711A0A6A712B71FEF727BDA6
:107C9000274B1B686B60FEF722BD264B1B686B6091
:107CA000FEF71DBD7278244B9AB91A70E378234A07
:107CB0001370194A92F84811214A11700022214983
:107CC0000A7021490A70214A11780B431370FEF79C
:107CD00006BD0122E9E7042202A940F2FB7000F090
:107CE000D9FF029BD4F803209A420ABF01236E6099
:107CF0006B60FEF7F4BCA3782A2B07D10422144949
:107D000040F2FB7000F033FFFEF7E9BC0323137071
:107D1000FEF7E5BC300A0020B40500208C0A0020E4
:107D2000080000208D0A002000000020004000080C
:107D3000880A0020A40A0020B00E0020B80E0020FF
:107D4000060F0020B30E00203B0F0020B10E0020D4
:107D50002B0A00207378032B47D8DFE803F01B02BF
:107D600034420022484CD4F84C1104F5A8738A42DE
:107D70003EF4B5AC53F82250854202F1010520D102
:107D800003EB8503043B01398A4214D3C4F84C1138
:107D9000FEF7A5BC3C4BD3F84C21092A8FBF092321
:107DA000511CC3F84C1103EB820394BFC3F850017C
:107DB0002B70FEF794BC53F8040F013243F8040C07
:107DC000E2E72A46D3E7002319462F4AC2F84C318E
:107DD00002F5A87242F8231001330A2BFAD1FEF7FC
:107DE0007EBC0A236B60FEF77ABC03232B70FEF780
:107DF00076BC7378812B7EF472ACB378922B7EF4D0
:107E00006EACB379A32B7EF46AAC7379B42B7EF499
:107E100066AC3379C52B7EF462ACF378D62B7EF456
:107E20005EAC1A4B5A6842F040525A604FF400421E
:107E30005A6102F015F801F087FC044601F084FC59
:107E4000001B0028B8BF4042B0F57A7FF6DBFCF794
:107E5000F1FA04F0DDFB002005F0AAF800210C483F
:107E600003F0A9FF0A4803F00BFF0A4803F096FA53
:107E700003F0D2FF4FF0804005F0F3F80020FCF74C
:107E8000D2FAFEF72CBC00BFB40500200010014060
:107E9000080002400024014000232DE9F04119466A
:107EA0004FF0FF35404A414C1360414AC4F8C4309A
:107EB0001360404AC4F8C83013603F4A84F8CC309D
:107EC00023706370201D40F82350D15401332F2BB1
:107ED000F9D13A4B5B7E002B3AD1394BC4F8D830FC
:107EE000C4F8E030C4F8DC30272100200025C4F8B5
:107EF000E43002F05BFD334B2621C4F8D000284665
:107F00001D7002F053FD304B1860304B28461D7039
:107F1000FCF75AFD2846FCF7EFFD2D4B2A461F467D
:107F200043F825200135B5F5807FF9D1294DAB7E89
:107F3000CBB9EB7E3BB3002384F879316B7D83B3FF
:107F4000FCF7D0FC68B3012384F8C030BDE8F081B1
:107F5000214BC4F8D830214BC4F8E030204BC4F892
:107F6000DC30204BC0E74FF4C366DFF87C80A6F21C
:107F70001461304604224144043600F08BFEB6F50D
:107F8000CD6FF4D1D5E74FF4A766A6F5A7613046CB
:107F900004223944043600F07DFEB6F5C36FF4D1F7
:107FA000C9E70023D0E700BF880A0020B4050020FD
:107FB000A40A0020300A00200C0F0020000A002034
:107FC000E9B20008F5090020200A0020240A002058
:107FD000A80A0020080000201DB2000881B2000895
:107FE00059B20008C1B20008340A0020F7B50F4C9E
:107FF00007460E4694E803008DE803000C498A709A
:108000000022C1F803300B4B0F704E701A70FEF750
:1080100081F921786368084A82F87A119DE80300A3
:1080200084E80300184603B0F0BD00BF9C0A00209E
:10803000280A0020970A0020B4050020014B93F87D
:108040007A017047B4050020F7B504461F4A6378EB
:108050001F4D1370A3780E4695E803005370E37824
:108060008DE80300937023796F46937163795371A0
:10807000A3791371E379D3700022164B1A70FEF7BF
:1080800049F9154B1A782B469AB9327072702A78D2
:10809000B2706A78F270EA793271AA7972716A798B
:1080A000B2712A79F27197E8030083E8030003B004
:1080B000F0BD012AF7D10948721EF11D10F8014FD9
:1080C00002F8014F8A42F9D1EDE700BF280A0020EB
:1080D0009C0A0020970A00208C0A00208D0A0020AC
:1080E0002DE9F047A44B8EB01B78A44C13B994F83B
:1080F0007B316BB1A24B1B78063BDBB2192B04D84A
:10810000A04A22FA03F3D90702D4002384F84831A5
:1081100094F848319C4E5A1E012A56D8012B14BFA0
:10812000082307238DF8183094F87C3197498DF88F
:1081300019300023CA688DF81A3007923278002A65
:1081400038D18B688DF827208DF82030904B197826
:108150008DF8211059788DF82210D9798DF82310D7
:1081600099798DF8241059791B798DF825108DF89F
:108170002630884B1B782BB906A801F023FA00287B
:1081800000F07A83844BDFF80C821A789946002A33
:1081900000F03181814B824F1B78013B062B00F2AE
:1081A0002681DFE813F0010101018B012401240184
:1081B0002401B201012ADCD17A48013306AA195CF4
:1081C0001A44082BD171F8D1D3E7032B40D194F88E
:1081D0007951002DD6D1337883BBDFF8B0816C4F55
:1081E00098F8020098F801503B7805441D447B78CC
:1081F0001D44FB791D44BB791D447B791D443B79AB
:108200001D4400F0F3FE98F8010000F0EFFE38780E
:1082100000F0ECFE787800F0E9FEF87900F0E6FE78
:10822000B87900F0E3FE787900F0E0FE3879EDB23D
:1082300000F0DCFE284600F0D9FEA3E7012BA1D117
:10824000584F785D013500F0D1FE092DF9D199E73D
:10825000042B2BD1002301224C4FDFF83481B87856
:108260007D7888F801300544154488F80020C8F866
:10827000043000F0BBFE787800F0B8FE98F80000FB
:1082800000F0B4FE98F8010000F0B0FE98F8070086
:1082900000F0ACFE98F8060000F0A8FE98F8050083
:1082A00000F0A4FEEDB298F80400C1E7072B41D11D
:1082B00094F87931002B7FF465AF327882BB334B71
:1082C0009F7893F80180324B8DF800701D785878B4
:1082D0004744D9798DF802503D449A798DF80300CE
:1082E000284493F805C08DF80410014493F804E085
:1082F0008DF805200A440CEB020373448DF80180CD
:108300008DF806C08DF807E08DF80830214B1B78FA
:10831000002B3FF437AF0921684601F0D3FD31E768
:10832000012AF3D11F495A5C0DF803200133092BB0
:10833000F9D1EBE7082B7FF425AF00230120144A85
:1083400012495370107053608A7849788DF8002074
:108350000A4402448DF801108DF802008DF80330B4
:108360008DF804308DF805308DF806308DF8073023
:108370008DF80820CAE700BF960A0020B405002047
:10838000280A0020110200028C0A002008000020A8
:108390009C0A0020A80E00203B0F0020060F0020A2
:1083A000B30E00208D0A0020C54A397893688DF8F5
:1083B00036108DF8303080238DF831308A238DF8D7
:1083C0003230002307218DF833308DF834308DF8AA
:1083D00035308DF829308DF82A30D3688DF8281083
:1083E0000B9398F8003013B90AA801F0EBF80023BA
:1083F0003B7089F80030002384F84831337084F8EA
:108400007B3194F8783113B10120FCF70CF894F823
:108410007D314BB194F87931B3FA83F35B0984F879
:108420007931002384F87D3198F80030002B40F03A
:108430005F8106A801F012F9002800F059819DF82B
:108440001830062B40F254819E4B9DF820201A7064
:108450009DF821205A709DF822209A709DF82320C3
:108460009A719DF824205A719DF825201A719DF863
:108470002620DA709DF81930079A84F87C31904BE9
:108480001B699A4204BF012384F87B3101F05CF937
:1084900000228D4B18608D4B1A709DF81830072BF9
:1084A0000CBF0123022384F8483194F8C0305A1ECF
:1084B000012A50D9052B4ED001224DE0DFF800A251
:1084C0003B789AF802009AF8015005440A351D4499
:1084D00000F08CFD9AF8010000F088FD802000F08B
:1084E00085FD8A2000F082FD002000F07FFD002045
:1084F00000F07CFD002000F079FDEDB2387800F04E
:1085000075FD284600F072FD71E780218DF80E1090
:108510008A218DF80F100021694A8DF81010937888
:1085200050788DF80C303A7803440A3313448DF8B0
:10853000143098F800308DF80D008DF811108DF87A
:1085400012108DF81320002B3FF451AF092103A81E
:1085500001F0B8FC4BE700225D4B1A7094F8C03074
:10856000042B04D1574B19780A0640F1888194F8FE
:108570004821082A04D840F25113D340DF0701D420
:10858000FDF7C8FE94F84831092B74D101F0DCF8EE
:10859000D4F8F0304F4DC01A00282A68B8BF4042C6
:1085A000904209D94C4B1A78012A04BF02221A7052
:1085B00001F0CAF8C4F8F00001F0C6F8D4F8F430BD
:1085C0006A68C01A0028B8BF4042904209D9424B9D
:1085D0005A78012A04BF02225A7001F0B5F8C4F893
:1085E000F40001F0B1F8D4F8F830AA68C01A0028F5
:1085F000B8BF4042904209D9374B9A78012A04BF4C
:1086000002229A7001F0A0F8C4F8F800237893B31E
:10861000637883BB1D46304A3048D15C022940F064
:10862000228150F823104E1C00F01C8184F8403148
:1086300000232B4A1268C4F824212A4A1268C4F87D
:108640002821D4F8C420C4F8C410C4F82C21264A28
:108650001268C4F8302194F8CC2084F8CC3001237F
:10866000C4F83421D4F820216370C4F83821D4F838
:108670001C21C4F83C2194F84831092B06D194F808
:10868000C020022A04BF052284F8C020D4F84C215F
:10869000002A00F0F180092B40F0EE8094F8C03001
:1086A000012B40F0E9800023D4F8C4100F4850F8A3
:1086B00023508D4240F0DC80052384F8C030DBE09D
:1086C00008000020280A0020F80E0020A90E002033
:1086D000970A0020C80E00200C0F0020B8050020CB
:1086E000880A0020A40A0020300A00200407002085
:1086F00094F87951002D62D103A800F091FC002874
:108700005DD000F0A9FC08B184F87E5194F87E2178
:108710009DF80C10531CDBB22244092B84F87E31E7
:1087200082F87F117FF41AAF002384F87E31694B01
:1087300094F87F215978914207D093F827100029A7
:108740003FF40CAF8A427FF409AF93F827306249B7
:10875000934204BF012384F87B3100235A5C013328
:108760001544082BEDB2F9D194F88731AB4222D1F0
:108770005A4B94F880211A7094F881215A7094F819
:1087800082219A7094F883219A7194F884215A7105
:1087900094F885211A7194F88621DA7000F0D4FFDC
:1087A0004F4B504A186000231370032284F87E3127
:1087B00084F8482179E6042384F84831CEE694F819
:1087C00079518DBB98F8003073B30AAE304601F092
:1087D00063FB48B32B46F25C01331544082BEDB222
:1087E000F9D19DF83020AA42E6D13C4B9DF82920D2
:1087F0001A709DF82A205A709DF82B209A709DF8C7
:108800002C209A719DF82D205A719DF82E201A71F6
:108810009DF82F20DA7000F097FF0022304B18608F
:10882000304B1A7007233EE694F8C030013B012B11
:108830003FF694AED4F8C430B3F5006F0ED2FCF717
:1088400051F858B1D4F8C4002449431CC4F8C430CA
:1088500000F054F8092384F848312DE6002384F809
:10886000C0307BE6D55401332F2B7FF4D6AE02E720
:1088700001339A427FF41BAF0EB0BDE8F08794F845
:108880004801082804D840F25112C240D207F3D45C
:10889000D4F84401144DD3F80330B0F5006F69707B
:1088A0006B6012D20D4900F039F90C49D4F844013B
:1088B00000F0A6F838B1D4F844310133C4F844319B
:1088C00065232B70D8E70723FBE707232B700023D2
:1088D000F3E600BF0800002033070020280A00202C
:1088E000000F0020050F00209C0A0020800000F1EE
:1088F000006000F5FE300068704700000022C0EB09
:10890000C00038B50C4600F5006503211046FCF7A1
:10891000A1F90022C5F307211046FCF79BF90022BC
:10892000E9B21046FCF796F9002211461046FCF712
:1089300091F90022207011461046FCF78BF90022B5
:10894000607011461046FCF785F90022A0701146B0
:108950001046FCF77FF90022E07011461046FCF744
:1089600079F90022207111461046FCF773F90021B5
:10897000607101220846FCF76DF9A07138BD38B569
:108980004FF40064012206210020FCF763F9002265
:1089900005211046FCF75EF9002101220846FCF78C
:1089A00059F98007F3D5002202211046FCF752F94D
:1089B0000022C4F307211046FCF74CF90022E1B273
:1089C0001046FCF747F90025A5F13F014A424A410C
:1089D000002101350846FCF73DF9402DF4D1002275
:1089E00005211046FCF736F9002101220846FCF764
:1089F00031F9C307F3D44034B4F5804FC2D138BD48
:108A0000F7B50022C0EBC00000F500650C4610462B
:108A10000321FCF71FF90022C5F307211046FCF7DC
:108A200019F90022E9B21046FCF714F900221146A8
:108A30001046FCF70FF90022074611461046FCF7D6
:108A400009F90022064611461046FCF703F90022F8
:108A5000054611461046FCF7FDF800228DF803008C
:108A600011461046FCF7F6F800228DF80400114676
:108A70001046FCF7EFF800218DF8050001220846AA
:108A8000FCF7E8F823788DF80600BB420ED1637836
:108A9000B3420BD1A378AB4208D1DDF80300D4F880
:108AA0000330C31A5842584103B0F0BD0020FBE721
:108AB00038B5012204460D4600200621FCF7CAF80D
:108AC000002205211046FCF7C5F8002101220846C6
:108AD000FCF7C0F88207F3D5002202211046FCF70C
:108AE000B9F80022C4F307211046FCF7B3F80022BE
:108AF000E1B21046FCF7AEF8012229460020FCF74F
:108B0000A9F8002205211046FCF7A4F80021012253
:108B10000846FCF79FF8C307F3D438BD38B50D46B7
:108B2000C0EBC00404F500600978FFF7C1FF697865
:108B300004F60100FFF7BCFFA97804F60200FFF776
:108B4000B7FFE97804F60300FFF7B2FF297904F6CE
:108B50000400FFF7ADFF697904F60500FFF7A8FFF1
:108B6000A97904F60600BDE83840FFF7A1BF2DE95A
:108B7000F843044688461646062101220020FCF7E9
:108B800069F8002205211046FCF764F80021012253
:108B90000846FCF75FF88507F3D50022022110464E
:108BA000FCF758F80022C4F307211046FCF752F8EE
:108BB0000022E1B21046FCF74DF80025771EB542C1
:108BC0000DD1002205211046FCF744F800210122B6
:108BD0000846FCF73FF8C307F3D4BDE8F883013437
:108BE00014F03F0918F8051039D0781B4242424171
:108BF0000020FCF72FF8B9F1000F2ED1BD422CD286
:108C0000002205211046FCF725F800210122084624
:108C1000FCF720F810F00100F2D101220621FCF748
:108C200019F8002205211046FCF714F80021012252
:108C30000846FCF70FF88207F3D500220221104600
:108C4000FCF708F80022C4F307211046FCF702F8ED
:108C50000022E1B21046FBF7FDFF0135AFE701222C
:108C6000C6E7002210B5032104461046FBF7F2FFC9
:108C70000022C4F307211046FBF7ECFF0022E1B20B
:108C80001046FBF7E7FFBDE810400021012208462F
:108C9000FBF7E0BFF8B51546002204460E46104625
:108CA0000321FBF7D7FF0022C4F307211046FBF78F
:108CB000D1FF0022E1B21046FBF7CCFF3446771912
:108CC000013DBC4200D1F8BD0021A21BAB1A5A42A3
:108CD0005A410846FBF7BEFF04F8010BF1E737B530
:108CE000002205211046FBF7B5FF002101220846AE
:108CF000FBF7B0FF10F07104F2D100F025FD05463E
:108D000000F022FD401B0028B8BF4042B0F5FA6FCA
:108D100018DA74B1264B1B78B3B9402225490020DC
:108D2000FFF7B8FF202224494020FFF7B3FF03B02C
:108D300030BD40F2FF70FFF794FFA0F142035C42A8
:108D40005C41DDE7002CE5D1002140F2FF70FFF728
:108D5000AFFEFFF714FE402216490020FFF707FF81
:108D6000202216494020FFF702FF00234FF4C3647E
:108D700002AD45F8043D2046042229460434FFF79D
:108D8000F6FEB4F5FF6FF6D100234FF4A76401930C
:108D90002046042229460434FFF7E9FEB4F5C36FE8
:108DA000F6D1422140F2FF70FFF782FEB5E700BF27
:108DB000B90E002008000020000A0020C80A01089F
:108DC00030B5054687B0524804F02AFE01214FF421
:108DD000804003F0C5FE0021042003F0D9FB0323EB
:108DE0008DF8063018230DEB03048DF807304FF48F
:108DF000007324F8143D2146464803F036FB48230F
:108E00008DF807304FF4806342482146ADF80430B6
:108E100003F02BFB02A804F095FE0B2D74D8DFE8BD
:108E200005F07306585B5E6164676A6D6F714FF49D
:108E300061530293029B02A95B083548029304F038
:108E40003DFE2523002401258DF8003007236846C8
:108E50008DF801308DF802408DF8035003F014FCBA
:108E600040F2FF312A4804F055FF224628212848C5
:108E700004F095FE2A4640F22771254804F08FFE43
:108E80002A4640F22661224804F089FE2A4640F232
:108E900025511F4804F083FE224640F224411C481D
:108EA00004F07DFE224640F64601194804F077FEA4
:108EB000224640F66A11164804F071FE22466021EF
:108EC000134804F06CFE2946114804F05CFE07B01C
:108ED00030BD4FF49643ACE74FF4E143A9E74FF4BC
:108EE0001643A6E74FF46143A3E74FF49633A0E798
:108EF0004FF4E1339DE74FF461339AE7064B98E76F
:108F0000064B96E7064B94E74FF4165391E700BFE4
:108F1000003801400008014090D0030020A1070064
:108F200040420F00684620F007018D4619B52A48D7
:108F300003889C0604D5294BDB68190430D5838847
:108F4000254803881A0616D5254B1A689AB9254B69
:108F5000DC6A196B8C4239D04FF400441F490C6114
:108F6000196B4C1C1C63194491F834108180196BE7
:108F7000202900D11A63184803885B060CD540F2FB
:108F8000266104F0EBFE174B1A6BDB6A9A4202BFB4
:108F90004FF40042114B5A61BDE8194085467047B5
:108FA000104B1A6859680132202A08BF00228A42F1
:108FB00005D0196880881944C0B208721A600A2165
:108FC000094A11609A6A064B1A60B9E740F22771A4
:108FD00004F0E5FDCFE700BF003801400008014084
:108FE0003C0F00203C070020400F00200A4AD36AB3
:108FF000116B0133202B08BF00238B420AD0D16AAA
:10900000114481F83400D36240F2277101220348F1
:1090100004F0C5BD704700BF3C0700200038014088
:10902000094B59681A6891420CD05A68511C596012
:109030001A44127A02705A68202A01D100225A601A
:1090400001207047002070473C070020014B9862C8
:10905000704700BF3C070020044B1A7802F0FF0065
:1090600012B1002201201A70704700BF440F002087
:1090700008B5FBF7DFF90022034B5A601A60BDE820
:109080000840FBF7D5B900BF3C07002010B5441ECF
:1090900014F8010F00B910BDFFF7A8FFF8E700BFF3
:1090A000684620F007018D4631B5254C254B2568D3
:1090B0001B680135082D08BF00259D4286B03AD0B7
:1090C00001A9002002F0C0FC9DF80C302268042B9E
:1090D0001D4B03EB021227D1012151702268029926
:1090E00003EB021251609DF80D20022A0CBF0121F2
:1090F0000021226803EB0212917022689DF80E1085
:10910000120199540022216801A8104403EB0111B7
:109110001144C07A0132082A0872F4D1256006B0E1
:10912000BDE83140854670470021517022680199A1
:1091300003EB0212D6E7002002F06CFCEFE700BF61
:10914000D40F0020480F0020540F0020684620F064
:1091500007018D4631B5254C254B25681B68013527
:10916000082D08BF00259D4286B03AD001A90120F4
:1091700002F06AFC9DF80C302268042B1D4B03EBB7
:10918000021227D1012151702268029903EB0212C9
:1091900051609DF80D20022A0CBF01210021226898
:1091A00003EB0212917022689DF80E10120199547F
:1091B0000022216801A8104403EB01111144C07A78
:1091C0000132082A0872F4D1256006B0BDE83140AA
:1091D00085467047002151702268019903EB021205
:1091E000D6E7012002F016FCEFE700BFD40F002005
:1091F000480F0020540F0020684620F007018D46DC
:109200002B4B11B52B4A1968126887B0914208D1CF
:109210000021012002F04AFB07B0BDE8114085465D
:1092200070471968244A02EB0111497801F0FF00E8
:10923000002930D004218DF80C100021019119680B
:1092400002EB011149680291196802EB011189785A
:1092500001F0FF0041B302218DF80D1019680901DA
:10926000515C8DF80E100021186802EB00100844C4
:10927000047A01A8084401310829C472F4D11A689B
:1092800001A801321A601A68082A04BF00221A6075
:1092900002F018FBC0E719688DF80C0002EB011111
:1092A000496802900191CFE78DF80D00D6E700BF25
:1092B000500F00204C0F0020D80F0020F0B50138CF
:1092C0008BB00E4615460C23072800F20E81DFE80E
:1092D00010F00A0108010601040102010C0100015D
:1092E000080002228DF8143003238DF81530002376
:1092F000ADF816208DF8133002F0ECF901214FF093
:10930000007003F039FC0121084603F029FC01211B
:10931000082003F025FC0021082003F039FC01217E
:109320004FF4EA1003F034F903238DF806301823C4
:109330008DF807304FF400730AAC24F8243D214621
:10934000814803F092F804238DF807304FF48073BE
:109350000127214600247C48ADF8043003F085F84D
:1093600003A88DF812408DF80C408DF80D708DF823
:109370000E408DF80F408DF810708DF8117002F0CE
:10938000B6F9B6F5006F8DF818408DF819408DF8D4
:109390001A7080F2AC807301ADF81C304FF6FF7389
:1093A000ADF81E40ADF82030ADF82230ADF82440C5
:1093B0008DF8267006A802F0F7F9012300228DF837
:1093C00018308DF819208DF81A30002D00F09E808D
:1093D000B5F5006F80F29A80ADF81E204FF6FF724F
:1093E0006901ADF81C10ADF82020ADF82220ADF8D1
:1093F00024308DF8263006A802F0D6F902238DF825
:1094000018307313F60046F0040600270124ADF867
:109410001E604FF6FF7606A8ADF81C308DF8197067
:109420008DF81A40ADF82060ADF82260ADF82470D8
:109430008DF8264002F0B8F90323BD428DF81830AC
:109440008DF819708DF81A406FDD6B13ED0045F043
:109450000405ADF81C30ADF81E50ADF82060ADF835
:109460002260ADF824408DF8264006A802F09CF951
:10947000012407260025142302A88DF808308DF852
:1094800009608DF80A508DF80B4003F0FDF81523A4
:1094900002A88DF808308DF809608DF80A508DF813
:1094A0000B4003F0F1F8132302A88DF808308DF873
:1094B00009608DF80A508DF80B4003F0E5F821465D
:1094C000022002F0F3F92146102002F0EFF90BB070
:1094D000F0BD042206E7102204E7142202E7282246
:1094E00000E76422FEE6C822FCE60822FAE64FF610
:1094F000FF73ADF81C40ADF81E40ADF82030ADF85C
:109500002230ADF824408DF8264053E74FF6FF7126
:10951000ADF81C20ADF81E20ADF82010ADF82210DB
:10952000ADF824308DF8262065E70423ADF81C70D3
:10953000ADF81E30ADF82060ADF82260ADF82440E3
:109540008DF8267091E700BF000C014037B500216F
:10955000022002F0ABF90021102002F0A7F900214F
:10956000012002F0A3F900240725142301A88DF897
:1095700004308DF805508DF806408DF8074003F053
:1095800083F8152301A88DF804308DF805508DF867
:1095900006408DF8074003F077F8132301A88DF8F3
:1095A00004308DF805508DF806408DF8074003F023
:1095B0006BF802F08FF821464FF0007003F0DCFAF0
:1095C00003B030BDF0B5437887B004464268002B45
:1095D00037D004238DF80C30002302920193A37836
:1095E00003B102238DF80D30234613F8081B06AA99
:1095F00002F80A1D04F1100113F8010B8B4202F866
:10960000010FF9D101A802F05DF9042816D1104F1D
:10961000104B3D681B680135082D08BF00259D4291
:1096200014D03B680C4E06EB031694E80F0086E856
:109630000F00012108463D6002F038F9012007B013
:10964000F0BD8DF80C3001920293C8E70020F6E7D8
:109650004C0F0020500F0020D80F002030B50C4BCD
:109660000C4C054622681B689A420FD02268531C96
:109670002360094B03EB02130FCB85E80F0023682F
:10968000082B01D100232360012030BD002030BD14
:10969000D40F0020480F0020540F0020684620F00F
:1096A00007018D4601B5BDE801408546704700BF02
:1096B000684620F007018D4601B5124B19781A460D
:1096C000E9B15B681049013353600B6801330B60EB
:1096D0000E4B196811B11968013919600023137014
:1096E0000B4B1A683AB11A68013A1A601B6813B931
:1096F0000122084B1A70BDE80140854670470122DF
:109700001A70EDE790070020980A00203C0F002017
:10971000400F0020440F002008B5042003F022FC75
:1097200048F6A04003F02AFC012003F02DFC054878
:109730000022032103F07CF8BDE80840012003F07B
:1097400037BC00BF9AC30200014B5868704700BF86
:1097500090070020000000002DE9F04100240325BF
:109760004FF0090892B001A945488DF80740ADF8BF
:1097700004808DF8065002F078FE01A941488DF86A
:109780000740ADF804508DF8065002F06EFE01213E
:10979000084603F0D9F901214FF4007003F0E0F915
:1097A000394802F06DFA394B04270793384B07A963
:1097B000089380230C934FF480730D934FF48063D0
:1097C0000E9320230F934FF400532F4810930994C6
:1097D0000B9411940A9702F0C3FA01212A4802F06F
:1097E000EAFA01264FF4602302A92A48029404935E
:1097F00005948DF80C608DF80D608DF8187001F0EF
:10980000FBFD2B4632462946224801F06DFE2B46D1
:10981000022241461F4801F067FE2B462A460821D6
:109820001C4801F061FE2B4621463A46194801F0DA
:109830005BFE22464FF4FC61164801F01CFE3146E7
:10984000144801F00FFE3146124801F002FE1148A3
:1098500001F01AFE0F4C204601F01BFE0028FAD141
:109860000C4801F01AFE0B4C204601F01BFE0028AC
:10987000FAD10121074801F019FE12B0BDE8F081CC
:1098800000080140000C0140080002404C24014047
:109890009807002000240140F8B50A2863D8DFE8C3
:1098A00000F006626262626262620A125F003C4B12
:1098B000188880B2F8BD3A4B588883B240F26B10DA
:1098C00058430013F8BD364BD88880B206F084F8B0
:1098D00005F050FC0022334B05F0A0FC24A3D3E993
:1098E000002305F09BFC04460D4602460B4620A1D2
:1098F000D1E9000105F0DEFA1FA3D3E900230646F3
:109900000F462046294605F0B3FD02460B46304679
:10991000394605F0ADFD05F059FF05F02BFC00229E
:10992000214B05F0A5FD06F03BFE15A3D3E900236E
:1099300005F074FC14A3D3E9002305F0BDFA024638
:109940000B4613A1D1E9000105F092FD12A3D3E962
:10995000002305F0AFFA05F039FF06F0E5F9F8BD90
:109960000F4B9888A9E70020F8BD00BFAFF3008037
:109970006666666666660A409A9999999999014061
:10998000C3F5285C8FA272400000000000FEAA40D0
:109990009A999999FD6F2F41C3F5285C8F127140F8
:1099A000980700200000303F000024400022014BB7
:1099B0001A607047A0070020034B9B7A13B1052261
:1099C000024B5A60704700BF64100020A0070020BF
:1099D0000422014B5A607047A0070020034B1A7AFB
:1099E000202A04BF00221A72704700BFA00700207F
:1099F0007047212810B508D1114B1B681B7803F064
:109A00007F03212B19D0022010BD2028FBD10C4B45
:109A10000C4A1B681B78107203F07F03212B0A4B42
:109A200018BF0023002BEED00024054A2046126800
:109A3000936154829847204610BD044BF4E700BF61
:109A4000C4100020A0070020859A00089D9A0008F5
:109A5000074B1B681B7803F07F03212B06D100F016
:109A6000DF00022814BF0220002070470220704748
:109A7000C410002021B901288CBF022000207047AB
:109A80000220704720B90822024B1B681A827047D7
:109A900001487047C410002048000020FFF7F2BFC3
:109AA00008B5032005F0B2F9064B0246D8604FF422
:109AB0008871054804F0A2FEBDE80840032004F0C8
:109AC0006BBF00BFA0070020CA10002038B50024DB
:109AD000C025324B20461B689C725D72DC7204F01C
:109AE000C9FE4FF40071204604F0E1FE102120462B
:109AF00004F0F4FE4021204605F094F88021204631
:109B000005F07EF8204604F077FF254B204693F8B9
:109B1000341005F028F8204604F03EFF21460120CD
:109B200004F0C5FE2946012005F06AF82021012035
:109B300004F0D4FE2146012004F0E5FE4FF4C0619C
:109B4000022004F0B4FE4FF48071022005F058F8B2
:109B50002146022004F0D7FE2021022004F0BEFEA0
:109B60002146032004F0A3FE4FF48871032005F082
:109B700059F84021032004F0F6FF4FF44051032030
:109B800004F0C1FE2146032004F0A8FE204604F0A4
:109B9000C7FC0122034B5A6038BD00BFC41000202F
:109BA00048000020A0070020014904F0C5BA00BF0A
:109BB00080000020014904F0BFBA00BF88000020E7
:109BC000054B1B68DB78042B04D8044901EBC30167
:109BD00004F0B2BA00207047C410002090000020AA
:109BE00008B5002002F03AFFBDE8084001214FF41B
:109BF000000002F0C1BF0322014B5A60704700BF52
:109C0000A0070020044B9A7A044B12B105225A6037
:109C100070470122FBE700BF64100020A00700206E
:109C2000202110B1024802F08CBC014802F08BBC2C
:109C3000000C01407047684620F007018D4679B559
:109C4000134C144E2368144D9BB2338028883188FE
:109C50000140480505D54FF6FF3323600F4BDB6805
:109C6000984733882A881340990507D54FF6FF5344
:109C70000B4923600B7C0133DBB20B7433881A4031
:109C8000130401D504F0B2FCBDE879408546704765
:109C9000445C00405A1000200A11002048000020B7
:109CA000A007002008B52021074802F04AFC012245
:109CB0000020064B06491A60064A186010604FF4EF
:109CC000E0520A801A6008BD000C0140405C004070
:109CD0000A110020445C004010B50024074B1B68AB
:109CE0009C72FFF7DFFF064B064A1C604FF40643E9
:109CF0001380054A1360054B5C6010BDC410002042
:109D0000445C00400A110020405C0040A007002095
:109D100038B501230024054D20462B60044B1C6000
:109D2000FFF77EFF032320462B6038BD405C0040D8
:109D3000445C0040074A13689BB243F00803136079
:109D400013689BB243F0040313600322024B5A6072
:109D5000704700BF405C0040A007002008B54FF6E8
:109D6000FB7305490A6813400B60FFF74BFF4FF484
:109D700006430B6008BD00BF405C004010B51D4CA1
:109D8000072818BF20702378052B06D8DFE803F0DA
:109D900003070B101823FFF7E1FF062306E0FFF788
:109DA000DDFF042302E0022363700323237006E037
:109DB0006378013BDBB263706378002BF1D010BD98
:109DC0000D4A13689BB243F0100313600523237000
:109DD0000A23637010BD6378013BDBB26370637864
:109DE000002BECD14FF6EF73034A11680B40136060
:109DF000D3E700BFC8100020405C0040142307B523
:109E00008DF8043000238DF805308DF806300123DD
:109E100001A88DF8073002F037FC03B05DF804FBB1
:109E200007B5FFF7DDFEFFF7E9FF04F0C5FB0121F1
:109E3000082002F095FE2023ADF8043003238DF8AE
:109E40000630102301A904488DF8073002F00DFBFD
:109E500003B05DF804FB00BF000C0140FFF7CEBF6C
:109E6000FFF756BF0A4B30B50446D86878B15A6838
:109E7000052A0BD10022074DD9688A4202D300225D
:109E8000DA6030BD515DA1540132F5E7002030BDEC
:109E9000A0070020CA100020084A10B5D368082B7C
:109EA0000AD90023064C195DC1540133092BFAD19C
:109EB00000230120D36010BD002010BDA0070020AA
:109EC000CA10002010B5074C8AB22160C02104F0EE
:109ED00083FC2188012004F025FEBDE8104001200C
:109EE00004F04BBDA0070020704710B5FFF72CFC15
:109EF000074C2368C01AB0F5FA7F07D9054AD36822
:109F000083F40063D360FFF71FFC206010BD00BF27
:109F10000C110020000C01407047704770477047DB
:109F2000054B064AD3F80310054B19B99B889BB221
:109F3000536070471B89FAE7280A00209C0A00201A
:109F4000006C004070477047704710B5FAF7AEFAE2
:109F500005280E4C0ED8012363600D4B1B7843B1CE
:109F60000C4B62681A600C4B62B91A6842F0080226
:109F70001A6010BDFAF79AFA40F2F9339842EAD81B
:109F80000023E9E71A6822F00802F1E79C0A0020A2
:109F9000970A0020880A0020300A002000000000F4
:109FA000014B1878704700BFB4070020024B03EB49
:109FB00080004068704700BFB40700202DE9F74FCC
:109FC000754CE36993B1754D2E787EB9FFF7BCFBF4
:109FD000734B1B68C01A0028E369B8BF404298421F
:109FE00004D9304601F0FAF801232B70236A93B1AB
:109FF0006C4D2E787EB9FFF7A7FB6B4B1B68C01A20
:10A000000028236AB8BF4042984204D9304601F084
:10A01000E5F801232B70FFF797FB644C237B04EBDF
:10A0200083039B68C01A0028B8BF40420A2823DD7A
:10A03000FFF78AFB21210746207B00F0B7FC06468C
:10A04000257B04EB85052869301A05F0C9FC80469C
:10A05000A868381A05F0C4FC0146404605F0C8FD62
:10A0600005F088F84AA3D3E9002305F0D7F805F0F6
:10A0700085FBAF6068602E613521207B00F096FC87
:10A0800010F0400705460DD0207B01F0A7F8012114
:10A09000237B474AD154474A0F33D15C012904BF7F
:10A0A0000221D154207B444E06EB40135B69002B08
:10A0B00059D0222100F07AFC94F80C80002806EB9D
:10A0C00048135B69B8BF404298424CD904EB08037F
:10A0D0001B7D6BB93421404600F068FC342140F40C
:10A0E0008062404600F038FC0122237B23441A752D
:10A0F000637DDFF8CCB06BB998465FFA88F0FAF769
:10A1000058F90BF8080008F10108B8F1080FF4D16C
:10A11000012363754FF027084FF0000902222749F9
:10A12000DFF890A05FFA89F08DE80600FAF741F9B0
:10A130009DE806001BF8093083424AD009F1040368
:10A1400051F823300BF80900022B3BD0032B03D02E
:10A15000012B3ED100283CD01AF80830012B08BF53
:10A160000AF8082035E094F80C8004EB08031B7D06
:10A17000002BBDD03421404600F018FC342120F4DF
:10A180008062404600F0E8FB237B00222344AEE7D8
:10A19000FCA9F1D24D62904008000020050F00207C
:10A1A000000F0020A90E0020F80E0020B4070020A8
:10A1B000FC0900200C0F0020000A0020C80E00201F
:10A1C000CA07002028B91AF80800012801D10AF8A6
:10A1D000083009F10109B9F1080F08F10108A1D10E
:10A1E000237B15F0010104EB030200F0D580917F81
:10A1F00071B901219177774A1A44127BD20707D5AA
:10A200008B40754A1B33D15C012904BF0221D15414
:10A21000237B15F0020104EB030200F0CA80D17F1A
:10A2200081B90121D1776B4A1A44527B12F0010F98
:10A2300008D0694A0E3312F81310012904BF022115
:10A2400002F8131015F0800100F0C080237B624AF1
:10A250000333D05C012801D10220D05447B1237BC5
:10A260005D4A0F33D05C012801D10220D054F9B1EE
:10A27000DFF870E1207B9EF8003043FA00F2D1074E
:10A2800011D50121DFF860C101FA00F28CF800203D
:10A29000DFF858C18CF800105049097819B923EA41
:10A2A00002038EF800308022352100F055FB27B1E3
:10A2B00040223521207B00F04FFB207B06EB401332
:10A2C0001B690BB36A051FD4392100F06FFB2121F4
:10A2D0000746207B00F06AFB237B381A06EB43120B
:10A2E00000281269B8BF404290420DD9184600F0CC
:10A2F00075FF0121237B3A4AD154374A1533D15C8B
:10A30000012904BF0221D154207B06EB4013DB68F6
:10A3100003B36B051ED4FAF7B9F921210546207B5A
:10A3200000F044FB237B281A06EB43160028F26852
:10A33000B8BF404290420DD9184600F04FFF0121AE
:10A34000237B274AD154244A1533D15C012904BF09
:10A350000221D154FFF7F8F9236AC01A0028B8BFC8
:10A3600040420A2804DDFAF7F1F8FFF7EDF9206220
:10A37000FAF7B8FA40BB257835B900F0A9FA2846B3
:10A3800000F02CFF01232370207B00F05FF80023F6
:10A39000237303B0BDE8F08F907F00283FF438AFFF
:10A3A00091770C4A1A44127B90077FF531AF5B001E
:10A3B00027E7D07F00283FF445AFD177054A1A44FC
:10A3C000527B12F0020F33E70023DCE7002F3FF44B
:10A3D00074AF44E7C80E00200C0F0020B00E002020
:10A3E000B20E0020B80E0020B30E00203B0F00205C
:10A3F00073B5134E0446335C0D463BB1114B262119
:10A4000053F8202000F0A8FA0023335585EAE572BE
:10A41000A2EBE5722046272100F09EFA01220A4BAA
:10A42000002D1A554FF00003D8BF0222009301926D
:10A4300020211A46204600F05BFA02B070BD00BF32
:10A44000240A0020200A0020F50900202DE9F04F01
:10A45000352185B0044600F0A9FA0346C0486101E1
:10A460004618327ED6F8048012F0400F18BF4158CB
:10A470004FEA530B03F0010517BF0BF0010950F829
:10A4800001A05FFA85FBC1F1000A12BFC8F1000804
:10A490005FFA85F90BF0010B150602F03F060393F6
:10A4A000204613D5FAF774FAB0FA80F77F09721EC6
:10A4B000039B072A00F27B81DFE812F00E000E00FA
:10A4C0000E000E001201120112011201FAF760FAD9
:10A4D000071C18BF0127EAE7A24D2A5D013A0E2AA0
:10A4E00000F26581DFE812F00F001E002D003B0036
:10A4F0004B00540063007200A200C400CA00630154
:10A50000F800E101DC013421204600F04FFA01227D
:10A5100005EB84035860023E934B96421A551BD8B4
:10A5200002231AE005EB84035A6842F00202342148
:10A53000204600F011FA51462046FFF759FF032349
:10A540000BE0BBF1000F00F032812121204600F02A
:10A550002DFA864B43F8240004232B5527E105EB05
:10A5600084035A6842F001023421204600F0F4F9D5
:10A57000CAF100012046FFF73BFF0523EDE7B9F1E3
:10A58000000F00F01481204600F028FE0623E4E7C7
:10A5900005EB84035A683421204622F0030200F0C0
:10A5A000DBF941462046FFF723FF0723D5E7B9F142
:10A5B000000F40F0FC8049462046FFF719FFC8F124
:10A5C00000012046FFF714FF0823C6E7B9F1000F8A
:10A5D00000F0ED802121204600F0E8F90646002138
:10A5E0002046FFF705FF614A342152F82430204607
:10A5F0009B1B42F8243005EB84035A6822F00302C7
:10A6000000F0AAF942462721204600F0A5F932467B
:10A610002D21204600F0A0F9002320210193009372
:10A620001A46204600F064F9092396E7990540F19F
:10A63000BE802121204600F0B9F94D4B0021186061
:10A640002046FFF7D5FE00222D21204600F084F998
:10A6500000222121204600F07FF9033E002239210B
:10A66000204600F079F9012E38D8C8F10001B2E097
:10A67000B9F1000F00F09B800B236EE7B9F1000FDA
:10A6800040F095802121204600F090F94946064689
:10A690002046FFF7ADFE05EB84035A68342122F013
:10A6A0000302204600F058F942462721204600F0D8
:10A6B00053F902222D2196FBF2F2204600F04CF9CC
:10A6C0004B46CDF80490CDF800901A462021204644
:10A6D00000F00EF90D2340E79A0568D50E233CE7FC
:10A6E000204D2A5D013A0E2A61D8DFE802F00819F0
:10A6F0002A4354606360608B9579B9DED9000122EA
:10A70000194B342120461A5500F050F905EB84030B
:10A71000062E58603FF404AF082E7FF41DAFFFE60D
:10A72000062E05D105EB84035A6822F00302FCE6ED
:10A73000082E7FF400AF05EB84035A6822F0030271
:10A74000F5E6731F012B07D8BBF1000F04D0062ECE
:10A750003FF402AF0F2300E74FB30C23FDE600BF29
:10A76000000A0020D8070020F5090020AC0E0020C8
:10A77000C40E0020052E05D105EB84035A6822F093
:10A780000302EFE6072E7FF4F3AE05EB84035A686D
:10A7900022F00302E8E6731F012B05D8B9F1000F80
:10A7A00002D0052ED6D1BBE6002F7FF4FEAE05B059
:10A7B000BDE8F08F002FFAD1073E012E0AD905EB34
:10A7C00084035A68342122F0030242F00202204638
:10A7D00000F0C2F841462046FFF70AFE0A23BCE615
:10A7E000002FE4D1073E012E7FF63FAF05EB840337
:10A7F0005A68342122F0030242F00102204600F0A0
:10A80000ABF832E7002FD2D02121204600F0CEF85D
:10A8100005EB840398602FE7002FC8D12121204643
:10A8200000F0C4F8064605EB8409D9F80420342169
:10A8300022F00302204600F08FF8424627212046EE
:10A8400000F08AF8D9F808202D211644022220466B
:10A8500096FBF2F200F080F8019700973B4634E750
:10A860009B05A4D50E23212120462B5500F09EF8F0
:10A87000124B002118602046FFF7BAFD2046002247
:10A880002D2100F069F820460022212100F064F813
:10A8900000223921204605B0BDE8F04F00F05CB839
:10A8A00000212046FFF7A4FD18E705EB84035A6852
:10A8B0003421204600F050F800234EE6C40E00205C
:10A8C000024B1A5C0AB901221A547047D8070020BB
:10A8D000024B1A5C0AB10F221A547047D8070020A5
:10A8E000014B185C704700BFD80700200000000033
:10A8F0002DE9F84391461F4680460E46002241F05E
:10A90000800101209DF820509DF82440FAF7A2F91B
:10A91000002249460120FAF79DF93946002201201C
:10A92000FAF798F9294600220120FAF793F9012253
:10A930002146104647EA0927FAF78CF945EA072528
:10A9400006F07F06034B464444EA052443F82640BC
:10A95000BDE8F883E407002070B5144606460D46AE
:10A96000002241F080010120FAF774F90022210E43
:10A970000120FAF76FF90022C4F307410120FAF72A
:10A9800069F90022C4F307210120FAF763F90122D3
:10A99000E1B21046FAF75EF905F07F05024B354447
:10A9A00043F8254070BD00BFE407002038B5264BB2
:10A9B00001F07F055B5D002B41D00022294601207C
:10A9C000FAF748F9002201201146FAF743F900226C
:10A9D00001201146FAF73EF9002201201146FAF74C
:10A9E00039F9012200211046FAF734F9002201203A
:10A9F0001146FAF72FF9002201201146FAF72AF939
:10AA00000022040211460120FAF724F9002204432F
:10AA100011460120FAF71EF9012224020443002105
:10AA20001046FAF717F92402222D40EA040001D05B
:10AA3000422D08D1030206D540F07F4038BD034BBC
:10AA4000054453F8250038BD990B0108E4070020A0
:10AA500070B50B4C0546221892F800220E465AB9E2
:10AA60006C21FFF7A3FF06F00F0320F00F021A433B
:10AA70006C212846FFF770FF631983F8016270BDEF
:10AA8000E407002038B50C466C210546FFF78EFF21
:10AA9000240104F0700420F0700222432846BDE82F
:10AAA00038406C21FFF758BF38B50C466C2105467D
:10AAB000FFF77CFFE40304F4C03420F4C0322243E7
:10AAC0002846BDE838406C21FFF746BF38B50C4634
:10AAD0006C210546FFF76AFF240504F4700420F496
:10AAE000700222432846BDE838406C21FFF734BF8E
:10AAF00038B50C466C210546FFF758FF240604F0D4
:10AB0000706420F0706222432846BDE838406C2112
:10AB1000FFF722BF38B50D466C210446FFF746FF0C
:10AB20003DB140F080422046BDE838406C21FFF73F
:10AB300013BF20F08042F6E738B50D466C2104467D
:10AB4000FFF734FF3DB140F400222046BDE8384015
:10AB50006C21FFF701BF20F40022F6E738B50D465F
:10AB60006C210446FFF722FF3DB140F480222046CD
:10AB7000BDE838406C21FFF7EFBE20F48022F6E7F5
:10AB800038B50D466C210446FFF710FF3DB140F487
:10AB900080422046BDE838406C21FFF7DDBE20F43E
:10ABA0008042F6E738B50D466C210446FFF7FEFEFD
:10ABB0003DB140F400522046BDE838406C21FFF71B
:10ABC000CBBE20F40052F6E738B50D466C210446A2
:10ABD000FFF7ECFE3DB140F480522046BDE838401E
:10ABE0006C21FFF7B9BE20F48052F6E738B50C4669
:10ABF0006C210546FFF7DAFE230748BF20F07000FE
:10AC00004FEA04124CBF40F4006020F4076002F0E9
:10AC1000700202436C212846BDE83840FFF79CBE15
:10AC200038B50C466C210546FFF7C0FEE40104F47C
:10AC3000F06420F4F06222432846BDE838406C21DD
:10AC4000FFF78ABEFFF7ECBF38B50D466C2104460E
:10AC5000FFF7ACFE3DB140F000522046BDE8384061
:10AC60006C21FFF779BE20F00052F6E738B50D46AB
:10AC70006C210446FFF79AFE3DB140F08052204619
:10AC8000BDE838406C21FFF767BE20F08052F6E740
:10AC900008B5074B034493F800222AB96C21FFF74B
:10ACA00085FE00F00F0008BD93F8010208BD00BF4B
:10ACB000E407002008B56C21FFF778FEC0F302100E
:10ACC00008BD08B56C21FFF771FEC0F3C13008BDA7
:10ACD00008B56C21FFF76AFEC0F3035008BD08B544
:10ACE0006C21FFF763FEC0F3036008BD08B56C215B
:10ACF000FFF75CFEC0F3807008BD08B56C21FFF75C
:10AD000055FEC0F3C04008BD08B56C21FFF74EFEEC
:10AD1000C0F3804008BD08B56C21FFF747FEC0F3C3
:10AD2000803008BD08B56C21FFF740FEC0F340300D
:10AD300008BD08B56C21FFF739FEC0F3003008BD2F
:10AD400008B56C21FFF732FEC0F30213020548BFBD
:10AD500043F00803184608BD08B56C21FFF726FE2E
:10AD6000C0F3C31008BDFFF7F7BF08B56C21FFF7AC
:10AD70001DFEC0F3407008BD08B56C21FFF716FE3C
:10AD8000C0F3007008BD38B50C466D210546FFF7CD
:10AD90000DFE640104F0600420F0600222432846A6
:10ADA000BDE838406D21FFF7D7BD38B50C466D21A1
:10ADB0000546FFF7FBFD640304F4C04420F4C042E1
:10ADC00022432846BDE838406D21FFF7C5BD38B5A0
:10ADD0000C466D210546FFF7E9FD240204F470647A
:10ADE00020F4706222432846BDE838406D21FFF709
:10ADF000B3BD38B50C466D210546FFF7D7FD04F00D
:10AE00000F0420F00F0222432846BDE838406D2190
:10AE1000FFF7A2BD38B50D466D210446FFF7C6FD0C
:10AE200020F47F0040EA05426D212046BDE838400D
:10AE3000FFF792BD38B50D466D210446FFF7B6FD0C
:10AE40003DB140F400422046BDE838406D21FFF797
:10AE500083BD20F40042F6E738B50D466D21044667
:10AE6000FFF7A4FD3DB140F080722046BDE83840B8
:10AE70006D21FFF771BD20F08072F6E708B56D21F6
:10AE8000FFF794FDC0F3411008BD08B56D21FFF731
:10AE90008DFDC0F3413008BD08B56D21FFF786FD7B
:10AEA000C0F3032008BD08B56D21FFF77FFD00F05A
:10AEB0000F0008BD08B56D21FFF778FD0314D8B267
:10AEC0001B0648BF60F0FF0008BD08B56D21FFF705
:10AED0006DFDC0F3C03008BD08B56D21FFF766FDFC
:10AEE000C0F3006008BD38B50C4670210546FFF779
:10AEF0005DFD04F0030420F4401242EA04522846A7
:10AF0000BDE838407021FFF727BD38B50D467021E8
:10AF10000446FFF74BFD3DB140F400222046BDE85A
:10AF200038407021FFF718BD20F40022F6E738B54D
:10AF30000D4670210446FFF739FD3DB140F48022F3
:10AF40002046BDE838407021FFF706BD20F480227E
:10AF5000F6E738B50C4670210546FFF727FD04F0EB
:10AF6000030420F4403242EA04422846BDE8384057
:10AF70007021FFF7F1BC38B50D4670210446FFF78C
:10AF800015FD20F47F4040EA052270212046BDE8EF
:10AF90003840FFF7E1BC38B50D4670210446FFF795
:10AFA00005FD20F0FF0045EA000270212046BDE8C3
:10AFB0003840FFF7D1BC08B57021FFF7F7FCC0F3AC
:10AFC000015008BD08B57021FFF7F0FCC0F3C04088
:10AFD00008BD08B57021FFF7E9FCC0F3804008BD4B
:10AFE00008B57021FFF7E2FCC0F3014008BD08B5C9
:10AFF0007021FFF7DBFCC0F3072008BD08B5702106
:10B00000FFF7D4FCC0B208BD70B50E466F211546DF
:10B010001C46FFF7CBFC16B1C0F30903336015B132
:10B02000C0F304432B700CB1000E207070BD37B517
:10B03000FEF78AFB0446FEF787FB001B0028B8BF1B
:10B0400040420928F7DD002113220846FFF784FC5F
:10B05000022253238DE80C000022412310466C216C
:10B06000FFF746FC062503238DE82800002309216D
:10B070001A461846FFF73CFC00240A2101230191DF
:10B08000224620460094FFF733FC3F4A1021537FAD
:10B090002046DB080193137F2246DB080093072339
:10B0A000FFF726FC394A70212046FFF755FC204661
:10B0B000FFF7EEFD364B83F80102042083F80042CF
:10B0C000FDF714FC01301CD00520FDF70FFC0B210F
:10B0D00002462046FFF740FC2846FDF707FCC1B2B8
:10B0E0002046FFF7B5FC0720FDF700FCC1B2204663
:10B0F000FFF7C8FC0820FDF7F9FBC1B22046FFF7B7
:10B100008FFD002220211046FFF726FC00222D2172
:10B110001046FFF721FC002221211046FFF71CFCFE
:10B12000012223210020FFF717FCDC22242100202C
:10B13000FFF712FC46F6DB0225210020FFF70CFC8E
:10B1400040F2B71226210020FFF706FC4DF2B7129D
:10B1500027210020FFF700FC40F2B7122821002031
:10B16000FFF7FAFBDC222A210020FFF7F5FB0A2279
:10B170002B210020FFF7F0FB14210020054A03B02B
:10B18000BDE83040FFF7E8BB000A00201E000CC4F9
:10B19000E4070020FFFF0F0038B5074C044494F883
:10B1A000001241B994F80152FFF752FC012384F8D0
:10B1B000015284F8003238BDE4070020064B0344F6
:10B1C00093F8002232B1002293F8011283F8002292
:10B1D000FFF73EBC704700BFE407002037B50125EC
:10B1E0000C4BC4B21D540C4B00221D542721204689
:10B1F000FFF7B2FB20464FF6FF722621FFF7ACFBAC
:10B200000023019500931A4620212046FFF770FB8A
:10B2100003B030BDF5090020240A0020002808B53D
:10B220000BDB03F095FF0AA3D3E9002304F020F918
:10B2300005F02AF904F0A2FA08BD03F089FF04A37F
:10B24000D3E9002304F014F905F08EF8F2E700BF0B
:10B2500034F7FFFF7F84EE3F08B503F079FF06A3C4
:10B26000D3E9002304F004F905F00EF904F086FA9E
:10B2700008BD00BFAFF30080EB1100A2941A5D403F
:10B28000002808B50BDB03F063FF0BA3D3E9002311
:10B2900003F0C4FF05F068F804F070FA08BD03F08D
:10B2A00057FF05A3D3E9002303F0B8FF05F0ECF83E
:10B2B000F2E700BFAFF3008034F7FFFF7F84EE3F7B
:10B2C00008B504F08DFB03F055FF05A3D3E9002377
:10B2D00003F0A4FF05F048F804F050FA08BD00BFE1
:10B2E000EB1100A2941A5D40704700BF7047FEE763
:10B2F000FEE7FEE7FEE7704770477047704770470C
:10B300007047704770477047704770477047704785
:10B310007047704770477047704770477047704775
:10B320007047014B1B681847B40E0020014B1B6887
:10B33000184700BF080F0020014B1B68184700BFCB
:10B34000BC0E0020014B1B68184700BFC00E002038
:10B350007047704770477047704770477047704735
:10B360007047704770477047704770477047704725
:10B370007047704770477047704770477047704715
:10B380007047704770477047704770477047704705
:10B390007047704770477047704700BF08B5154B3E
:10B3A000984213D003F5A053984218D0A3F5C05388
:10B3B00098421DD101214FF4007001F0E9FB0021FA
:10B3C0004FF40070BDE8084001F0E2BB01214FF4EA
:10B3D000806001F0DDFB00214FF48060F2E7012185
:10B3E0004FF4004001F0D4FB00214FF40040E9E7A6
:10B3F00008BD00BF0028014043680A7923F4702388
:10B4000023F4807343EA02230A6810B513434360B0
:10B410008A68CB6884681343084A224013434A79F8
:10B4200043EA420383600A7CC36A013A23F470034F
:10B43000D2B243EA0253C36210BD00BFFDF7F1FF71
:10B4400000230360037143718360C36001230374AD
:10B450007047836819B143F001038360704723F09C
:10B460000103FAE7836819B143F48073836070477E
:10B4700023F48073FAE7C9B2436812B119434160FB
:10B48000704723EA0101FAE7836843F00803836009
:10B4900070478068C0F3C0007047836843F00403BE
:10B4A000836070478068C0F380007047836819B17B
:10B4B00043F4A0038360704723F4A003FAE7806895
:10B4C000C0F3805070474368013923F4604343EA76
:10B4D000413343607047436819B143F400634360EC
:10B4E000704723F40063FAE7092970B51BD90726D2
:10B4F000A1F10A04C56804EB4404A64025EA060548
:10B5000003FA04F42C43C460062A18D81F24013A15
:10B51000436B02EB8202944023EA040301FA02F235
:10B520001A43426370BD0724056901EB4106B4402C
:10B5300025EA040503FA06F42C430461E4E70C2A27
:10B540000CD81F24073A036B02EB8202944023EAD3
:10B55000040301FA02F21A43026370BD1F240D3A7C
:10B56000C36A02EB8202944023EA04039140194328
:10B57000C16270BD836819B143F480138360704762
:10B5800023F48013FAE7C06C80B27047014B18684F
:10B59000704700BF4C240140436819B143F48063F5
:10B5A0004360704723F48063FAE7436819B143F4BA
:10B5B00080534360704723F48053FAE7836823F491
:10B5C000E043194381607047836819B143F4004335
:10B5D0008360704723F40043FAE7836819B143F4AA
:10B5E00002138360704723F40213FAE78068C0F304
:10B5F00040507047092970B51CD90726A1F10A04EB
:10B60000C56804EB4404A64025EA060503FA04F4E1
:10B610002C43C460836B0232C3F30154121B1F24FA
:10B62000D2B202EB8202944023EA04039140194310
:10B63000816370BD0724056901EB4106B44025EA2A
:10B64000040503FA06F42C430461E3E7836B013934
:10B6500023F4401343EA0153836370474250704719
:10B660002830405880B27047436823F4400323F4E5
:10B6700000731943416070474162826270474368BA
:10B6800023F01F03194341607047054B9A6818B1B6
:10B6900042F400029A60704722F40002FAE700BF09
:10B6A000002401400368194214BF012000207047A4
:10B6B000C943016070474368006810EA112004D054
:10B6C000C9B2194214BF0120002070476FEA11214E
:10B6D0000160704708B501214FF0007001F064FA75
:10B6E000BDE8084000214FF0007001F05DBA012371
:10B6F0002C4A1360536813F0010351D00378012BD7
:10B7000013680CBF43F0800323F080031360437879
:10B71000012B244B1A680CBF42F0400222F0400279
:10B720001A608278012A1A680CBF42F0200222F0C7
:10B7300020021A60C378012B1A4B1A680CBF42F022
:10B74000100222F010021A600279012A1A680CBF56
:10B7500042F0080222F008021A604379012B114BD3
:10B760001A680CBF42F0040222F004021A60C37986
:10B7700082791B0643EA8273027A43EA0243427AE1
:10B7800043EA02534289013A1343064AD3611368DC
:10B7900023F0010313605068C04300F001007047BC
:10B7A000184670470064004030B501250378364ADA
:10B7B0009D40ADB2EC43D2F8001241F00101C2F855
:10B7C0000012D2F81C122140C2F81C128178002904
:10B7D00034D1D2F80C12DB002140C2F80C1242899D
:10B7E000C18841EA024103F1804202F5C842C2F831
:10B7F00040128388018943EA0143C2F84432437806
:10B800002149A3BBD1F804322340C1F80432838913
:10B810001D4A83BBD1F814321C40C1F81442837B0B
:10B82000012B02BFD2F81C322B43C2F81C32D2F8D3
:10B83000003223F00103C2F8003230BD0129DED10D
:10B84000D2F80C12DB002943C2F80C128188C2889E
:10B8500003F1804342EA014203F5C843C3F84022A2
:10B860000189428942EA0142C3F84422C7E7D1F87C
:10B8700004322B43C9E7012B02BFD2F814322B4309
:10B88000C2F81432CBE700BF00640040002303700D
:10B8900043708370C370037143718371C371032359
:10B8A000037202234372012343817047044B5A6998
:10B8B00011B110435861704722EA0000FAE700BF57
:10B8C000006400402A4B02469968F0B5480132D422
:10B8D0009968090148D49B68DB0047D40420F0BD77
:10B8E0001168D3F880614905116021433143C3F8E1
:10B8F0008011917A01F00F019172D3F8844124F004
:10B900000F04C3F88441D3F884412143C3F8841160
:10B91000D2F80B4005F1804101F5C841C1F88841DA
:10B92000D2F80F20C1F88C21D3F8802142F0010217
:10B93000C3F88021F0BD0020050105F1804303F527
:10B94000C843D3F8801101F00101C3F88011117AC6
:10B95000547A0029C4D05668D3F88071F600314378
:10B96000214356603943C2E70120E5E70220E3E7BF
:10B9700000640040012814D003D302281FD0002304
:10B980000CE016498B688A6889689B0003F0040301
:10B99000C1F380610B4302F002021343104AD05CF2
:10B9A00070470E498B688A689B09120A02F00202EE
:10B9B00003F0040313438A68C2F3C062EDE707494A
:10B9C0008B688A689B0B120C02F0020203F00403DE
:10B9D00013438A68C2F30072DFE700BF00640040CF
:10B9E000190C0108012809D002D302280BD0704796
:10B9F000074A936843F0800393607047044A936852
:10BA000043F40043F8E7024A936843F40003F3E782
:10BA100000640040034B202208B9DA6070471A61C5
:10BA2000704700BF0064004020B9064BD86800F0A2
:10BA300003007047012802D1024B1869F7E7002084
:10BA4000704700BF00640040030103F1804202F52B
:10BA5000C84210B4D2F8B04104F004040C72B4BB74
:10BA6000D2F8B041640D0C60D2F8B04103F18043CC
:10BA700004F002044C72D2F8B44103F5C84304F058
:10BA80000F048C72D2F8B42110BC120ACA74D3F815
:10BA9000B821CA72D3F8B821120A0A73D3F8B821B0
:10BAA000120C4A73D3F8B821120E8A73D3F8BC2152
:10BAB000CA73D3F8BC21120A0A74D3F8BC21120C41
:10BAC0004A74D3F8BC311B0E8B74FFF7A3BFD2F8B6
:10BAD000B041E4084C60C7E7044B1A6842F0020228
:10BAE0001A601868C0F34000704700BF006400404F
:10BAF000054B1A6822F002021A60186880F00200F2
:10BB0000C0F34000704700BF00640040034B9B69D6
:10BB1000034214BF01200020704700BF00640040B2
:10BB2000024A936923EA0000906170470064004074
:10BB3000202840D011D806282ED005D8042835D08A
:10BB4000052824D00020704707282AD00828F9D1DA
:10BB5000214BD868C0F300107047B0F5007F30D09B
:10BB600007D840282AD0B0F5807FEBD11A4B9869CE
:10BB70000FE0B0F5803F2CD0B0F5003F26D0B0F5F7
:10BB8000806FDFD1144B9869C0F380007047124B6F
:10BB9000986800F0010070470F4B9868C0F30020D0
:10BBA00070470D4B9868C0F3004070470A4BD86847
:10BBB000C0F3C0007047084B1869F9E7064B1869D5
:10BBC000C8E7054B9869C0F340007047024B5868BE
:10BBD000C0E7014B5868EBE700640040202835D0EF
:10BBE0000CD8062826D004D8042829D005281DD032
:10BBF0007047072821D0082826D07047B0F5007F6D
:10BC000030D005D8402825D0B0F5807F24D07047AB
:10BC1000B0F5803F2BD0B0F5003F2CD0B0F5806F51
:10BC200028D1164A936923F0040319E00122134B2B
:10BC30009A6070474FF48072F9E74FF48032F6E76C
:10BC400008220E4BDA6070471022FAE708220B4BED
:10BC50001A6170471022FAE7084A936923F001033A
:10BC600093617047054A936923F00203F8E70822BD
:10BC7000024B5A6070471022FAE700BF0064004090
:10BC8000036823F0010303600023036043608360C3
:10BC9000C3602D4B984243D011D83C3B984230D0E2
:10BCA00006D8283B984222D01433984224D07047BB
:10BCB000264B98422AD0143398422CD07047244BFC
:10BCC00098423AD008D8A3F5677398422ED003F56E
:10BCD000627398422FD070471E4B98422FD0143376
:10BCE00098422ED0283B98421FD11B4A0AE01B4A9B
:10BCF000536843F00F0317E0184A536843F0F0030A
:10BD000012E0164A536843F470630DE0134A536817
:10BD100043F4704308E0114A536843F4702303E08E
:10BD20000E4A536843F47003536070470B4A5368DC
:10BD300043F07063F8E7084ADAE7074ADDE7064AA6
:10BD4000E5E7054AE8E700BF6C0002404400024016
:10BD50001C0402404404024000040240000002406F
:10BD60008B6810B50C6A026823430C6922F4FF4209
:10BD700023434C6922F0700223438C692343CC692E
:10BD800023434C6A23438C6A234313430360CB68E9
:10BD900043600B6883604B68C36010BD0023036081
:10BDA00043608360C360036143618361C361036275
:10BDB000436283627047036819B143F00103036073
:10BDC000704723F00103FAE7036812B119430160D9
:10BDD000704723EA0101FAE7406880B27047C30068
:10BDE0004CBF044B044B1B68034214BF01200020CE
:10BDF000704700BF0004024000000240FFF7EFBFA1
:10BE0000C3004CBF014B024B586070470004024016
:10BE100000000240FFF7F4BF0022044B1A605A6092
:10BE20009A60DA60024A5A61704700BF000401401C
:10BE3000FFFF0700827930B50168037942B3CC4334
:10BE4000184A03F18043156803F5823325401560D5
:10BE500055682C4054601C6821431960036894683D
:10BE6000D9430C409460D4682140D16041791029B5
:10BE700006D1916819439160D1680B43D36030BDFE
:10BE800001F1804202F5823211680B43136030BD2C
:10BE900003F1804303F582331A6822EA0101196035
:10BEA00030BD00BF0004014000230C220360037179
:10BEB000427183717047024A1369184310617047D9
:10BEC00000040140034B5B69034214BF01200020C2
:10BED000704700BF00040140014B5861704700BF2C
:10BEE00000040140054B1A685B69034004D002421C
:10BEF00014BF01200020704718467047000401401D
:10BF0000014B5861704700BF00040140044B1A68A0
:10BF100002F038021A601A6810431860704700BFB8
:10BF200000200240044B1A6822F008021A601A68C6
:10BF300010431860704700BF00200240044B1A688D
:10BF400022F010021A601A6810431860704700BF90
:10BF500000200240034B044A5A6002F188325A60C2
:10BF6000704700BF0020024023016745024A136961
:10BF700043F080031361704700200240014BD869F1
:10BF80008008704700200240014B186A704700BFCC
:10BF900000200240024BD869C0F34000704700BF48
:10BFA00000200240024B1868C0F34010704700BFE9
:10BFB00000200240044B1A6911B110431861704708
:10BFC00022EA0000FAE700BF002002400128064BE9
:10BFD00003D1D86900F001007047DB68184214BF34
:10BFE00001200020704700BF00200240014BD860B4
:10BFF000704700BF00200240084BDA68D10709D41F
:10C00000DA68520708D4DB6813F0100F14BF03205E
:10C010000420704701207047022070470020024032
:10C0200073B504460025FFF7E7FFFF2601280FD16F
:10C0300014B9052002B070BD01950196019B1BB992
:10C04000FFF7DAFF013CF1E7019B013B0193F5E7C4
:10C05000002C08BF0520EDE738B5054640F6FF7017
:10C06000FFF7DEFF042815D10B4C40F6FF70236963
:10C0700043F0020323616561236943F040032361B8
:10C08000FFF7CEFF012805D0236923F00203DB046C
:10C09000DB0C236138BD00BF0020024010B540F624
:10C0A000FF70FFF7BDFF042814D10B4C40F6FF7062
:10C0B000236943F004032361236943F040032361B0
:10C0C000FFF7AEFF012805D0236923F00403DB044A
:10C0D000DB0C236110BD00BF0020024010B540F60C
:10C0E000FF70FFF79DFF04282BD1164C164B40F62E
:10C0F000FF70A36003F18833A360236943F020033A
:10C100002361236943F040032361FFF789FF04287B
:10C110000FD1A52223690F2023F02003DB04DB0CC1
:10C120002361236943F010032361084B1A80FFF752
:10C1300077FF012805D0236923F01003DB04DB0C13
:10C14000236110BD002002402301674500F8FF1F56
:10C1500070B506460F200D46FFF762FF042818D180
:10C160000C4C0F20236943F001032361ABB23380F1
:10C17000FFF756FF042804D12D0C75800F20FFF720
:10C180004FFF012805D0236923F00103DB04DB0CFA
:10C19000236170BD0020024070B505460F200E4699
:10C1A000FFF73EFF042810D1084C0F20236943F00D
:10C1B000010323612E80FFF733FF012805D0236997
:10C1C00023F00103DB04DB0C236170BD002002407F
:10C1D00070B506460F200D46FFF722FF042816D142
:10C1E0000B4C0C4BADB2A36003F18833A360236901
:10C1F0000F2043F0100323613580FFF711FF012862
:10C2000005D0236923F01003DB04DB0C236170BD30
:10C21000002002402301674510B504460F20FFF7B8
:10C22000FFFE04282AD1E443204B214AE1B29A6060
:10C2300002F188329A601A69FF2942F010021A61ED
:10C2400013D1C4F30723FF2B19D1C4F30743FF2BEA
:10C250001DD1240EFF2C22D10420144A136923F08F
:10C260001003DB04DB0C136108E0124B0F20198173
:10C27000FFF7D6FE0428E4D00128EED110BD0D4A08
:10C280000F205381FFF7CCFE0428DED0F4E7094AE3
:10C290000F209381FFF7C4FE0428DAD0ECE7054BAA
:10C2A000A4B2DC810F20FFF7BBFEE5E700200240CF
:10C2B0002301674500F8FF1F38B5054640F6FF70BB
:10C2C000FFF7AEFE042839D11D4C1E4B40F6FF701F
:10C2D000A36003F18833A360236943F02003236143
:10C2E000236943F040032361FFF79AFE04281DD120
:10C2F000236923F02003DB04DB0C2361236943F073
:10C3000010032361104B7DB100221A8040F6FF70AC
:10C31000FFF786FE012811D0094A136923F01003A4
:10C32000DB04DB0C136138BDA522EEE7012805D044
:10C33000236923F02003DB04DB0C236138BD00BF3D
:10C34000002002402301674500F8FF1FF8B5124C9A
:10C35000124B0546A36003F18833A3600F200E46FD
:10C360001746FFF75DFE042814D1236947F0F8074C
:10C3700043F0100323613E43094B35435D800F209A
:10C38000FFF74EFE012805D0236923F01003DB04DC
:10C39000DB0C2361F8BD00BF00200240230167458C
:10C3A00000F8FF1F08B5294B984236D015D8A3F5E1
:10C3B0000063984223D003F58063984226D0A3F50A
:10C3C0000063984240D10121042000F0E1FB0021EC
:10C3D0000420BDE8084000F0DBBB1D4B984223D091
:10C3E00003F58063984226D0A3F5006398422BD1D1
:10C3F0000121402000F0CCFB00214020E9E7012191
:10C40000082000F0C5FB00210820E2E701211020F0
:10C4100000F0BEFB00211020DBE70121202000F00E
:10C42000B7FB00212020D4E70121802000F0B0FBE1
:10C4300000218020CDE701214FF4807000F0A8FB9F
:10C4400000214FF48070C4E708BD00BF0014014014
:10C45000001C0140012108B5084600F099FBBDE829
:10C4600008400021012000F093BBCB782DE9F0417A
:10C47000DA0648BF8A780E8803F00F0548BF1543D7
:10C4800016F0FF0F1AD000214FF0010E4FF00F0CE5
:10C4900002680EFA01F737EA06040BD18C000CFA99
:10C4A00004F822EA080205FA04F4282B42EA0402FE
:10C4B00025D1476101310829EBD10260FF2E1CD93B
:10C4C00000214FF0010E4FF00F0C426801F10804FB
:10C4D0000EFA04F434EA06070BD18F000CFA07F8C1
:10C4E00022EA080205FA07F7282B42EA07020AD1D6
:10C4F000446101310829E9D14260BDE8F081482B4F
:10C5000008BF0761D6E7482B08BF0461F1E74FF683
:10C51000FF730380022383700423C3707047836812
:10C52000194214BF012000207047806880B2704714
:10C53000C368194214BF012000207047C06880B250
:10C54000704701617047416170470AB101617047EE
:10C5500041617047C160704741F4803383618161FC
:10C560008361836983697047054A136823F07F03F9
:10C570001B041B0C194341EA00111160704700BFF6
:10C5800000000140014B1860704700BF1C002042B2
:10C5900030B5134A00F44015B5F5401F536884B216
:10C5A0000ED1556823F0706325F07065556021B198
:10C5B000400D000104FA00F00343094A536030BD06
:10C5C000C2024DBF0322420D1201C0F303454CBF0E
:10C5D000AA4004FA02F223EA020343F07063E6E79A
:10C5E0000000014010B50F2401F0030301F0FC012D
:10C5F00001F1804101F580318A689B009C4022EA6C
:10C6000004028A608A6898401043886010BD00BFA9
:10C610006FF070424FF0FF31094BC3F88010C3F840
:10C620008420C3F88011C3F884210022104602F14F
:10C63000C00101320F2A43F82100F8D1704700BF32
:10C6400000E100E04FF02062084B09495A600022E7
:10C650009A60D9601A615A619A61DA611A625A6203
:10C660004FF0FF329A62DA621A63704700ED00E021
:10C670000000FA0540F0BF60024B40F40030D86083
:10C68000704700BF00ED00E030B5C37802786BB3AF
:10C690001C4BD9684378C943C1F30221C1F104049A
:10C6A000A3400F2424FA01F1FF24807801400B43BA
:10C6B00002F0FC0101F1604101F5614102F003006B
:10C6C000D1F80053C0001B0183406B4004FA00F016
:10C6D00003406B40C1F800330123510902F01F02EF
:10C6E00003FA02F2084B43F8212030BD012153091F
:10C6F00002F01F0201FA02F20349203341F823201D
:10C7000030BD00BF00ED00E000E100E00023037059
:10C7100043708370C3707047F7F71FBDF7F71FBDF5
:10C72000F7F71FBDF7F71FBD0001F7F71EBDF7F7BD
:10C730001FBD024B5868C0F30930704700ED00E0A0
:10C74000012300F01F0293404009044A403052F890
:10C75000202093430CBF01200020704700E100E03F
:10C76000014B1860704700BF00EF00E00122430951
:10C7700000F01F0002FA00F0024A603342F8230082
:10C78000704700BF00E100E0024B5868C0F30900A9
:10C79000704700BF00ED00E0012300F01F0293404E
:10C7A0004009044A803052F8202093430CBF0120F6
:10C7B0000020704700E100E0014B1868704700BF9F
:10C7C00000ED00E021F0604121F07F01014B0143C9
:10C7D0009960704700ED00E0014A024BDA60704753
:10C7E0000400FA0500ED00E0014A024BDA607047F0
:10C7F0000100FA0500ED00E0044B1A6911B1104385
:10C800001861704722EA0000FAE700BF00ED00E07F
:10C81000012300F01F0003FA00F0044B5A6A11B123
:10C8200010435862704722EA0000FAE700ED00E08A
:10C83000114B30B5DC68FF25E443C4F30224C4F196
:10C84000040325FA04F4994004EA02030B43C0F3FD
:10C850000121C0F38110800000F1604000F56D40BF
:10C860008269C9008D4022EA0505856182691B0144
:10C870008B401343836130BD00ED00E00123C0F322
:10C88000832003FA00F0044B5B6A30EA03030CBF19
:10C8900001200020704700BF00ED00E000F01F0104
:10C8A0000120034B88405A6810435860704700BF0E
:10C8B00000ED00E000F01F00431E0120024A9840F6
:10C8C000516808435060704700ED00E00123C0F359
:10C8D000833003FA00F0044B5B6A30EA03030CBFB9
:10C8E00001200020704700BF00ED00E0C0F381434D
:10C8F000094A0BB9D06A7047012B0AD1C0F3015322
:10C90000906ADA00D040022B14BF00F00F00C0B2D2
:10C910007047106B704700BF00ED00E0034B10F450
:10C92000800F0CBF586B986B704700BF00ED00E0A4
:10C930000C4B1A6842F001021A6059680A4A0A4010
:10C940005A601A6822F0847222F480321A601A68DF
:10C9500022F480221A605A6822F4FE025A600022F1
:10C960009A607047001002400000FFF80C4BB0F5D1
:10C97000803F1A6822F480321A601A6822F48022FA
:10C980001A6003D0B0F5802F05D070471A6842F4C2
:10C9900080321A6070471A6842F4A022F9E700BF9B
:10C9A00000100240034A136823F0F80343EAC00072
:10C9B0001060704700100240014B1860704700BFC4
:10C9C00000004242034A536823F47C131943014395
:10C9D0005160704700100240014B1860704700BF63
:10C9E00060004242034A536823F003031843506037
:10C9F000704700BF00100240024B586800F00C0066
:10CA0000704700BF00100240034A536823F0F00350
:10CA100018435060704700BF00100240034A53683B
:10CA200023F4E06318435060704700BF00100240D9
:10CA3000034A536823F4605343EAC00050607047D0
:10CA400000100240044B1A7811B11043187070475F
:10CA500022EA0000FAE700BF09100240014B18600B
:10CA6000704700BFD8004242034A536823F4404352
:10CA700018435060704700BF001002400022064B70
:10CA800001281A701A7002D0042802D0704718705A
:10CA9000704705221A70704720100240014B186041
:10CAA000704700BF80044242024A136A1843106272
:10CAB000704700BF00100240014B1860704700BF74
:10CAC0003C0442421C4A10B5536803F00C03042B8B
:10CAD00001D0082B1FD0194B036053681849C3F3CA
:10CAE0000313CC5C0368E34043605468C4F302243E
:10CAF0000C5D23FA04F484605468C4F3C2240C5D12
:10CB0000E340C3605268C2F3813211440A7CB3FB34
:10CB1000F2F3036110BD53685168C3F38343CC0340
:10CB200003F1020302D407494B43D5E75168890357
:10CB3000F9D40249F8E700BF0010024000127A0061
:10CB4000210C010800093D00044B5A6911B1104342
:10CB50005861704722EA0000FAE700BF0010024067
:10CB6000044B9A6911B110439861704722EA0000A2
:10CB7000FAE700BF00100240044BDA6911B110431C
:10CB8000D861704722EA0000FAE700BF00100240B7
:10CB9000044BDA6811B11043D860704722EA0000F4
:10CBA000FAE700BF00100240044B1A6911B11043AC
:10CBB0001861704722EA0000FAE700BF0010024047
:10CBC000014B1860704700BF40044242014B18609F
:10CBD000704700BF4C004242014B1870704700BFC5
:10CBE000071002404209012A074B07D11B6800F0D9
:10CBF0001F0023FA00F000F001007047022A0CBF6A
:10CC00001B6A5B6AF3E700BF0010024010B540F2F8
:10CC1000FF140A493120FFF7E5FF08704B68013324
:10CC20004B600B7813B94B68A342F3D13120FFF767
:10CC3000D9FF003018BF012010BD00BFE809002057
:10CC4000024A536A43F080735362704700100240F7
:10CC5000034B9B68184214BF01200020704700BF9F
:10CC600000100240014B1870704700BF0A100240CC
:10CC700008B5164B98421FD003F5744398420FD065
:10CC8000A3F57843984220D101214FF48040FFF76B
:10CC90008BFF00214FF48040BDE80840FFF784BFC0
:10CCA00001214FF48050FFF773FFBDE808400021D9
:10CCB0004FF48050FFF76CBF01214FF40040FFF7A5
:10CCC00073FF00214FF40040E6E708BD003C004040
:10CCD000038810B503F441524C880B8823438C8899
:10CCE0002343CC8823430C8923434C8923438C89D9
:10CCF0002343CC89234313439BB20380838B23F4C8
:10CD000000631B041B0C83830B8A038210BD838B7F
:10CD1000F0B523F47B6323F00F031B041B0C838308
:10CD2000022303840B89868B022B87B005460C46B1
:10CD3000B6B23AD08B8801A8002B14BF0227012776
:10CD4000FFF7C0FEE3882289B3F5007F4FF00A03A6
:10CD500001991CBF7F017A4303FB01F308BF120254
:10CD6000B3FBF2F30A2205339BB2B3FBF2F303F0F9
:10CD700001021202C3F34F03991E89B2FE2924BF98
:10CD8000002202231343E28813439BB262882B8460
:10CD900023881343A28843F4006313436289134337
:10CDA0001E43B6B2AE8307B0F0BD0022E4E7002315
:10CDB000038043808380C380038143818381C38157
:10CDC000072303827047002302220380438083806D
:10CDD000C380028143817047038821B19BB243F035
:10CDE00040030380704723F040031B041B0CF8E74B
:10CDF000838B21B19BB243F480638383704723F418
:10CE000080631B041B0CF8E70B0901219940838800
:10CE100089B29BB212B119438180704723EA0101A4
:10CE2000FAE783889BB212B119438180704723EAE5
:10CE30000101FAE781817047808980B270474FF61F
:10CE4000FF63994203880BBF23F480739BB21B04DA
:10CE500043F4807308BF1B0C03807047838821B1A3
:10CE60009BB243F004038380704723F004031B0448
:10CE70001B0CF8E7038823F400631B041B0C0380DE
:10CE800003889BB219430180704703889BB243F427
:10CE9000805303807047038821B19BB243F4005351
:10CEA0000380704723F400531B041B0CF8E701298F
:10CEB00014BF008B808A80B27047008A80B27047AE
:10CEC0000388B1F5804F15BF23F480439BB21B0448
:10CED00043F4804318BF1B0C038070470389194239
:10CEE00014BF012000207047202906D10389038840
:10CEF0009BB243F0400303807047402901D00829CA
:10CF000001D103897047C94389B201817047012368
:10CF100010B58488008901F00F0280B203FA02F292
:10CF20001040A4B205D009098B401C4214BF012057
:10CF3000002010BD552906D1038903889BB243F018
:10CF4000400303807047562901D0532901D103893A
:10CF50007047012301F00F018B40DB439BB203813B
:10CF6000704700BF044B04281A680CBF42F004024B
:10CF700022F004021A60704710E000E0014B586094
:10CF8000704700BF10E000E00128084B04D11A6888
:10CF900042F001021A607047023003D11A6822F091
:10CFA0000102F7E700229A60704700BF10E000E03E
:10CFB000044B1A6818B142F002021A60704722F05E
:10CFC0000202FAE710E000E0014B9868704700BFEA
:10CFD00010E000E0C308022B044B0CBF1B68DB68A9
:10CFE00023FA00F000F00100704700BF10E000E0FD
:10CFF00030B5048C42EA031324F001042404240C09
:10D000000484048B058C24F0F3042404240C1C43B6
:10D0100025F002031B041B0C41F00101A4B20B43D9
:10D020000483038430BD30B5048C120224F0100454
:10D030002404240C0484058B048C42EA033324F07A
:10D04000200225F4407512042D05120C2D0D42EA24
:10D0500001111D4341F01001ADB289B20583018475
:10D0600030BD08B5314B984240D014D8A3F50063C9
:10D0700098422DD003F58063984230D0B0F1804FB4
:10D0800052D101210846FFF78FFD00210120BDE8A4
:10D090000840FFF789BD264B984235D004D8A3F548
:10D0A0008063984229D008BD224B984204D003F5F2
:10D0B000006398422FD008BD01214FF40060FFF7B4
:10D0C00067FD00214FF40060BDE80840FFF760BD38
:10D0D00001210220FFF768FD00210220D7E701218E
:10D0E0000420FFF761FD00210420D0E70121082082
:10D0F000FFF75AFD00210820C9E701211020FFF7A2
:10D1000053FD00211020C2E701212020FFF74CFD34
:10D1100000212020BBE701214FF40050FFF738FD2C
:10D1200000214FF40050CFE708BD00BF000C0040C5
:10D1300000140040002C0140038810B503F08F0359
:10D1400003804C88CB880288234313439BB203801F
:10D150008B8883850B880385054B984203D003F5A4
:10D160000063984201D10B7A03860123838210BDAC
:10D17000002C0140038C30B523F001031B041B0C71
:10D180000384038C8288048B0D8824F070042404AB
:10D19000240C23F002032C431B040D891B0C2B438E
:10D1A0004D8892B22B43CD8885860D4DA84203D081
:10D1B00005F50065A8420FD14D8923F008032B43E4
:10D1C0008D8823F0040322F440722B4352048D898E
:10D1D000520CC9892A430A4382800483038430BDE8
:10D1E000002C0140038C70B523F010031B041B0CB2
:10D1F0000384038C8488028B0D8822F4E04212049D
:10D20000120C42EA05224E880D8923F020031B04EC
:10D2100035431B0C43EA0513CD88A4B20587114D95
:10D2200092B2A8429BB203D005F50065A84215D181
:10D230004D8923F0800343EA05134FF6BF751D4067
:10D240008B8824F4406445EA03138D89C9896404FA
:10D25000640C294344EA81049BB2A4B28480028313
:10D26000038470BD002C0140038C70B523F48073DF
:10D270001B041B0C0384038C8288848B0D8824F090
:10D2800070042404240C4E882C4323F400730D896D
:10D290001B0435431B0C43EA0523CD8892B28587D6
:10D2A000104D9BB2A84203D005F50065A84215D1E8
:10D2B0004D8923F4006343EA05234FF6FF351D40F3
:10D2C0008B8822F4405245EA03238D89C989520490
:10D2D000520C294342EA01129BB292B282808483AB
:10D2E000038470BD002C0140038C70B523F480537F
:10D2F0001B041B0C0384038C8488828B0D8822F40E
:10D30000E0421204120C42EA05224E880D8923F4F1
:10D3100000531B0435431B0C43EA0533CD88A4B2EC
:10D32000A0F84050094D92B2A8429BB203D005F537
:10D330000065A84205D18989C4F30D0444EA81142B
:10D34000A4B284808283038470BD00BF002C01409E
:10D350004A880B8813438A881343CA8813430A896F
:10D3600013434A8913438A8913439BB2A0F844307C
:10D3700070474FF6FF73838000230380C380438090
:10D38000037270470023038043808380C38003813E
:10D3900043818381C381704700230122038043803E
:10D3A0008280C38003817047002303804380838091
:10D3B000C3800381438183817047038821B19BB27D
:10D3C00043F001030380704723F001039B059B0D8D
:10D3D000F8E7B0F8443039B16FEA43436FEA53439A
:10D3E0009BB2A0F844307047C3F30E03F9E7818283
:10D3F00070470A43A0F84820704783899BB212B156
:10D4000019438181704723EA0101FAE7FFF7F5BF6D
:10D41000038923F007031B041B0C03817047038956
:10D4200023F070031B041B0C1943018103899BB279
:10D4300043F007030381704738B50D46602D114650
:10D4400004464FF001020ED1FFF7EDFD218921F0D6
:10D4500070010904090C2943218123899BB243F0FF
:10D460000703238138BDFFF7C3FDEFE710B504893B
:10D4700042EA0323E4B219430C43A4B2048110BD71
:10D4800010B5FFF7F3FF038923F077031B041B0C90
:10D4900043F07703038110BD10B5FFF7E7FF038961
:10D4A0009BB243F48043038110BD018582827047A3
:10D4B000038823F070039B059B0D1943018070477F
:10D4C000038923F070031B041B0C1943018170476F
:10D4D00070B50689048B058C24F4407424F0030491
:10D4E00025F0220526F0070624042D043604240C1A
:10D4F0002D0C42EA0313360C44F480741D4331436F
:10D5000044F00104ADB201810483058470BD038B36
:10D5100023F070031B041B0C194301837047038B1A
:10D5200023F4E0431B041B0C43EA012189B201836D
:10D530007047838B23F070031B041B0C19438183FA
:10D540007047838B23F4E0431B041B0C43EA012147
:10D5500089B281837047038821B19BB243F0800375
:10D560000380704723F080039B059B0DF8E78388B9
:10D5700021B19BB243F004038380704723F004037E
:10D580001B041B0CF8E7838821B19BB243F008030E
:10D590008380704723F008031B041B0CF8E7838883
:10D5A00021B19BB243F001038380704723F0010354
:10D5B0001B041B0CF8E7038B23F008031B041B0C54
:10D5C000194301837047038B23F400631B041B0C76
:10D5D00043EA012189B201837047838B23F008035A
:10D5E0001B041B0C194381837047838B23F4006356
:10D5F0001B041B0C43EA012189B281837047038B12
:10D6000023F004031B041B0C194301837047038B95
:10D6100023F480631B041B0C43EA012189B20183BC
:10D620007047838B23F004031B041B0C1943818375
:10D630007047838B23F480631B041B0C43EA012196
:10D6400089B281837047038B23F080031B041B0C7A
:10D65000194301837047038BC3F30E0343EA01218F
:10D6600089B201837047838B23F080031B041B0C5A
:10D67000194381837047838BC3F30E0343EA01216F
:10D6800089B281837047038C23F002031B041B0CB7
:10D69000194301847047038C23F008031B041B0CFF
:10D6A000194301847047038C23F020031B041B0CD7
:10D6B00043EA011189B201847047038C23F080038F
:10D6C0001B041B0C43EA011189B201847047038CCF
:10D6D00023F400731B041B0C43EA012189B201846B
:10D6E0007047038C23F400631B041B0C43EA0121E5
:10D6F00089B201847047038C23F400531B041B0C74
:10D7000043EA013189B20184704710B50124038CCA
:10D710008C409BB223EA04030384038C02FA01F1D8
:10D72000194389B2018410BD10B50424038C8C40C8
:10D730009BB223EA04030384038C02FA01F1194328
:10D7400089B2018410BD10B50124038C8C409BB2BA
:10D7500023EA0403038421F00803183053B949086D
:10D76000435823F070031B041B0C435043581A43C7
:10D77000425010BD0439C1F34E014358120223F444
:10D78000E0431B041B0C4350435892B2EFE703885D
:10D7900021B19BB243F002030380704723F00203E0
:10D7A0009B059B0DF8E7038821B19BB243F004036E
:10D7B0000380704723F004039B059B0DF8E78388E3
:10D7C00021B19BB243F080038380704723F0800334
:10D7D0001B041B0CF8E7038823F008039B059B0D33
:10D7E000038003889BB2194301807047838823F02C
:10D7F00070031B041B0C838083889BB219438180B8
:10D800007047038923F007031B041B0C0381038962
:10D810009BB2194301817047038923F080031B04E5
:10D820001B0C038103899BB21943018170478184DA
:10D83000704781857047818670470187704781876F
:10D840007047A0F840107047038B23F00C031B04B3
:10D850001B0C0383038B9BB2194301837047038B1B
:10D8600023F440631B041B0C0383038B9BB243EA2A
:10D87000012189B201837047F8B50C464988A28816
:10D880000029B4F800E00CBF02260026012A0CBFD4
:10D89000022701272389BEF1000F0ED1FFF7A8FB55
:10D8A000E188FFF7D1FF314623893A46FFF7BBFBFA
:10D8B000E188BDE8F840FFF7D2BFFFF7B4FBE1888D
:10D8C000FFF7CDFF314623893A46FFF791FBE18808
:10D8D000BDE8F840FFF7B8BF838B23F00C031B04AF
:10D8E0001B0C8383838B9BB2194381837047838B8B
:10D8F00023F440631B041B0C8383838B9BB243EA9A
:10D90000012189B281837047F8B50E880D460B89D5
:10D910008A88498836B9FFF76BFBE988BDE8F8408B
:10D92000FFF792BF042E06D1FFF77DFBE988BDE823
:10D93000F840FFF794BF082EEE88058C1CD125F423
:10D9400080752D042D0C0584878B058CBFB227F0C4
:10D95000F307ADB23A4342EA031225F4007343F4ED
:10D96000807343EA01239BB292B2828331460384DF
:10D97000BDE8F840FFF7B0BF25F480552D042D0C0D
:10D980000584878B058C1B03ADB227F4407743EAEF
:10D9900002223F0525F400533F0D43F480533A43E0
:10D9A00043EA01339BB292B2828331460384BDE8DD
:10D9B000F840FFF79CBF0388DBB2038003889BB26B
:10D9C000194301807047808E80B27047008F80B20B
:10D9D0007047808F80B27047B0F8400080B27047C7
:10D9E000808C80B27047008D80B27047038A1942E4
:10D9F00014BF012000207047C94389B201827047DB
:10DA0000038A828911EA030092B203D0114214BF43
:10DA1000012000207047C94389B20182704700BFCE
:10DA200008B5244B984231D008D8A3F5006398423A
:10DA300017D003F5806398421FD008BD1E4B984253
:10DA40002DD003F56843984232D101214FF4804034
:10DA5000FFF79EF8BDE8084000214FF48040FFF733
:10DA600097B801214FF40030FFF79EF800214FF4E2
:10DA70000030BDE80840FFF797B801214FF480203F
:10DA8000FFF792F800214FF48020F2E701214FF4D4
:10DA90000020FFF789F800214FF40020E9E7012179
:10DAA0004FF48010FFF780F800214FF48010E0E77A
:10DAB00008BD00BF004C00400050004030B5044697
:10DAC000038ACA889BB223F4405313430382838999
:10DAD0008A8823F4B05323F00C031B041B0C13435C
:10DAE0000A8987B013434A890D4613439BB2838149
:10DAF000838A8A899BB223F440731343838201A8EB
:10DB0000FEF7E0FF039B049A0D498C4218BF1A46AA
:10DB1000192353432A689200B3FBF2F36422B3FB48
:10DB2000F2F102FB11331B013233B3FBF2F303F0CA
:10DB30000F0343EA01139BB2238107B030BD00BF3E
:10DB4000003801404FF416530C2203600023428139
:10DB50008380C3800381838170470B8810B54C8814
:10DB6000028A23438C88C98892B223430B4322F450
:10DB7000706213439BB2038210BD00230380438075
:10DB80008380C3807047838921B19BB243F40053E3
:10DB90008381704723F400531B041B0CF8E701F04A
:10DBA0001F0310B5C1F342140121012C01FA03F146
:10DBB00005D10C3003683AB11943016010BD022C45
:10DBC0000CBF10301430F5E723EA0101F5E7838A32
:10DBD0009BB212B119438182704723EA0101FAE72F
:10DBE000038A23F00F031B041B0C0382038A9BB2DE
:10DBF000194301827047838923F400631B041B0CC3
:10DC0000838183899BB2194381817047838921B1C4
:10DC10009BB243F002038381704723F002031B048D
:10DC20001B0CF8E7038A23F020031B041B0C038260
:10DC3000038A9BB2194301827047038A21B19BB2C8
:10DC400043F480430382704723F480431B041B0C7E
:10DC5000F8E7C1F30801818070478088C0F30800AD
:10DC6000704783899BB243F0010383817047038B24
:10DC7000DBB20383038B9BB243EA0121018370472C
:10DC8000038B03F47F430383038B9BB2194301830C
:10DC90007047838A21B19BB243F02003838270478F
:10DCA00023F020031B041B0CF8E7838A21B19BB2ED
:10DCB00043F010038382704723F010031B041B0CF6
:10DCC000F8E7838A21B19BB243F00803838270474F
:10DCD00023F008031B041B0CF8E7838A23F00403DA
:10DCE0001B041B0C8382838A9BB219438182704779
:10DCF000838A21B19BB243F002038382704723F0F1
:10DD000002031B041B0CF8E70388194214BF01200F
:10DD100000207047C94389B2018070470123C1F3D5
:10DD2000421210B5012A01F01F0403FA04F30ED1C8
:10DD3000828992B21340028892B26BB10123090A20
:10DD400003FA01F10A4214BF1846002010BD022A4E
:10DD50000CBF028A828AECE7184610BD0B0A01212B
:10DD60009940C94389B20180704700BF684620F0DE
:10DD700007018D4601B50C4A0C4B0D498B420AD365
:10DD800000210C4B0C4A93420AD302F0ADF9BDE8D6
:10DD900001408546704752F8040F43F8040BEDE745
:10DDA00043F8041BEFE700BF540C010800000020FB
:10DDB00064050020680500201811002010B5064CED
:10DDC00018B9012223681A8210BD044B1B681B6816
:10DDD000984720680A3010BDC41000208010002031
:10DDE00010B5064C18B9012223681A8210BD044BE5
:10DDF0001B689B68984720680C3010BDC410002039
:10DE00008010002010B5204B18B902221B681A821E
:10DE100010BD00201D491C68088023780A4613F0B5
:10DE20007F0313D1637A990644BF0221117013F066
:10DE3000400F137814BF23F0010343F00103137064
:10DE4000134B1B681B699847104810BD012B18D055
:10DE5000022B17D1617901F00F039B0003F180437E
:10DE600003F5B84311F0800F1B6805D003F03003B1
:10DE7000102BE5D10123E2E703F44053B3F5805FB3
:10DE8000F7E7084610BD00BFC410002010110020A5
:10DE9000801000202DE9F843234FDFF8A0803D6873
:10DEA0002C8AD4B92E7A042E17D120490B78012B55
:10DEB0000ED11F4B1A681F4B92B213445B001C60BB
:10DEC00030230C70A8F800303B681E72BDE8F88360
:10DED00010230726A8F80030F6E7AB8A9C4294BFCF
:10DEE000042602269C4228BF1C46AB692046984760
:10DEF0008146002000F0A6FE22460146484600F07A
:10DF00006BFC2146002000F00DFE2B8A4FF440529E
:10DF10001B1B2B826B8A1C443023A8F80030064B55
:10DF20006C821A80D0E700BFC4100020F0090020E6
:10DF3000505C00400230002012110020141100201B
:10DF400010B50A4B0A491B684978DA7891420AD31E
:10DF5000997841B99C8834B99A72064B1B685B6802
:10DF60009847204610BD022010BD00BFC4100020FD
:10DF7000D80000208010002038B50F4A0F4D1268DD
:10DF80002B689269D978587990472B6804469A7A19
:10DF90007AB170B91A7962B99B7853B9084B1B688A
:10DFA000DB6898472B685A79DA72DA781A73204658
:10DFB00038BD0224FBE700BF5C100020C410002025
:10DFC0008010002038B52D4B1B68187810F07F00AA
:10DFD00004D15A7A22F020025A7238BD02284BD15D
:10DFE0005A88002A49D11A79002A46D15979244DF4
:10DFF00021F08000840004F1804202F5B8421268EA
:10E0000049B22D780029B4BF02F0300202F4405228
:10E01000A84231D282B39B7A73B304F1804404F5F1
:10E02000B8440029236811DA03F03003102B07D11C
:10E03000C4B2204600F04BFD3021204600F04EFCDB
:10E04000104B1B685B699847002038BD03F44053B0
:10E05000B3F5805FF4D10C4D58B90C4B93F82C10EC
:10E0600000F081FD23682B409BB283F44053236072
:10E07000E6E700F019FDF5E7022038BDC4100020E6
:10E08000D8000020801000208FBFFFFF500000202C
:10E0900038B51D4B1D4D18682D78417921F080044D
:10E0A000A30003F1804202F5B842126849B2002988
:10E0B000B4BF02F0300202F44052AC4221D2448894
:10E0C000FCB9F2B1827AE2B103F1804303F5B843BF
:10E0D0001A680029B5BF22F4E04222F4804222F0FF
:10E0E000400222F07002B5BF92B292B282F01002EA
:10E0F00082F480521A60064B1B689B699847002087
:10E1000038BD022038BD00BFC4100020D800002058
:10E110008010002008B5064B1A68537A43F020039C
:10E120005372044B1B68DB699847002008BD00BF91
:10E13000C410002080100020054B10B51C68628AB6
:10E1400018B98B889B1A238210BD0868104410BD33
:10E15000C410002008B50B4B002093F82C1000F0E1
:10E1600002FD094B1B68187A082806D14FF480522B
:10E17000064B1A801022064B1A80A0F10903584260
:10E18000584108BD50000020C4100020121100208A
:10E1900014110020F7B5984C984E276832683B7AE6
:10E1A000092B19D0964B92B213445B001D886D0069
:10E1B00005F1804505F5C0452B783B706B787B7089
:10E1C000A88800F06DFE78802889276800F068FE36
:10E1D000B880AA892368DA80012223681A72DA8853
:10E1E0005D78002A63D11A7812F07F024CD1092D94
:10E1F00003D1FFF7A5FEB0B126E0052D1FD193F99D
:10E200000320002A06DA082322681372FFF7A2FF10
:10E2100003B0F0BD9A78002AF5D19A88002AF2D18D
:10E220009B7A002BEFD13268764B92B213440022D6
:10E230005B001A603022744B1A800623E4E7032D3A
:10E2400014D1DA78012A08D0704B28461B685B6924
:10E250009847032828D10923D6E79A88002AF3D1C2
:10E260005B7A9806F0D5FFF755FFC4E7012DEBD197
:10E27000DA78012AE8D19A88002AE5D15B7A9906F2
:10E28000E2D5FFF79FFEB6E7012A04D10B2DDBD1C3
:10E29000FFF772FEAFE7022AD6D1012DF1D0032D90
:10E2A000D2D1FFF7F5FEA6E70028ACD1BBE7062DDB
:10E2B00014D11A7852065DD19A78544B012A03D1B1
:10E2C0001B68DB69EBB955E0022A02D11B681B6AA7
:10E2D000F8E7032A4ED11B685B6AF3E7002D55D19E
:10E2E0005988002946D15A6822F47F42B2F5003F8E
:10E2F00040D11A7812F07F0216D19B88002B39D1B9
:10E30000434B00252268284655829361984728464A
:10E310004FF6FF7123681A8A8A4234D0022801D04E
:10E32000002A56D108222FE0012A0AD1374A58790B
:10E33000126892699047E8B923689B7A002BDFD175
:10E3400018E0022A16D15A79324802F00F018B00E8
:10E3500003F1804303F5B8431B68007812F0800F87
:10E3600014BF03F0300303F44053814202D212F091
:10E37000700FE3D0254B22681B6850781B699847C3
:10E380000328C5D1236809221A723FE7082D04D15A
:10E390001B785B06EED1204BB3E70A2DEAD11A7841
:10E3A00002F07F02012AE5D19A7A002AE2D0598848
:10E3B0000029DFD15A6822F47F42B2F5803FD9D1DB
:10E3C000124A58791268926990470028D2D1134BAB
:10E3D00097E793F90010002935DAD9880B4C0191A1
:10E3E000019882421CD9019A1A82226892F82C2044
:10E3F0009A82FFF74FFD09E7C4100020505C0040EF
:10E400000430002002300020141100205C10002095
:10E4100005DE0008D8000020BDDD0008E1DD0008B1
:10E420008A42E2D2216891F82C00824203D2002174
:10E43000084A1170D9E792FBF0F100FB1122002A83
:10E44000D3D10121F4E703221A724FF44052024B58
:10E450001A80DBE6F009002012110020F8B52A4DE1
:10E460002C68237A032B01D0052B44D1A369268A7B
:10E47000ABB1A6B1A28A964228BF1646304698474D
:10E48000238A07469B1B2382638A002033446382CE
:10E4900000F0E8FB32460146384600F0AFF9238A27
:10E4A00053B100214FF44052184B08461A8000F037
:10E4B00039FB3022164B1A80A38A228A93422B689A
:10E4C00009D803221A722B681B7A2A681372BDE8D6
:10E4D000F840FFF73FBE0AB10522F3E706211972A3
:10E4E0000C4B19680C4B89B20B445B001A6030224C
:10E4F000074B1A80E7E7072B03D1084B1B68DB6843
:10E5000098470823E1E700BFC41000201211002043
:10E5100014110020505C0040023000205C100020EC
:10E5200030B5002248F68F75094B1C78A24204D3FF
:10E53000084B40F08000186030BD02F1805303F5B5
:10E54000B8539B0019682940114319600132EDE767
:10E55000D80000204C5C004010B5134C23681A7A98
:10E56000022A01D0042A09D1FFF794FC23681B7A00
:10E5700022681372BDE81040FFF7ECBD062A10D1E7
:10E580005A78052A09D11A78520606D1D878FFF7A9
:10E59000C7FF064B1B681B6A9847054B1B689B68A7
:10E5A00098470823E4E700BFC41000208010002033
:10E5B0005C100020704700BF064B074A07491360F4
:10E5C00002221A72064B074A1360074A1B68116041
:10E5D000184700BF64100020C4100020B4000020C1
:10E5E000500000205C100020801000202DE9F8432E
:10E5F000DFF86481DFF86491D8F800304F4A99B2AF
:10E600001B04118001D4BDE8F88347F6FF73C8F8F6
:10E610000030138803F00F0389F80030002B62D11B
:10E62000474C484E2368484D03F4405333802368D9
:10E63000464F03F030032B8023683B409BB283F4AA
:10E6400000532360236823F4E04323F040039BB28C
:10E6500083F020032360138813F0100F236828D160
:10E6600023F4E14323F070031B041B0C2360FFF72A
:10E6700073FF236832883B409BB2D70448BF83F4C2
:10E68000805396042E4A48BF83F4005313601368E6
:10E69000298823F4E04323F040039BB2CC0648BF13
:10E6A00083F01003880648BF83F020031360BDE8A1
:10E6B000F883190601D52368D2E71A0508D523681F
:10E6C00023F070031B051B0D2360FFF763FDD0E7EC
:10E6D0001B0491D5236823F070031B051B0D2360D9
:10E6E000FFF7BCFEC5E79A0002F1804202F5B8428E
:10E6F000146821040AD51168013B21F07001090555
:10E70000090D1160124A52F82330984722067FF50E
:10E7100073AF99F80020930003F1804303F5B843E9
:10E720001968013A21F4E14121F070010904090C52
:10E730001960084B53F8223098475DE75A100020C3
:10E74000005C004012110020141100208FBFFFFF59
:10E75000DC000020F8000020445C00406010002035
:10E7600070B5184D184C194E2B689AB21B042280B4
:10E7700000D470BD47F6FF732B60238803F00F03AE
:10E780009A0002F18042337002F5B8421168080421
:10E790000BD51168013B21F070010905090D1160CD
:10E7A0000B4A52F823309847DEE70906DCD511689A
:10E7B000013B21F4E14121F070010904090C1160D1
:10E7C000044AEEE7445C00405A100020601000202C
:10E7D000DC000020F8000020002310B501F10051FA
:10E7E000013201F54051521049009A4200D110BD4A
:10E7F00030F8024B21F823400133F6E7002310B52F
:10E8000001F10051013201F54051521049009A4284
:10E8100000D110BD51F8234020F813400133F6E732
:10E82000014B1860704700BF405C0040014B186806
:10E8300080B27047405C0040014B1860704700BFD9
:10E84000445C0040014B186880B27047445C004053
:10E85000014B186880B27047485C0040014B18605B
:10E86000704700BF4C5C0040014B186880B2704795
:10E870004C5C00404FF6F873014A03401360704748
:10E88000505C0040014B186880B27047505C0040FB
:10E89000800000F1804000F5B840016070478000C2
:10E8A00000F1804000F5B840006880B270478000F9
:10E8B00000F1804000F5B840036823F4EC4323F0F6
:10E8C0007003194389B201607047800000F18040F5
:10E8D00000F5B840006800F4C0607047800000F1A7
:10E8E000804000F5B8400368CA0623F4E04323F0F3
:10E8F00040039BB248BF83F010038A0648BF83F0F1
:10E90000200303607047800000F1804000F5B840AC
:10E910000368CA0423F4804323F070039BB248BF0A
:10E9200083F480538A0448BF83F400530360704724
:10E93000800000F1804000F5B8400129036805D14E
:10E9400023F480531B041B0C036070470229FCD185
:10E9500023F01003F6E7800000F1804000F5B84096
:10E96000006800F030007047800000F1804000F542
:10E97000B840006800F440507047800000F18040CB
:10E9800000F5B840036823F4E04323F040039BB252
:10E9900083F0300303607047800000F1804000F591
:10E9A000B840036823F4804323F070039BB283F4E0
:10E9B000405303607047800000F1804000F5B8408C
:10E9C000036823F4E04323F0700343F480739BB2A5
:10E9D00003607047FFF7EFBFFFF7EDBF800000F166
:10E9E000804000F5B840036823F4E24323F070034D
:10E9F0001B041B0C03607047FFF7F0BFFFF7EEBF6F
:10EA0000800000F1804000F5B840006800F0300060
:10EA1000A0F11003584258417047800000F1804037
:10EA200000F5B840006800F44050A0F5805358420B
:10EA300058417047800000F1804000F5B8400368FD
:10EA400023F070031B051B0D03607047800000F16D
:10EA5000804000F5B840036823F4E14323F07003DD
:10EA60001B041B0C03607047800000F1804000F520
:10EA7000B840036823F4E04323F070031B041B0C2D
:10EA800043F4804303607047800000F1804000F54C
:10EA9000B840036823F4E04323F070031B041B0C0D
:10EAA00043F0400303607047800000F1804000F5B0
:10EAB000B84003685B0409D5036823F4E04323F0FE
:10EAC00070031B041B0C43F48043036070478000F9
:10EAD00000F1804000F5B84003685B0609D5036883
:10EAE00023F4E04323F070031B041B0C43F04003AA
:10EAF00003607047800000F1804000F5B840036873
:10EB000023F4E04323F070031B041B0C1943016042
:10EB10007047800000F1804000F5B840006800F0C8
:10EB20000F007047044B1B689BB203EBC000034B04
:10EB300003445B0019607047505C004002300020C5
:10EB40003E290AD94B09C90604BF03F1FF339BB222
:10EB50009B0243F40043036070474B08CA0748BF59
:10EB600001339B02F7E70E4B0E4A1B683E299BB20E
:10EB700003EBC00002444FEA42020AD94B09C8061F
:10EB800004BF03F1FF339BB29B0243F400431360C5
:10EB900070474B08C90748BF01339B02F7E700BF26
:10EBA000505C00400630002010B50B4CC0002368BC
:10EBB00049089BB2034403F1005303F540535B0043
:10EBC00049001960236852089BB21844034B520055
:10EBD00003445B001A6010BD505C0040043000200C
:10EBE000064B49081B6849009BB203EBC00000F1CB
:10EBF000005000F54050400001607047505C0040FC
:10EC0000FFF7EEBF054B49081B6849009BB203EBB9
:10EC1000C000034B03445B0019607047505C004028
:10EC200004300020FFF7EEBF054B1B689BB203EBDF
:10EC3000C00000F1005000F54050400000887047CF
:10EC4000505C0040FFF7F0BF044B1B689BB203EB26
:10EC5000C000034B03445B0018887047505C0040C1
:10EC600004300020FFF7F0BF012910B52BD1254C4F
:10EC7000C0002168244B89B201440B443E2A4FEA6C
:10EC8000430119D9530912F01F0F04BF03F1FF33D9
:10EC90009BB29B0243F400430B6023681B499BB269
:10ECA000184401443E2A4FEA41011FD85308D207B5
:10ECB00048BF01339B0222E0530812F0010F18BF36
:10ECC00001339B02E8E702291BD10E4CC0002168EA
:10ECD0000D4B89B201440B445B001A6023689BB260
:10ECE00018440A4B03445B001A6010BD5309D00658
:10ECF00004BF03F1FF339BB29B0243F400430B605C
:10ED000010BD10BD505C00400230002006300020D5
:10ED100001291BD1134B14491B683E2A9BB203EBFC
:10ED2000C00001444FEA41010AD95309D00604BF8B
:10ED300003F1FF339BB29B0243F400430B60704727
:10ED40005308D20748BF01339B02F7E7022908D1D5
:10ED5000044B1B689BB203EBC000034B03445B00F6
:10ED60001A607047505C00400230002001291BD11E
:10ED7000134B14491B683E2A9BB203EBC0000144AD
:10ED80004FEA41010AD95309D00604BF03F1FF330A
:10ED90009BB29B0243F400430B6070475308D207B9
:10EDA00048BF01339B02F7E7022908D1044B1B68D7
:10EDB0009BB203EBC000034B03445B001A60704737
:10EDC000505C004006300020054B1B689BB203EBF3
:10EDD000C000044B03445B001868C0F3090070478F
:10EDE000505C004002300020FFF7EEBF054B1B686F
:10EDF0009BB203EBC000044B03445B001868C0F3F4
:10EE000009007047505C004006300020FFF7EEBF5D
:10EE10000D49C0000B689BB2C2180C4B13445B0039
:10EE20001B6813F47C4F0DD10B689BB21844084B40
:10EE300003445B001B68C3F30903002B14BF0220CB
:10EE40000020704701207047505C004006300020D1
:10EE50000230002001290FD1800000F1804000F530
:10EE6000B840036823F4E04323F070031B041B0C39
:10EE700043F04003036070470229FCD1800000F199
:10EE8000804000F5B840036823F4E04323F07003AA
:10EE90001B041B0C43F48043ECE741EA002070475D
:10EEA000C3B2000A40EA0320704700BF81F000416E
:10EEB00002E000BF83F0004330B54FEA41044FEA5F
:10EEC000430594EA050F08BF90EA020F1FBF54EAFA
:10EED000000C55EA020C7FEA645C7FEA655C00F096
:10EEE000E2804FEA5454D4EB5555B8BF6D420CDD67
:10EEF0002C4480EA020281EA030382EA000083EAEA
:10EF0000010180EA020281EA0303362D88BF30BD89
:10EF100011F0004F4FEA01314FF4801C4CEA1131DF
:10EF200002D0404261EB410113F0004F4FEA03333E
:10EF30004CEA133302D0524263EB430394EA050FC9
:10EF400000F0A780A4F10104D5F1200E0DDB02FA38
:10EF50000EFC22FA05F2801841F1000103FA0EF2CC
:10EF6000801843FA05F359410EE0A5F120050EF192
:10EF7000200E012A03FA0EFC28BF4CF0020C43FAC3
:10EF800005F3C01851EBE37101F0004507D54FF0D0
:10EF9000000EDCF1000C7EEB00006EEB0101B1F520
:10EFA000801F1BD3B1F5001F0CD349085FEA300066
:10EFB0004FEA3C0C04F101044FEA445212F5800F71
:10EFC00080F09A80BCF1004F08BF5FEA500C50F10E
:10EFD000000041EB045141EA050130BD5FEA4C0CF1
:10EFE000404141EB010111F4801FA4F10104E9D17A
:10EFF00091F0000F04BF01460020B1FA81F308BF71
:10F000002033A3F10B03B3F120020CDA0C3208DD3C
:10F0100002F1140CC2F10C0201FA0CF021FA02F117
:10F020000CE002F11402D8BFC2F1200C01FA02F187
:10F0300020FA0CFCDCBF41EA0C019040E41AA2BFAC
:10F0400001EB0451294330BD6FEA04041F3C1CDA74
:10F050000C340EDC04F11404C4F1200220FA04F094
:10F0600001FA02F340EA030021FA04F345EA03013E
:10F0700030BDC4F10C04C4F1200220FA02F001FA00
:10F0800004F340EA0300294630BD21FA04F0294682
:10F0900030BD94F0000F83F4801306BF81F480111B
:10F0A0000134013D4EE77FEA645C18BF7FEA655C8E
:10F0B00029D094EA050F08BF90EA020F05D054EA60
:10F0C000000C04BF1946104630BD91EA030F1EBF65
:10F0D0000021002030BD5FEA545C05D14000494169
:10F0E00028BF41F0004130BD14F580043CBF01F55C
:10F0F000801130BD01F0004545F0FE4141F4700142
:10F100004FF0000030BD7FEA645C1ABF194610461C
:10F110007FEA655C1CBF0B46024650EA013406BF1D
:10F1200052EA033591EA030F41F4002130BD00BFDC
:10F1300090F0000F04BF0021704730B54FF4806499
:10F1400004F132044FF000054FF0000150E700BF1A
:10F1500090F0000F04BF0021704730B54FF4806479
:10F1600004F1320410F0004548BF40424FF0000166
:10F170003EE700BF42004FEAE2014FEA31014FEAA9
:10F1800002701FBF12F07F4393F07F4F81F06051F8
:10F19000704792F0000F14BF93F07F4F704730B567
:10F1A0004FF4607401F0004521F0004120E700BFFA
:10F1B00050EA010208BF704730B54FF000050AE081
:10F1C00050EA010208BF704730B511F0004502D582
:10F1D000404261EB41014FF4806404F132045FEA84
:10F1E000915C3FF4DCAE4FF003025FEADC0C18BF29
:10F1F00003325FEADC0C18BF033202EBDC02C2F11F
:10F20000200300FA03FC20FA02F001FA03FE40EAB0
:10F210000E0021FA02F11444C1E600BF70B54FF0B0
:10F22000FF0C4CF4E06C1CEA11541DBF1CEA135592
:10F2300094EA0C0F95EA0C0F00F0DEF82C4481EAFA
:10F24000030621EA4C5123EA4C5350EA013518BF1A
:10F2500052EA033541F4801143F4801338D0A0FB07
:10F2600002CE4FF00005E1FB02E506F00042E0FBB4
:10F2700003E54FF00006E1FB03569CF0000F18BFBA
:10F280004EF0010EA4F1FF04B6F5007F64F5407462
:10F2900004D25FEA4E0E6D4146EB060642EAC621F5
:10F2A00041EA55514FEAC52040EA5E504FEACE2E62
:10F2B000B4F1FD0C88BFBCF5E06F1ED8BEF1004F65
:10F2C00008BF5FEA500E50F1000041EB045170BDE1
:10F2D00006F0004646EA010140EA020081EA030125
:10F2E000B4EB5C04C2BFD4EB0C0541EA045170BD21
:10F2F00041F480114FF0000E013C00F3AB8014F19B
:10F30000360FDEBF002001F0004170BDC4F10004E3
:10F31000203C35DA0C341BDC04F11404C4F1200564
:10F3200000FA05F320FA04F001FA05F240EA0200BF
:10F3300001F0004221F0004110EBD37021FA04F6F5
:10F3400042EB06015EEA430E08BF20EAD37070BDAF
:10F35000C4F10C04C4F1200500FA04F320FA05F00E
:10F3600001FA04F240EA020001F0004110EBD37010
:10F3700041F100015EEA430E08BF20EAD37070BD80
:10F38000C4F1200500FA05F24EEA020E20FA04F359
:10F3900001FA05F243EA020321FA04F001F0004108
:10F3A00021FA04F220EA020000EBD3705EEA430E79
:10F3B00008BF20EAD37070BD94F0000F0FD101F0A8
:10F3C0000046400041EB010111F4801F08BF013CE1
:10F3D000F7D041EA060195F0000F18BF704703F01F
:10F3E0000046520043EB030313F4801F08BF013DA6
:10F3F000F7D043EA0603704794EA0C0F0CEA135562
:10F4000018BF95EA0C0F0CD050EA410618BF52EA1B
:10F410004306D1D181EA030101F000414FF0000021
:10F4200070BD50EA410606BF1046194652EA43062F
:10F4300019D094EA0C0F02D150EA013613D195EAA3
:10F440000C0F05D152EA03361CBF104619460AD1EB
:10F4500081EA030101F0004141F0FE4141F47001F5
:10F460004FF0000070BD41F0FE4141F4780170BDE5
:10F4700070B54FF0FF0C4CF4E06C1CEA11541DBF4A
:10F480001CEA135594EA0C0F95EA0C0F00F0A7F84C
:10F49000A4EB050481EA030E52EA03354FEA013179
:10F4A00000F088804FEA03334FF0805545EA13138C
:10F4B00043EA12634FEA022245EA111545EA106554
:10F4C0004FEA00260EF000419D4208BF964244F1EB
:10F4D000FD0404F5407402D25B084FEA3202B61A0A
:10F4E00065EB03055B084FEA32024FF480104FF4DE
:10F4F000002CB6EB020E75EB030E22BFB61A754652
:10F5000040EA0C005B084FEA3202B6EB020E75EBE4
:10F51000030E22BFB61A754640EA5C005B084FEA4C
:10F520003202B6EB020E75EB030E22BFB61A754619
:10F5300040EA9C005B084FEA3202B6EB020E75EB24
:10F54000030E22BFB61A754640EADC0055EA060EE5
:10F5500018D04FEA051545EA16754FEA06164FEA28
:10F56000C30343EA52734FEAC2025FEA1C1CC0D1D4
:10F5700011F4801F0BD141EA00014FF000004FF061
:10F58000004CB6E711F4801F04BF01430020B4F122
:10F59000FD0C88BFBCF5E06F3FF6AFAEB5EB030CDA
:10F5A00004BFB6EB020C5FEA500C50F1000041EBD7
:10F5B000045170BD0EF0004E4EEA113114EB5C04A4
:10F5C000C2BFD4EB0C0541EA045170BD41F4801177
:10F5D0004FF0000E013C90E645EA060E8DE60CEA7F
:10F5E000135594EA0C0F08BF95EA0C0F3FF43BAF9C
:10F5F00094EA0C0F0AD150EA01347FF434AF95EA53
:10F600000C0F7FF425AF104619462CE795EA0C0F36
:10F6100006D152EA03353FF4FDAE1046194622E703
:10F6200050EA410618BF52EA43067FF4C5AE50EADD
:10F6300041047FF40DAF52EA43057FF4EBAE12E7CD
:10F640004FF0FF3C06E000BF4FF0010C02E000BFAE
:10F650004FF0010C4DF804CD4FEA410C7FEA6C5C91
:10F660004FEA430C18BF7FEA6C5C1BD001B050EA34
:10F67000410C0CBF52EA430C91EA030F02BF90EA1F
:10F68000020F0020704710F1000F91EA030F58BFDE
:10F69000994208BF90422CBFD8176FEAE37040F040
:10F6A000010070474FEA410C7FEA6C5C02D150EADE
:10F6B000013C07D14FEA430C7FEA6C5CD6D152EA99
:10F6C000033CD3D05DF8040B704700BF844610465E
:10F6D00062468C461946634600E000BF01B5FFF75D
:10F6E000B7FF002848BF10F1000F01BD4DF808ED2D
:10F6F000FFF7F4FF0CBF012000205DF808FB00BFFE
:10F700004DF808EDFFF7EAFF34BF012000205DF857
:10F7100008FB00BF4DF808EDFFF7E0FF94BF0120A4
:10F7200000205DF808FB00BF4DF808EDFFF7CEFFA5
:10F7300094BF012000205DF808FB00BF4DF808EDE4
:10F74000FFF7C4FF34BF012000205DF808FB00BFB5
:10F750004FEA410C7FEA6C5C02D150EA013C0AD1CD
:10F760004FEA430C7FEA6C5C02D152EA033C02D1BF
:10F770004FF0000070474FF0010070474FEA410220
:10F7800012F5001215D211D56FF47873B3EB6252F3
:10F7900012D94FEAC12343F0004343EA505311F01A
:10F7A000004F23FA02F018BF404270474FF00000AC
:10F7B000704750EA013005D111F0004008BF6FF0EA
:10F7C000004070474FF00000704700BF4FEA410211
:10F7D000B2F1E04324BFB3F5001CDCF1FE5C0DD9AF
:10F7E00001F0004C4FEAC0024CEA5070B2F1004FF9
:10F7F00040EB830008BF20F00100704711F0804FFC
:10F8000021D113F13872BCBF01F00040704741F4C0
:10F8100080114FEA5252C2F11802C2F1200C10FAC4
:10F820000CF320FA02F018BF40F001004FEAC123A8
:10F830004FEAD32303FA0CFC40EA0C0023FA02F34C
:10F840004FEA4303CCE77FEA625307D150EA013322
:10F850001EBF4FF0FE4040F44000704701F00040F2
:10F8600040F0FE4040F40000704700BF80F00040D0
:10F8700002E000BF81F0004142001FBF5FEA410388
:10F8800092EA030F7FEA226C7FEA236C6AD04FEA88
:10F890001262D2EB1363C1BFD218414048404140CD
:10F8A000B8BF5B42192B88BF704710F0004F40F47F
:10F8B000000020F07F4018BF404211F0004F41F49B
:10F8C000000121F07F4118BF494292EA030F3FD067
:10F8D000A2F1010241FA03FC10EB0C00C3F120037A
:10F8E00001FA03F100F0004302D5494260EB400009
:10F8F000B0F5000F13D3B0F1807F06D340084FEA74
:10F90000310102F10102FE2A51D2B1F1004F40EB68
:10F91000C25008BF20F0010040EA030070474900D0
:10F9200040EB000010F4000FA2F10102EDD1B0FA9B
:10F9300080FCACF1080CB2EB0C0200FA0CF0AABF90
:10F9400000EBC25052421843BCBFD040184370472E
:10F9500092F0000F81F4000106BF80F40000013234
:10F96000013BB5E74FEA41037FEA226C18BF7FEA0B
:10F97000236C21D092EA030F04D092F0000F08BF4D
:10F980000846704790EA010F1CBF0020704712F034
:10F990007F4F04D1400028BF40F00040704712F173
:10F9A00000723CBF00F50000704700F0004343F0D8
:10F9B000FE4040F4000070477FEA226216BF08460E
:10F9C0007FEA23630146420206BF5FEA412390EAD1
:10F9D000010F40F4800070474FF0000304E000BFC7
:10F9E00010F0004348BF40425FEA000C08BF704778
:10F9F00043F0964301464FF000001CE050EA01023C
:10FA000008BF70474FF000030AE000BF50EA010250
:10FA100008BF704711F0004302D5404261EB41013D
:10FA20005FEA010C02BF84460146002043F0B64362
:10FA300008BFA3F18053A3F50003BCFA8CF2083A87
:10FA4000A3EBC25310DB01FA02FC634400FA02FC90
:10FA5000C2F12002BCF1004F20FA02F243EB020097
:10FA600008BF20F00100704702F1200201FA02FCF9
:10FA7000C2F1200250EA4C0021FA02F243EB0200EC
:10FA800008BF20EADC7070474FF0FF0C1CEAD05230
:10FA90001EBF1CEAD15392EA0C0F93EA0C0F6FD0F1
:10FAA0001A4480EA010C400218BF5FEA41211ED0CF
:10FAB0004FF0006343EA501043EA5111A0FB0131BB
:10FAC0000CF00040B1F5000F3EBF490041EAD37190
:10FAD0005B0040EA010062F17F02FD2A1DD8B3F10C
:10FAE000004F40EBC25008BF20F00100704790F07B
:10FAF000000F0CF0004C08BF49024CEA502040EACD
:10FB000051207F3AC2BFD2F1FF0340EAC250704792
:10FB100040F400004FF00003013A5DDC12F1190FD0
:10FB2000DCBF00F000407047C2F10002410021FA42
:10FB300002F1C2F1200200FA02FC5FEA310040F15A
:10FB4000000053EA4C0308BF20EADC70704792F0D3
:10FB5000000F00F0004C02BF400010F4000F013A0B
:10FB6000F9D040EA0C0093F0000F01F0004C02BF06
:10FB7000490011F4000F013BF9D041EA0C018FE775
:10FB80000CEAD15392EA0C0F18BF93EA0C0F0AD07B
:10FB900030F0004C18BF31F0004CD8D180EA0100A1
:10FBA00000F00040704790F0000F17BF90F0004F3A
:10FBB000084691F0000F91F0004F14D092EA0C0F1C
:10FBC00001D142020FD193EA0C0F03D14B0218BFAF
:10FBD000084608D180EA010000F0004040F0FE40F5
:10FBE00040F40000704740F0FE4040F44000704791
:10FBF0004FF0FF0C1CEAD0521EBF1CEAD15392EA10
:10FC00000C0F93EA0C0F69D0A2EB030280EA010CFF
:10FC100049024FEA402037D04FF0805343EA111198
:10FC200043EA10130CF000408B4238BF5B0042F1F6
:10FC30007D024FF4000C8B4224BF5B1A40EA0C009B
:10FC4000B3EB510F24BFA3EB510340EA5C00B3EBCD
:10FC5000910F24BFA3EB910340EA9C00B3EBD10FBB
:10FC600024BFA3EBD10340EADC001B0118BF5FEA0D
:10FC70001C1CE0D1FD2A3FF650AF8B4240EBC25036
:10FC800008BF20F0010070470CF0004C4CEA5020F7
:10FC90007F32C2BFD2F1FF0340EAC250704740F446
:10FCA00000004FF00003013A37E792F0000F00F038
:10FCB000004C02BF400010F4000F013AF9D040EAB6
:10FCC0000C0093F0000F01F0004C02BF490011F44A
:10FCD000000F013BF9D041EA0C0195E70CEAD15342
:10FCE00092EA0C0F08D142027FF47DAF93EA0C0F29
:10FCF0007FF470AF084676E793EA0C0F04D14B020D
:10FD00003FF44CAF08466EE730F0004C18BF31F0BE
:10FD1000004CCAD130F000427FF45CAF31F00043B8
:10FD20007FF43CAF5FE700BF42000ED2B2F1FE4F5E
:10FD30000BD34FF09E03B3EB126209D44FEA0023BA
:10FD400043F0004323FA02F070474FF00000704781
:10FD500012F1610F01D1420202D14FF0FF30704722
:10FD60004FF00000704700BF7BB972B90029BEBFD9
:10FD700000204FF0004106E008BF00281CBF6FF0D4
:10FD800000414FF0FF3000F0ADB9ADF1080C6DE966
:10FD900004CE002909DB002B1ADB00F035F8DDF872
:10FDA00004E0DDE9022304B07047404261EB410109
:10FDB000002B1BDB00F028F8DDF804E0DDE902236E
:10FDC00004B0404261EB4101524263EB4303704790
:10FDD000524263EB430300F017F8DDF804E0DDE97D
:10FDE000022304B0404261EB41017047524263EB91
:10FDF000430300F009F8DDF804E0DDE9022304B074
:10FE0000524263EB430370472DE9F0478C460E46A0
:10FE10000446089D002B50D18A4217466CD9B2FA8D
:10FE200082FEBEF1000F0BD0CEF1200C01FA0EF6CF
:10FE300020FA0CFC02FA0EF74CEA060C00FA0EF45B
:10FE40003A0CBCFBF2F9BBB202FB19CC09FB03FA7A
:10FE50004FEA144848EA0C46B2450AD9F61909F1A6
:10FE6000FF3180F02581B24540F22281A9F10209DB
:10FE70003E44A6EB0A06B6FBF2F002FB106600FB5E
:10FE800003F3A4B244EA0644A34209D9E41900F1F9
:10FE9000FF3280F00B81A34240F2088102383C44DB
:10FEA0000021E41A40EA0940002D62D0002324FA20
:10FEB0000EF42C606B60BDE8F0878B4207D9002DF3
:10FEC00055D0002185E841000846BDE8F087B3FA27
:10FED00083F1002940F08F80B34202D3824200F2C6
:10FEE000FC80841A66EB03060120B446002D40D046
:10FEF00085E81010BDE8F08712B90127B7FBF2F7CB
:10FF0000B7FA87FEBEF1000F35D10121F61B4FEA8B
:10FF1000174C1FFA87F8B6FBFCF20CFB126608FBC5
:10FF200002F0230C43EA0646B04207D9F61902F163
:10FF3000FF3302D2B04200F2D2801A46361AB6FB24
:10FF4000FCF00CFB106608FB00F8A3B243EA064481
:10FF5000A04507D9E41900F1FF3302D2A04500F211
:10FF6000B9801846A4EB080440EA02409CE7294601
:10FF70002846BDE8F08707FA0EF7CEF1200326FAEF
:10FF800003F24FEA174CB2FBFCF11FFA87F80CFBA7
:10FF9000112206FA0EF620FA03F301FB08F93343A7
:10FFA0001E0C46EA0246B14500FA0EF409D9F619CC
:10FFB00001F1FF3280F08C80B14540F28980023936
:10FFC0003E44A6EB0906B6FBFCF00CFB106200FBFE
:10FFD00008F99EB246EA0246B14507D9F61900F182
:10FFE000FF3371D2B1456FD902383E44A6EB090602
:10FFF00040EA01418FE7C1F1200722FA07F88B4060
:020000040801F1
:1000000048EA030326FA07F44FEA134EB4FBFEF95D
:100010001FFA83FC0EFB19448E4020FA07F809FBF7
:100020000CFA48EA06084FEA184646EA0444A24594
:1000300002FA01F200FA01F608D9E41809F1FF30DA
:1000400044D2A24542D9A9F102091C44A4EB0A04F6
:10005000B4FBFEF00EFB104400FB0CFC1FFA88F80A
:1000600048EA0444A44507D9E41800F1FF3E29D228
:10007000A44527D902381C4440EA0940A0FB028964
:10008000A4EB0C0CCC45C246CE4615D312D055B1CC
:10009000B6EB0A036CEB0E0606FA07F7CB401F43DC
:1000A000CE402F606E600021BDE8F0871046F7E675
:1000B0008946DEE64645EAD2B8EB020A69EB030E52
:1000C0000138E4E77046D7E718468FE78146BDE779
:1000D000114676E702383C4444E7084606E7023A10
:1000E0003E442BE7704700BF2DE9F34100256A4CE1
:1000F000FCF71EFC4FF480302570FCF737FCFCF752
:1001000085FD0128064626D11020FBF717FF28465B
:10011000FCF77AFC2846FCF78BFC4FF48060FCF778
:100120007DFC4FF440304FF4E011FCF74BFC3046BF
:10013000FCF752FC3920FCF755FD0028FAD00220CC
:10014000FBF7E4FE0220FCF74DFCFCF755FC082809
:10015000FBD10123237001210420FCF701FD4FF4A2
:100160008073ADF8043003238DF80630182301A9FD
:100170004A488DF80730FCF778F90620FCF72CFD8B
:1001800001210846FCF7ECFC01214FF0C050FCF7C0
:10019000F3FC434C4FF480414FF00060FCF712FB3E
:1001A0004FF44070FCF766FA3E4DF4F719F8F4F797
:1001B000B5FCF3F7E5FFF4F73BF9F9F7CDFAF9F7FA
:1001C000ABFAF8F78CFDF4F7A9F82078F8F7F8FD0A
:1001D000E078F8F73BFF2B7823B92269A1686079B2
:1001E000F9F76CF82B780BB1F9F71AFEFAF71FFF45
:1001F000F4F7A6FAF4F7E2FBF7F74EFEF9F774FE10
:10020000294B01275A68294E22F030425A605A6819
:1002100042F080425A60F9F797FA8046F7F760FF9C
:10022000F9F7CCFEF9F761FEF9F78EFAA0EB0800BA
:100230000028B8BF4042B0F57A7F14DD2B78FBB1BF
:10024000B36813F480530BD12B70F9F709FEF9F75B
:10025000D5FDF3F795FF2269A1686079F9F72EF8CB
:10026000F9F772FA8046F4F701FBF4F747FB002830
:10027000D4D0FAF7DCFEF7F70FFEF9F74DFECDE725
:10028000B368DB04ECD5F9F761F92F70F3F778FF69
:10029000F9F7C6FDE4E700BFFC0E002000080140AE
:1002A00008000020A80E002000100140000C0140B2
:1002B0002DE9F843C1F30A57A7F2FF35132D0B467A
:1002C0000446864611DC002D42DB264F47FA05F531
:1002D00001EA050757EA000E1DD101F00045C2E909
:1002E000000170462946BDE8F883332D1FDC4FF02E
:1002F000FF35A7F2134725FA07F710EA070C1FD0BE
:100300000D4620EA0704C2E900450B462246FEF7E7
:10031000D1FDBDE8F8834FF0000821EA0509C2E9E4
:1003200000894B464246FEF7C5FDBDE8F883002430
:1003300001F00045C2E9000120462946BDE8F883E6
:1003400001F00045C2E9000160462946BDE8F88396
:10035000002001F0004106460F4620461946C2E93A
:100360000067C0E7FFFF0F00C1F30A522DE9F04715
:10037000A2F2FF36132E0B4604460D46074688466A
:10038000824622DC002E4FDB3D4A42FA06F901EAA2
:10039000090202431ED038A3D3E90023FEF78CFDE7
:1003A00000220023FFF7CAF950B1002D04DD4FF4FD
:1003B000801343FA06F6B0444FF0000A28EA090514
:1003C000544629462046BDE8F087332E06DDB6F5B3
:1003D000806F3DD019462046BDE8F0874FF0FF39C9
:1003E000A2F2134229FA02F910EA090FF2D022A36D
:1003F000D3E90023FEF760FD00220023FFF79EF9FA
:100400000028DDD0002D09DD142E2FD00123C6F1E8
:10041000340603FA06F6371928BF9844454627EAFA
:10042000090A54462946CDE713A3D3E90023FEF772
:1004300043FD00220023FFF781F90028C0D0002DE2
:100440000FDB55EA040709D04FF0000A0D4DB7E75E
:1004500002460B46FEF730FD0446BCE7BA463D4671
:10046000AEE74FF0000A4FF00045A9E705F101089B
:10047000D4E700BFAFF300809C7500883CE4377E72
:10048000FFFF0F000000F03FC1F30A522DE9F843CF
:10049000A2F2FF36132E0B4604460D468846074649
:1004A0001DDC002E40DB3C4A864642FA06F901EA92
:1004B0000902024318D036A3D3E90023FEF7FCFC5F
:1004C00000220023FFF73AF920B1002D42DB00277C
:1004D00028EA09053C4629462046BDE8F883332E24
:1004E00006DDB6F5806F2FD019462046BDE8F883AB
:1004F0004FF0FF39A2F2134229FA02F910EA090F6C
:10050000F2D023A3D3E90023FEF7D6FC0022002378
:10051000FFF714F90028DDD0002D21DB454627EA3E
:1005200009073C462946D7E719A3D3E90023FEF77C
:10053000C3FC00220023FFF701F90028CAD0002DD8
:1005400019DB00273D46C5E702460B46FEF7B4FC23
:100550000446CAE74FF4801343FA06F6B044B6E700
:10056000142E10D00123C6F1340603FA06F637190B
:1005700028BF9844D2E725F00042084B224318BF19
:100580001D460027A6E705F10108C7E7AFF3008085
:100590009C7500883CE4377EFFFF0F000000F0BF31
:1005A0002DE9F0438BB004460D4600F079F8374B47
:1005B000804693F900608946731C0DD022462B4675
:1005C00020462946FFF7C4F830B900220023204610
:1005D0002946FFF7B3F820B1404649460BB0BDE8C5
:1005E000F0832B4B0890CDE90245CDE904450193FA
:1005F000DEB94FF06046274F2046294600220023EF
:10060000CDE90667FFF772F8002837D00223009380
:10061000684600F039FAC8B1089BE3B9DDE90689FC
:10062000404649460BB0BDE8F0834FF00008DFF8C4
:100630006C902046294600220023CDE90689FFF769
:1006400055F868B102239E420093E1D100F024FAEC
:1006500022230360E0E700F01FFA089B0360DDE758
:100660000123022E00930BD100F016FA2123036020
:10067000094800F00BFACDE90601CDE7012300930C
:10068000684600F001FA0028F2D1EDE7600500208D
:10069000400C0108FFFFEFC7440C01080000F0FF09
:1006A0002DE9F04FB1F5801F85B006460F460B4689
:1006B0005ADA024621F00044224300F0F880002973
:1006C000C0F27A810022D64BFEF7A8FD0B46D54A30
:1006D000064693420F466FF0350C4ADCC3F3130510
:1006E00005F5152E0EF6647E0EF4801E8EF07F52F8
:1006F00082F440121C1542EA0507A4F2FF34644458
:100700000022C94B3046394604EB1E54FEF7D2FB9B
:10071000AB1CC3F31303022B82468B464FF000023F
:1007200030DC0023FEF7E2FF002800F0C980002C37
:1007300000F04B812046FEF70BFDA5A3D3E9002373
:1007400006460F46FEF76AFDA3A3D3E9002304463D
:100750000D4630463946FEF761FD02460B462046FF
:100760002946FEF7A9FB0AE0AE4A4FF0000C93427F
:10077000B4DD32463B4630463946FEF79DFB05B0B8
:10078000BDE8F08F4FF08043FEF796FB02460B4624
:1007900050465946FEF76CFE064620460F46FEF7C9
:1007A000D7FC3246CDE900013B4630463946CDE91B
:1007B0000267FEF733FD02460B4680468946FEF788
:1007C0002DFD87A3D3E9002306460F46FEF726FD3D
:1007D00085A3D3E90023FEF76FFB32463B46FEF7C5
:1007E0001DFD83A3D3E90023FEF766FB32463B469B
:1007F000FEF714FD80A3D3E90023FEF75DFB42461C
:100800004B46FEF70BFD7EA3D3E9002380468946C5
:1008100030463946FEF702FD7BA3D3E90023FEF7FD
:100820004BFB32463B46FEF7F9FC79A3D3E90023A4
:10083000FEF742FB32463B46FEF7F0FC0B46024613
:1008400049464046FEF738FBA5F5C223C5F5D72536
:10085000A3F27A4351351D43002D8046894656DD6B
:100860000022724B50465946FEF7D8FC52465B4672
:10087000FEF7D4FC06460F46002C68D132463B46B4
:1008800040464946FEF718FBDDE90223FEF7C6FCA9
:1008900002460B4630463946FEF70CFB02460B4635
:1008A00050465946FEF706FB05B0BDE8F08F002222
:1008B000002300205E49FEF7DBFD05B0BDE8F08FA8
:1008C00055A3D3E9002350465946FEF7A7FC02463C
:1008D0000B4600205549FEF7EDFA524606460F46F4
:1008E0005B4650465946FEF799FC02460B46304699
:1008F0003946FEF793FC06460F46002C40F09A80DE
:1009000002460B4650465946FEF7D4FA37E7002C0C
:1009100000F0A4802EA3D3E90023DDE90001FEF757
:100920007DFC42464B4604460D4650465946FEF76E
:10093000C1FADDE90223FEF771FC27A3D3E9002306
:1009400006460F46DDE90001FEF768FC21E020A322
:10095000D3E90023DDE90001FEF760FC32463B46A7
:1009600004460D4640464946FEF7A6FADDE9022355
:10097000FEF754FC18A3D3E9002380468946DDE93D
:100980000001FEF74BFC02460B4640464946FEF787
:1009900093FA02460B4630463946FEF78BFA52462A
:1009A0005B46FEF787FA02460B4620462946FEF7CD
:1009B00081FA05B0BDE8F08F02460B46FEF77AFAE1
:1009C00000220023FEF754FDD9E600200021D6E6E0
:1009D0000000E0FE422EE63F763C7935EF39EA3DF5
:1009E00044523EDF12F1C23FDE03CB966446C73F5E
:1009F000599322942449D23F935555555555E53F77
:100A00009FC678D0099AC33FAF788E1DC571CC3F81
:100A100004FA97999999D93F555555555555D53F4C
:100A200000005043FFFFEF7F0000F03F0000E03F79
:100A3000000050C32046FEF78BFB0FA3D3E9002331
:100A400080468946FEF7EAFB0DA3D3E9002304465E
:100A50000D4640464946FEF7E1FB9AE702460B4643
:100A600050465946FEF726FADDE90223FEF7D6FB8B
:100A700014E700BFAFF300800000E0FE422EE63F27
:100A8000763C7935EF39EA3D002070470020014976
:100A9000704700BF0000F87F014B1868704700BF27
:100AA0003001002064000000C80000009001000038
:100AB0002003000040060000800C00000019000028
:100AC000003200000064000050C3000088130000E2
:100AD0000080000000000000000000000000000096
:100AE0000101C80080080000320354007200690050
:100AF0006E0061006D006900630020005300740007
:100B00006500700070006500720020004400650000
:100B1000760069006300650020002603540072001F
:100B200069006E0061006D00690063004D006F0098
:100B3000740069006F006E002000430074006C00B8
:100B40000403090409024300020100C03209040041
:100B5000000102020100052400100105240100012A
:100B6000042402020524060001070582030800FF91
:100B700009040100020A000000070503024000000A
:100B80000705810240000012011001020000403CF4
:100B90002A0001012D0102030101010100010000F1
:100BA0000001000000010000000000010000000042
:100BB0000000000000000000000101010000000032
:100BC0000000000000000100000000000001010121
:100BD0000001010001010000000000000000000011
:100BE0000000000000000000000000000000000005
:100BF00000000000000000000000000000000000F5
:100C000000000001010100000100010101000000DD
:100C100000000000000000000002000000000000D2
:100C2000010000000001020304010203040607089A
:100C300009020406083132343056313435000000E0
:080C40006C6F6700000000006A
:040C4800F8B500BF3C
:040C4C00F8B500BF38
:080C5000B8F1FF7F0100000074
:100C5800350C010800010000000102000008000036
:100C68000100000002000000000000000000000079
:100C7800000000000000000000000000000000006C
:100C8800000000000000000000000000000000005C
:100C9800000000000000000000C201000000080081
:100CA800D99C0008CD9A0008DD990008F199000840
:100CB800F3990008519A0008759A0008A99B000842
:100CC800B59B0008C19B0008000000004000000020
:100CD800870B010812000000440B010843000000C4
:100CE800400B0108040000001A0B01082600000050
:100CF800E80A010832000000140100201A00000070
:100D080001000000B5E50008B9990008B5E500083C
:100D1800B5E50008B5E50008B5E50008B5E5000843
:100D2800B5E50008D199000804010000B5E5000800
:100D3800B5E50008A19A0008B5E50008B5E5000882
:100D4800B5E50008B5E50008AD990008B5E5000867
:100D5800B5E50008B5E50008B5E50008B5E5000803
:100D6800B5E500081A0354004D0043005300540031
:100D780045005000000000000000000000000000D6
:100D880038010020000000000000000024040020BA
:100D98008C040020F4040020000000000000000083
:100DA800000000000000000000000000000000003B
:100DB800000000000000000000000000000000002B
:100DC800000000000000000000000000000000001B
:100DD800000000000000000000000000000000000B
:100DE80000000000000000000000000000000000FB
:100DF80000000000000000000000000000000000EB
:100E080000000000000000000000000000000000DA
:100E180000000000000000000000000000000000CA
:100E280000000000000000000000000000000000BA
:100E380001000000000000000E33CDAB34126DE657
:100E4800ECDE05000B0000000000000000000000C0
:100E5800000000000000000000000000000000008A
:100E6800000000000000000000000000000000007A
:100E7800000000000000000000000000000000006A
:100E8800000000000000000000000000000000005A
:0411B8000100000032
:04000005080041109E
:00000001FF
